:020000040000FA
:06000000E1EFB2F0120076
:020006001200E6
:060008004CEF9CF0120019
:02000E000203EB
:0100100003EC
:020011000100EC
:020013000000EB
:06001800BBEF3DF01200F9
:02001E000B00D5
:10002000CA670100000B000040000000AF6701003C
:10003000400B00001B000000AA670100F909000046
:100040000500000075670100C805000035000000CC
:1000500030670100630A000045000000CD66010022
:10006000000A000063000000626601008E090000C3
:100070006B00000013000000FD07000002000000FC
:1000800037660100C80700002B0000002066010051
:10009000E80A00001700000011000000FE04000044
:0400A000020000005A
:0C00A40066EC2AF0EDEC25F001340FE2D0
:1000B00000501008270E01540AE2100EF36EFD0ED8
:1000C000F3CFDBFF270EF36EFE0EF3CFDBFF4BEC1F
:1000D0002BF003E3F36AF46A4ED0DE6ADD6AEDECDE
:1000E00025F0013430E20050B808240E01542BE210
:1000F000B80E035D240E04590DE2EDEC25F0B80EA8
:10010000005E240E015A026A036A01AE05D002683D
:10011000036802D049EC26F0280E56EC29F02C0E8C
:100120000026010EF9EC2BF0580E2B6E020E39EC66
:1001300025F0B80EF36EFD0EF3CFDBFF240EF36E49
:10014000FE0EF3CFDBFF4BEC2BF00FE249EC26F079
:10015000B40E56EC29F05C0E0026120EF9EC2BF0D2
:10016000B80E2B6E240E39EC25F095EC24F000C06F
:10017000F3FF01C0F4FF020EE15C02E2E16AE55226
:10018000E16E10EF23F00BEC23F00E0EE1260BECEA
:1001900025F063EC26F0040E02C0DBFF050EA9EC8F
:1001A00024F029EC27F0080E02C0DBFF090EC4EC96
:1001B00024F00A0E00C0DBFF0B0E01C0DBFF0C0EAB
:1001C00002C0DBFF0D0E03C0DBFFCDC9E6FFCEC9C9
:1001D000E6FFCFC9E6FFD0C9E6FFC70EE66EFF0E09
:1001E000E66E000EF7EC2DF0E5EC74F0DBEC2CF095
:1001F0006EEC27F0BF0EE66EFF0EE66E000E53ECBF
:100200002BF014EC26F09DEC28F053EC2BF0A5EC31
:1002100026F04BEC2CF0D9C9E6FFDAC9E6FF4BEC2F
:100220002CF009019F51DDEC2DF00901E051DDECCE
:100230002DF0E3C900F0016A00BE016872EC23F002
:100240009DEC28F0D6EC22F00901E951DDEC2DF00F
:1002500030EC27F001AE02D002680368040E85EC92
:1002600025F0FDE1FEEC2BF09DEC28F04EEC2CF09F
:10027000D4EC74F0046E090EC2EC2AF09AEC23F070
:10028000080EDBCF02F0090EDBCF03F0A3EC21F068
:10029000DFEC2CF00FEC28F008EC28F0A3EC21F0B8
:1002A000DFEC2CF077EC23F0BBEC2AF02CEC24F004
:1002B000DFEC2CF06A0EE66E090EE66E42EC2DF0D5
:1002C000006E0E0EE15C02E2E16AE552E16E005062
:1002D00010EF23F002EC2CF0010EDB6A020EDB6A59
:1002E000DF6ADF50006E016AFD0EDBCF02F0FE0E0A
:1002F000DBCF03F003500118E8AE02D0013402D086
:1003000028EC26F001E28ED06AEC26F0E3EC27F030
:1003100004BE05683BEC2AF024C003F025C004F0BD
:1003200026C005F0C7EC2CF00800F55033E13C0E78
:10033000066E4E0E076E010E086E010EDBCF09F041
:10034000020EDBCF0AF00B6A0ABE0B68E3EC2CF05E
:10035000A2EC2BF073EC8DF024C009F025C00AF05C
:1003600026C00BF006502424F36E07502520F46EAF
:1003700008502620A2EC29F09BEC2BF00BE16AEC54
:1003800026F0E3EC27F004BE056867EC23F0F55097
:10039000DF6E41D0DF50006E016AFD0EDB500018A9
:1003A0003AE1FE0EDB50011836E17F0E0501C85D13
:1003B00023E1010EDBCFE6FF020EDBCFE6FFAC0E42
:1003C000E66EFF0EE66E000EF7EC2DF078EC2CF0EA
:1003D00016EC28F0AA0EE66EFF0EE66E000EE66E34
:1003E000030EDBCFE6FF040EDBCFE6FF46EC22F088
:1003F00016EC28F082EC29F0A390A392010EDBCF3B
:10040000E8FA020EDBCFE9FA15D85CD90A01E869EF
:10041000E969A382A380010EDB2A020E01E261D703
:10042000DB2A5FD7050EE15C02E2E16AE552E16E8C
:1004300010EF23F002EC2CF00A01800EE9154DE1DB
:10044000CEEC26F008BE0968A1EC23F00EBE0F68C2
:10045000E0EC23F0030E00C0DBFF040E01C0DBFF65
:10046000D950030FBFEC2CF0550EEE1809E1010E28
:10047000ED1806E1DF6A56EC2BF004AE04D002D092
:10048000000E16D1056867EC23F0F5CFE7F8030EF0
:10049000DB6A040EDB6A030EDBCF00F0040EDBCF59
:1004A00001F0080E12EC26F030E2DAEC26F007BE7E
:1004B00008689DEC25F0030EDBCF09F0040E47EC35
:1004C00025F0030EDBCFE9FF040E5AEC27F0030EF4
:1004D000DB2A040EE0E3DB2ADED7010E6014DF6EB8
:1004E0000F0E65140801E76F66CFE8F867CFE9F8EB
:1004F00068CFEAF869CFEBF86ACFECF86BCFEDF88C
:100500006CCFEEF86DCFEFF8609EDF5001E0CFD0FA
:10051000540E0801EB5D01E0CAD0ECC803F0026A9A
:10052000ED5168EC25F02CE237EC27F0026A02343A
:10053000000E021807E6D880400E00549C0E0154AD
:10054000000E02541DE3010EDBCF03F9020EDBCFD8
:1005500004F90901D89004330333D89004330333EA
:100560000351095D04510A5904E203C909F904C998
:100570000AF90551035D0651045902E277EC27F0B0
:100580000F0E0801E915036E026AEA5168EC25F0C6
:1005900001E38DD037EC27F0000E005C0F0E015800
:1005A00001E385D0010EDBCF15F9020EDBCF16F982
:1005B0000901D00ED8801557070E16573E51135D0E
:1005C0003F51145907E33E51135D006E14513F55DE
:1005D000016E21D01DEC28F0086A096A010E0A6E2E
:1005E0000B6A3EC90CF03FC90DF00E6A0F6A0C5041
:1005F000085C046E0D500958056E0E500A58066EC0
:100600000F500B58076E045000260550012206506B
:10061000022207500322A9EC2BF013C93EF914C99A
:100620003FF937EC27F0026A036ADEEC25F0EEECC6
:1006300024F0163521E215510008000E16551CE273
:1006400030EC27F001AE02D002680368DEEC25F042
:10065000040EBEEC29F0EEEC24F030EC27F001AEF5
:1006600002D00268036800506227015063230250E1
:100670006423035065231BD01EEC27F001AE02D08B
:1006800002680368DEEC25F0080EBEEC29F0EEEC03
:1006900024F01EEC27F001AE02D00268036800507F
:1006A0006627015067230250682303506923010E17
:1006B000006E050EE15C02E2E16AE552E16E005077
:1006C00010EF23F00BEC23F00E0EE1260A01800E52
:1006D000E91570E1CEEC26F008BE0968A1EC23F024
:1006E0000EBE0F68E0EC23F068EC24F0F5EC22F08D
:1006F000900E0016050E0116900E001805E1050E6D
:10070000011802E1020E1BD0F5EC22F0900E00164B
:10071000060E0116900E001805E1060E011802E102
:10072000030E0DD0F5EC22F0500E0016050E01164A
:10073000500E001816E1050E011813E1040EDF6ECD
:100740000F0EE76E040EDBCF00F0050EE75000162B
:10075000016A010E00C0DBFF56EC2BF004AE04D0A2
:1007600002D0000E03D3056867EC23F0F5CFE7F85D
:10077000040EDB6A050EDB6AF5EC22F0080E12ECC3
:1007800026F041E2DAEC26F007BE08689DEC25F081
:10079000040EDBCF09F0050E47EC25F0040EDBCF8D
:1007A000E9FF050E5AEC27F0040EDB2A050EE4E300
:1007B000DB2AE2D7070E0F015015DF6EE00E52154F
:1007C000E00BE838E840006E010E5115080DF350BB
:1007D0000024E76E010EE7CFDBFF0F0E5515080171
:1007E000E76F56CFE8F857CFE9F858CFEAF859CF76
:1007F000EBF85ACFECF85BCFEDF85CCFEEF85DCFBD
:10080000EFF80F01509F020EDF5C01E0A4D0010E53
:10081000DB500E0A01E185D0070A31E00E0A01E043
:10082000A4D20801E8AB08D0E60E09018E6F8F6BE9
:1008300009010A0E906F05D009018E6B8F6B0901BB
:10084000906BE9C817F9100E090117150AE00901A4
:100850009951800B06E1000E09013E6F3F6B136F4B
:10086000146B0801EF51000801E37FD2F00EEF5D39
:1008700001E37BD2280EEF5D0901C06F76D2600ED6
:10088000090117150BE1FF0E0801ED5D07E0ED51C1
:10089000000804E2ED5109010B6F0C6BEEC803F088
:1008A000026A0801EF51C6EC2AF063EC26F0D95039
:1008B000020FBFEC2CF0FF0EEE1802E1FF0EED1858
:1008C00001E153D2020EDBCF28F0030EDBCF29F07B
:1008D00009010D51285C006E0E512958016E29EC5A
:1008E00027F09AEC23F0D890015004E60A0E005C41
:1008F000000E015802E3010E0AD09AEC23F00134F5
:1009000008E30050F608FF0E015403E3020E3D6FAA
:1009100001D03D6B020EDBCF0DF9030EDBCF0EF9DC
:1009200024D2E8C801F0006A0801E9510901002455
:10093000136F000E0120146F0801ED51280808E222
:10094000F00EED5D05E2280EED5D0901C16F0DD2DF
:100950000901C16B0AD2030EDF5C35E1010EDB50E9
:100960000F0A01E002D20901B55101E1FED10F0EDB
:100970000801EB15300F0901AE6F0801EB390F0BC1
:10098000300F0901AF6F0F0E0801EA15300F090192
:10099000B06F0801EA390F0B300F0901B16F0F0E6C
:1009A0000801E915300F0901B26F0801E9390F0B91
:1009B000300F0901B36F0F0E0801E815300F090160
:1009C000B46FB56BD2D1040EDF5C01E078D1090EB3
:1009D000FEC0DBFF010EDB500F0A01E125D1010A49
:1009E00001E1E5D0090A01E19BD0030A6CE0020AAB
:1009F00001E0BBD1FF0E0801E85D01E1B6D199EC41
:100A000028F001E1B2D164EC28F0CCEC25F0FDE156
:100A10000801E9390F0B000100108E6F01C08FF043
:100A20003EEC27F000010010966F01C097F0A1EC9A
:100A300027F0CCEC25F0FDE10801EC390F0B0001AB
:100A400000109E6F01C09FF045EC27F000010010E0
:100A5000A66F01C0A7F00801EE51006E016A040EF6
:100A6000CCEC25F0FDE10801EF390F0B000100107F
:100A7000AE6F01C0AFF0090EDB50FC0B3C0803E188
:100A80003F0EFE6F72D1090EDB50FC0B01E16DD100
:100A9000090EDB50030B010FE76E080EE7CFDBFFFB
:100AA000DB50030803E1090EDB6A06D1080EDBCF39
:100AB000E6FF090EDB50FC0BE552E710E76E090E6E
:100AC000E7CFDBFFF9D0FF0E0801E85D01E14DD172
:100AD00099EC28F001E149D1080EDB6A070EF36EAC
:100AE000080EDBCFF4FFF350F45C13E2080EDB508A
:100AF000EA6AE80FE96E080EEA22EF50E66E080E89
:100B0000DB50FFEC22F0E552E750EF6E080EDB2AD7
:100B1000E5D7090EDB84FAEC26F001E283D07DD024
:100B2000FF0E0801E85D01E120D199EC28F001E118
:100B30001CD164EC28F0CCEC25F0FDE10801E9398A
:100B40000F0B00010010B66F01C0B7F03EEC27F0AC
:100B500000010010BE6F01C0BFF0A1EC27F0CCEC8B
:100B600025F0FDE10801EC390F0B00010010C66F04
:100B700001C0C7F045EC27F000010010CE6F01C0A6
:100B8000CFF00801EE51006E016A040ECCEC25F0A6
:100B9000FDE10801EF390F0B00010010D66F01C015
:100BA000D7F0090EDB86FAEC26F03CE336D0FF0ED8
:100BB0000801E85D01E1D9D099EC28F001E1D5D038
:100BC00064EC28F0CCEC25F0FDE10801E9390F0BCD
:100BD00000010010DE6F01C0DFF03EEC27F00001E5
:100BE0000010E66F01C0E7F0A1EC27F0CCEC25F097
:100BF000FDE10801EC390F0B00010010EE6F01C0A0
:100C0000EFF045EC27F000010010F66F01C0F7F09F
:100C1000090EDB88FAEC26F005E33F0EF36E090EB1
:100C2000F3CFDBFF090E48D0FF0E0801ED5D01E1B7
:100C30009CD099EC28F001E198D0ED51026E036A46
:100C4000040ED89002360336E804FBE10801EE39C1
:100C50000F0B00010210006E0A0E00C0DBFF0B0E2E
:100C600003C0DBFF0F0E0801EE15036E026AEF51A1
:100C700000010210006E0C0E00C0DBFF0D0E03C061
:100C8000DBFF24EC28F00A0EDB5000240001606F2B
:100C90000B0EDB50000101200001616FD890613321
:100CA0006033090EDB8AFAEC26F005E33F0EF36EA3
:100CB000090EF3CFDBFF090EDBCFFEF056D0050E99
:100CC000DF5C53E1010EDB50070A4FE1EDC800F095
:100CD000016A026A036A040E2BEC28F0FDE1ECC8FD
:100CE00004F0056A066A076A040E1F0B03E0F1ECC4
:100CF00024F0FDE1045000120550011206500212CA
:100D000007500312EBC808F0096A0A6A0B6A0C0E56
:100D10001F0B07E0D890083609360A360B36E8066E
:100D2000F9E108500012095001120A5002120B504A
:100D30000312EAC80CF00D6A0E6A0F6A140E1F0B3C
:100D400007E0D8900C360D360E360F36E806F9E17E
:100D500000500C1009010F6F01500D10106F025060
:100D60000E10116F03500F10126F010E006E0E0E59
:100D7000E15C02E2E16AE552E16E005010EF23F01F
:100D800002EC2CF007EC2CF07F0E0501C85D04E0AE
:100D9000200EC85D01E0B0D0030EE66ED3EC27F064
:100DA00068EC2CF0A60EE66EFF0EE66E000EF4EC7C
:100DB00025F005E0010EF36E020EF3CFDBFFA30E6C
:100DC000E66EFF0EE66E000EF4EC25F005E0010E77
:100DD000F36E030EF3CFDBFF090118A11ED0030E43
:100DE000DB500CE00A01635109E00A01645106E19D
:100DF00094EC2BF0CD0EB0EC2BF01891020EDB50E2
:100E00000CE062EC27F0C4EC1CF006EC2EF00009BC
:100E100002E041EC5AF009011891090118A322D00F
:100E2000030EDB5010E00A0163510DE00A0164512A
:100E30000AE194EC2BF0CF0EA1EC26F07FEC0EF043
:100E4000A7EC27F01893020EDB500CE062EC27F0C1
:100E500054EC0EF006EC2EF0000902E041EC5AF0E2
:100E600009011893090118A90CD00A01630509E1C9
:100E70000A01645106E194EC2BF0CE0EB0EC2BF09D
:100E80001899090118A524D00A01630521E10A0176
:100E900064511EE1020EF36E040EF3CFDBFFD00EA1
:100EA000E66EE66A040EDBCFE6FFAAEC27F069ECFB
:100EB00028F0DBCFE6FFC3EC00F0E55269EC28F048
:100EC000DB50020802E02FEC2EF00901189518897A
:100ED000090118A711D00A0163050EE10A01645146
:100EE0000BE1020EE66EC3EC00F0E552020802E0F0
:100EF0002FEC2EF009011897050EE15C02E2E16A81
:100F0000E552E16E10EF23F03BDF010C0BEC23F018
:100F1000070EE1260601EF51DE6EDD6AF051E66E46
:100F2000D950020F76EC25F0F151E66ED950040F3E
:100F300076EC25F04B0E0701CB5D38E177EC23F022
:100F4000013418E28DEC26F015E24CEC27F0033466
:100F500002E2C4EC27F003E3006A016A09D077ECEF
:100F600023F0A8EC29F092EC26F0FDE197EC26F0B6
:100F700063EC26F0F5EC22F0013418E28DEC26F05B
:100F800015E2BBEC2AF0033402E2C4EC27F003E3E1
:100F9000006A016A09D0F5EC22F0A8EC29F092EC85
:100FA00026F0FDE197EC26F068EC24F00901A52B72
:100FB000000EA623A723A823320E0901016A0325E8
:100FC000006E04510122640EE4EC29F028C0A0F95F
:100FD00080EC27F05EEC2BF0D880000E2654000E3B
:100FE0002754000E2854000E295406E30901CD6B46
:100FF000CE6BCF6BD06B2AD00FC900F010C901F0B7
:1010000011C902F012C903F0AAEC2CF080EC27F011
:10101000E8EC2DF0AAEC2CF0E7EC22F0050E005ED7
:10102000000E015A025A035A040E2BEC28F0FDE17F
:1010300000C0CDF901C0CEF902C0CFF903C0D0F98C
:101040000901CD2B000ECE23CF23D023D7EC27F0E0
:1010500027E1320E0901036A0D25026E0E510322AB
:10106000640E2D6E2E6A02C028F003C029F0ABEC8E
:10107000B2F028C002F029C003F0000ED880285436
:10108000000E295403E3006A016A0CD0D1EC2CF065
:10109000A8EC29F092EC26F0FDE197EC26F002D0C6
:1010A000D1EC2CF000C09FF90901000ED8808E55BC
:1010B000000E8F5505E20901998709019D8904D029
:1010C0000901999709019D99600E090117152008DA
:1010D00004E109019985998902D0090199990901C9
:1010E00017A910D0090199BF2ED0998F0901A96BBA
:1010F000AA6BAB6BAC6B010EF8EC24F0F7EC14F0C0
:101100008CD921D0090199AF1ED0999FA5C9A9F901
:10111000A6C9AAF9A7C9ABF9A8C9ACF90901A907D9
:10112000000EAA5BAB5BAC5B010EF8EC24F0D88040
:10113000E40E09011D55570E1E55000E1F55000ED9
:10114000205501E2188386EC15F073D9090199A99D
:10115000E0D0640E006E016A0CEC2CF02D6E01C024
:101160002EF0ABECB2F0060E28C0DBFF0901000E3A
:10117000D8800755000E08553FE2000ED880035571
:10118000000E045539E2000ED8800555000E0655B4
:1011900033E2C6EC22F00CEC2CF02DEC8BF060EC82
:1011A00029F047EC8CF0E3EC8DF028C00BF929C056
:1011B0000CF90901000ED8802854000E29540EE2C3
:1011C00000EC27F004E30901A36BA46B07D06BECE0
:1011D0002DF092EC26F0FDE1EBEC27F0F5EC22F09F
:1011E000013406E28DEC26F003E219EC23F004D082
:1011F000A3C9A1F9A4C9A2F9150E0901945D03E1DF
:10120000040EF8EC24F009019451020808E2010EE2
:10121000946F03C909F904C90AF9FFD861D009011B
:10122000000ED8800355000E04552CE295EC24F0F6
:10123000013428E28DEC26F025E2060EDB50026E2A
:10124000036ADECF04F0DDCF05F003500518E8AEE9
:1012500002D0053404D00450025C0550035812E358
:101260000051066E076ADECF08F0DDCF09F00750A7
:101270000918E8AE02D0093404D00850065C0950C1
:10128000075828E300EC27F02DE2020EDBCF0AF02E
:10129000030EDBCF0BF00B3425E20A500008000EE2
:1012A0000B5420E2020EDBCF0CF0030EDBCF0DF06F
:1012B00009010C50A15D0D50A25914E3020EDBCFC1
:1012C0000EF0030EDBCF0FF009010E50015D0F5041
:1012D000025908E20901020E946F040EF8EC24F0A2
:1012E000020E0DD0020E0901945D0BE00901B80E4B
:1012F000035D240E045905E30901020E946FF8EC16
:1013000024F0060EDBCF00F9A1C901F9A2C902F948
:1013100047D0090100EC27F01CE200EC27F004E3C1
:101320000901A36BA46B07D06BEC2DF092EC26F0B7
:10133000FDE1EBEC27F0F5EC22F0013406E28DEC58
:1013400026F003E219EC23F004D0A3C9A1F9A4C943
:10135000A2F909019451020813E30901100E095D75
:10136000270E0A5903E30901040E02D00901150EE4
:10137000946F040EF8EC24F0020EF8EC24F010D078
:1013800009019951800B0CE09951100B09E1995119
:10139000040B06E099950901040E946F77EC27F091
:1013A0000901000ED8800D55000E0E5516E20601FB
:1013B000ED51000812E2C8C700F0C9C701F0050EE0
:1013C0002D6E2E6AC8C728F0C9C729F0ABECB2F061
:1013D0002450251002E109011887000E006E070E47
:1013E000E15C02E2E16AE552E16E005010EF23F0A9
:1013F000090117BF0DD0400E176F09018E6B8F6B5F
:101400000901906B09010D6B0E6B156B166B000CCF
:10141000179F000C09011885000CA39091EC2AF08D
:1014200013C93EF914C93FF9B1EC25F0A3809BEF35
:101430002AF00BEC23F0100EE126090117A9EFD0DA
:101440000901E35103E1C2EC26F0E9D009015C5146
:101450005D115E115F1107E1ACEC26F0A390B1ECD9
:1014600025F0A380DCD05C0EE96E090EEA6EEE502A
:101470000F5D266EEE501059276EEE501159286EF2
:10148000EE501259296EAAEC2CF0BEECB1F022C03D
:10149000DEFF23C0DEFF24C0DEFF25C0DDFFDD52FE
:1014A000DD5293EC2CF0D890030EEB50000A08E6C6
:1014B000640EEE5C000EEE58000EEE58000EEE5874
:1014C00001E2ADD0A390080E62C9DBFF090E63C92B
:1014D000DBFF0A0E64C9DBFF0B0E65C9DBFF0C0ED8
:1014E00066C9DBFF0D0E67C9DBFF0E0E68C9DBFFA7
:1014F0000F0E69C9DBFF0901B1EC25F0A380605133
:101500000901DB5D006EDC5109016155016E68EC7B
:1015100024F0F5EC22F0026A036A01AE02D0026800
:101520000368640E56EC29F0B1EC29F0F4EC8CF071
:10153000060E26C0DBFF070E27C0DBFFACEC26F053
:101540009AEC23F0D890015002E66EEC28F02BE3E1
:10155000DF5009014027010EDB504123020EDB5012
:101560004223030EDB504323B6EC2BF028504427D4
:1015700029504523080EDB504627090EDB50472330
:101580000A0EDB5048230B0EDB5049230C0EDB50B8
:101590004A270D0EDB504B230E0EDB504C230F0E53
:1015A000DB504D233CD09AEC23F0013438E300505B
:1015B000FF08FF0E015433E3DF5009014E27010EEF
:1015C000DB504F23020EDB505023030EDB50512320
:1015D00028682968040EDBCF2DF0050EDBCF2EF036
:1015E00028EC8DF026500901522727505323080E6E
:1015F000DB505427090EDB5055230A0EDB505623CF
:101600000B0EDB5057230C0EDB5058270D0EDB5012
:1016100059230E0EDB505A230F0EDB505B23100EA6
:10162000E15C02E2E16AE552E16E10EF23F00BECBF
:1016300023F0190EE1260C0EDB6A0D0EDB6A0E0E8E
:10164000DB6A0BEC25F000C0DFFF010E01C0DBFF01
:10165000020E02C0DBFF030EA9EC24F068EC24F0BC
:10166000060E02C0DBFF070EC4EC24F0080E00C01B
:10167000DBFF090E01C0DBFF0A0E02C0DBFF0B0E11
:1016800003C0DBFFD9CFE9FF94EC29F045E219C98B
:1016900000F01AC901F01BC902F01CC903F09CEC50
:1016A0002CF019C926F01AC927F01BC928F01CC94B
:1016B00029F011EC2CF00C0E26C0DBFF25C900F040
:1016C00026C901F027C902F028C903F09CEC2CF0D0
:1016D00025C926F026C927F027C928F028C929F0EE
:1016E00011EC2CF00D0E26C0DBFF31C900F032C921
:1016F00001F033C902F034C903F09CEC2CF031C97D
:1017000026F032C927F033C928F034C929F011EC8A
:101710002CF00E0E26C0DBFF1FEC2BF07CEC2CF027
:10172000F5EC22F071EC26F00050011002100310CD
:1017300007E093EC2CF0D8800A0E49EC2DF003E37F
:1017400018EC2AF0B5D0FE0EDB50740801E0B8D0DA
:1017500018EC2AF0FBEC28F0010EE66EE66A93EC3A
:101760002CF0EECF00F0EECF01F0EECF02F0EFCF95
:1017700003F0E80E2B6E030E2C6EB0EC28F0B0ECEC
:101780002CF08F0EE66EFF0EE66E000E60EC2CF075
:10179000B6EC2DF006EC2BF00C0EC3EC2CF0830E07
:1017A000E66EFF0EE66E000EBAEC28F01DC900F0E2
:1017B0001EC901F01FC902F020C903F002EC2AF093
:1017C000FDEC2CF0FBEC28F00D0EC3EC2CF0730EAE
:1017D000E66EFF0EE66E000EBAEC28F029C900F0A6
:1017E0002AC901F02BC902F02CC903F002EC2AF03F
:1017F0002DC900F02EC901F02FC902F030C903F045
:10180000FBEC28F00E0EC3EC2CF0670EE66EFF0E1C
:10181000E66E000EBAEC28F035C900F036C901F0CA
:1018200037C902F038C903F002EC2AF039C900F0D8
:101830003AC901F03BC902F03CC903F0FBEC28F0C7
:10184000A4EC2AF05E0EE66EFF0EE66E000E33ECA0
:1018500022F046C900F047C901F048C902F049C961
:1018600003F0F4EC2AF04AC900F04BC901F04CC96E
:1018700002F04DC903F0FBEC28F0ADEC2AF04F0E5E
:10188000E66EFF0EE66E000E33EC22F054C900F057
:1018900055C901F056C902F057C903F0F4EC2AF01B
:1018A00058C900F059C901F05AC902F05BC903F0E8
:1018B000FBEC28F0940EE66EFF0EE66E000E28D1CB
:1018C00093EC2CF0150EEECFDBFF160EEECFDBFF08
:1018D000170EEECFDBFF180EEECFDBFF06EC22F08B
:1018E00013E262EC23F010E2DCEC28F0100E2B6E19
:1018F000270E3BEC29F0430EE66EFF0EE66E000E5F
:10190000B0EC21F0B5EC28F0040E1DC9DBFF050E8C
:101910001EC9DBFF060E1FC9DBFF070E20C9DBFF58
:10192000080E21C9DBFF090E22C9DBFF0A0E23C9FD
:10193000DBFF0B0E24C9DBFF150E19C9DBFF160EEA
:101940001AC9DBFF170E1BC9DBFF180E1CC9DBFF12
:1019500006EC22F00DE262EC23F00AE20C0EC3EC7E
:101960002CF02E0EE66EFF0EE66E000E51EC2CF003
:10197000040E29C9DBFF050E2AC9DBFF060E2BC9A1
:10198000DBFF070E2CC9DBFF080E2DC9DBFF090E9C
:101990002EC9DBFF0A0E2FC9DBFF0B0E30C9DBFFA0
:1019A000150E25C9DBFF160E26C9DBFF170E27C94A
:1019B000DBFF180E28C9DBFF06EC22F00DE262EC1B
:1019C00023F00AE20D0EC3EC2CF0220EE66EFF0EA1
:1019D000E66E000E51EC2CF0040E35C9DBFF050E4F
:1019E00036C9DBFF060E37C9DBFF070E38C9DBFF40
:1019F000080E39C9DBFF090E3AC9DBFF0A0E3BC9E5
:101A0000DBFF0B0E3CC9DBFF150E31C9DBFF160EE9
:101A100032C9DBFF170E33C9DBFF180E34C9DBFFF9
:101A200006EC22F00DE262EC23F00AE20E0EC3ECAB
:101A30002CF0190EE66EFF0EE66E000E51EC2CF047
:101A4000040E46C9DBFF050E47C9DBFF060E48C979
:101A5000DBFF070E49C9DBFF080E4AC9DBFF090E91
:101A60004BC9DBFF0A0E4CC9DBFF0B0E4DC9DBFF78
:101A7000150E40C9DBFF160E41C9DBFF170E42C928
:101A8000DBFF180E43C9DBFF06EC22F00EE262EC2E
:101A900023F00BE271EC28F0130EE66EFF0EE66EFB
:101AA000000EECEC2CF0B5EC28F0040E54C9DBFF72
:101AB000050E55C9DBFF060E56C9DBFF070E57C9D9
:101AC000DBFF080E58C9DBFF090E59C9DBFF0A0E00
:101AD0005AC9DBFF0B0E5BC9DBFF150E4EC9DBFFDE
:101AE000160E4FC9DBFF170E50C9DBFF180E51C988
:101AF000DBFF06EC22F00EE262EC23F00BE276EC68
:101B000028F0080EE66EFF0EE66E000EECEC2CF0F0
:101B1000B5EC28F0190EE15C02E2E16AE552E16EF3
:101B200010EF23F00BEC23F0020ECAEC26F0D00EDF
:101B3000EE1801E0AED0ED5001E0ABD0E80EE66E5D
:101B4000FE0EE66E000E04EC29F019C9E6FF1AC974
:101B5000E6FF1BC9E6FF1CC9E6FF00EC22F01DC929
:101B6000E6FF1EC9E6FF1FC9E6FF20C9E6FF00EC3D
:101B700022F021C9E6FF22C9E6FF23C9E6FF24C9F6
:101B8000E6FF00EC22F025C9E6FF26C9E6FF27C9DB
:101B9000E6FF28C9E6FF00EC22F029C9E6FF2AC9C2
:101BA000E6FF2BC9E6FF2CC9E6FF00EC22F02DC9A9
:101BB000E6FF2EC9E6FF2FC9E6FF30C9E6FF00ECBD
:101BC00022F031C9E6FF32C9E6FF33C9E6FF34C966
:101BD000E6FF00EC22F035C9E6FF36C9E6FF37C95B
:101BE000E6FF38C9E6FF00EC22F039C9E6FF3AC942
:101BF000E6FF3BC9E6FF3CC9E6FF00EC22F040C926
:101C0000E6FF41C9E6FF42C9E6FF43C9E6FF00EC33
:101C100022F0A4EC2AF0DFEC2CF046C9E6FF47C91D
:101C2000E6FF48C9E6FF49C9E6FF00EC22F04AC9D1
:101C3000E6FF4BC9E6FF4CC9E6FF4DC9E6FF00ECE5
:101C400022F04EC9E6FF4FC9E6FF50C9E6FF51C971
:101C5000E6FF00EC22F0ADEC2AF0DFEC2CF054C9EA
:101C6000E6FF55C9E6FF56C9E6FF57C9E6FF00EC97
:101C700022F058C9E6FF59C9E6FF5AC9E6FF5BC919
:101C8000E6FF00EC22F06C0EE66E090EE66E5CECF0
:101C900024F0FE0EDB50DBEC27F002E2E16AE552B5
:101CA000E16E005010EF23F00BEC23F0E652FE0E35
:101CB000DB500FE00601F3B50CD0ADEC29F003E0EA
:101CC0007EEC23F008E1BEEC28F003E07EEC23F08C
:101CD00002E1000E11D0E8EC2AF004E07DEC25F0E2
:101CE000200901D0650EDF6E0601006BDFCFE6FF35
:101CF0009EDCE55206EC2DF0E55210EF23F00BECE4
:101D000023F0030ECAEC26F0D00EEE1811E1ED50D0
:101D10000FE1FE0EDB5005E081EC25F0AAEC27F088
:101D200020D089EC27F0AAEC27F0020829E026D081
:101D3000ECEC2AF005E08CEC25F0EF50200901D006
:101D4000650EE76E020EE7CFDBFFD5EC29F0020E41
:101D5000DBCFE6FF6CDCE552FE0EDB500BE03FEC28
:101D60002EF0EAEC29F00CEC2DF071EC2DF0F4ECF7
:101D70002CF006D012EC2EF03FEC2EF02FEC2EF0D3
:101D8000010E006E030EE15C02E2E16AE552E16ED3
:101D9000005010EF23F066EC2AF0FE0EDBCFE6FFDA
:101DA0007CEC31F0E552E76EFE0EE7CFDBFF8BEC0B
:101DB0002CF003E078EC26F003D0C80E006E016A28
:101DC0000BEC2AF0090117515EEC2AF0A7EC22F087
:101DD0000901995177EC2DF009019D5177EC2DF017
:101DE00009019451DDEC2DF00DC9E6FF0EC9E6FFA7
:101DF0004BEC2CF015C9E6FF16C9E6FF4BEC2CF0B6
:101E00008DEC27F000EC22F080EC28F04BEC2CF06D
:101E100085EC28F04BEC2CF08AEC28F04BEC2CF005
:101E20000BC9E6FF0CC9E6FF4BEC2CF007C9E6FF37
:101E300008C9E6FF4BEC2CF0A3C9E6FFA4C9E6FFF6
:101E40004BEC2CF0A1C9E6FFA2C9E6FF4BEC2CF04D
:101E50000701CA51DDEC2DF0B2EC27F002E1010ED2
:101E600002D0FE0EDB50DBEC27F002E2E16AE55225
:101E7000E16E005010EF23F00BEC23F0E150FA0F6D
:101E8000BFEC22F00AE08CEC25F0EF5006E0F1EC1C
:101E900029F0BAEC25F096EC27F0FE0EDB5006E0B8
:101EA00081EC25F078DFE552E552E552010E10EFA6
:101EB00023F066EC2AF0E8EC2AF009E07DEC25F04E
:101EC00006E0FFEC24F0BAEC25F096EC27F00601D2
:101ED000F3B50CD0ADEC29F003E07EEC23F008E183
:101EE000BEEC28F003E07EEC23F002E1000ECFD040
:101EF000FE0EDB5002E093EC23F08FEC28F009019A
:101F00001751E66EE66AC40EE66EFE0EE66E000E31
:101F1000A7EC22F08DEC27F0BE0EE66EFE0EE66E0C
:101F2000000EFFEC29F0DBEC2CF01DEC28F0FEECB1
:101F30002BF0B90EE66EFE0EE66E000EDCEC22F023
:101F40003EC900F03FC901F0026A036AFEEC2BF0C3
:101F5000B40EE66EFE0EE66E000EDCEC22F0090119
:101F6000E951E66EE66AAF0EE66EFE0EE66E000E14
:101F700038EC29F082EC29F07F0E0501C85D35E1CF
:101F80008FEC28F00901E051E66EE66AA70EE66ED6
:101F9000FE0EE66E000E38EC29F06EEC27F0A10E76
:101FA000E66EFE0EE66E000E68EC2BF014EC26F0EA
:101FB0009B0EE66EFE0EE66E000E68EC2BF0A5ECB6
:101FC00026F0950EE66EFE0EE66E000E38EC29F059
:101FD000D9C9E6FFDAC9E6FF8F0EE66EFE0EE66EA1
:101FE000000E38EC29F082EC29F08FEC28F066C066
:101FF000E6FF67C0E6FF880EE66EFE0EE66E000E98
:10200000A7EC22F068C0E6FF69C0E6FF830EE66E2B
:10201000FE0EE66E000EA7EC22F06AC0E6FF6BC073
:10202000E6FF7D0EE66EFE0EE66E000EA7EC22F0D9
:1020300000016C51E66EE66A780EE66EFE0EE66E04
:10204000000EA7EC22F000016D51E66EE66A730EF9
:10205000E66EFE0EE66E000EA7EC22F000016E5159
:10206000E66EE66A6D0EE66EFE0EE66E000EA7ECFC
:1020700022F00001FE51E66EE66A680EE66EFE0E84
:10208000E66E000EA7EC22F082EC29F0010EDBECEC
:1020900027F002E2E16AE552E16E005010EF23F012
:1020A00066EC2AF01FEC2BF068EC2CF0090199A5E6
:1020B0003FD009019451040A10E0060A08E0030A1F
:1020C00012E15F0EE66EFE0EE66E000E11D0490EB6
:1020D000E66EFE0EE66E000E0BD03B0EE66EFE0EBA
:1020E000E66E000E05D02A0EE66EFE0EE66E000EBF
:1020F000A3EC28F0FDEC2CF0A3EC21F0220EE66E10
:10210000FE0EE66E000EDCEC22F0940EE66EFF0E84
:10211000E66E000EA3EC28F0040E0901945D1EE0AB
:10212000CDEC23F0190EE66EFE0EE66E000E14D016
:10213000060EE66EFE0EE66E000EA3EC28F0090118
:10214000100E035D270E045909E2CDEC23F0F60EC4
:10215000E66EFD0EE66E000E7DEC2DF0D7EC27F05E
:102160001CE1A3C9E6FFA4C9E6FFEC0EE66EFD0E76
:10217000E66E000E38EC29F0A1C9E6FFA2C9E6FF21
:10218000E80EE66EFD0EE66E000E38EC29F0E40E69
:10219000E66EFD0EE66E000E27D0A3C900F0A4C9BE
:1021A00001F0040ECCEC25F0FDE1F1EC2DF0EC0E8D
:1021B000E66EFD0EE66E000ED6EC22F0A1C900F030
:1021C000A2C901F0040ECCEC25F0FDE1F1EC2DF0FC
:1021D000E80EE66EFD0EE66E000ED6EC22F0E00E86
:1021E000E66EFD0EE66E000EA3EC28F0020EE66E23
:1021F000E66A03C900F004C901F0026A036A80ECD0
:1022000028F034EC25F0D80EE66EFD0EE66E000EDA
:1022100082EC24F0020EE66EE66A05C900F006C9FB
:1022200001F0026A036A85EC28F034EC25F0D40E44
:10223000E66EFD0EE66E000E82EC24F0020EE66EF7
:10224000E66A09C900F00AC901F0026A036A8AEC69
:1022500028F034EC25F0D00EE66EFD0EE66E000E92
:1022600082EC24F0CD0EE66EFD0EE66E000EA3ECC1
:1022700028F0D7EC27F01DE1CDC900F0CEC901F060
:10228000CFC902F0D0C903F02DEC26F042EC2CF0BF
:10229000BBEC2DF0B0EC2CF0C50EE66EFD0EE66E3C
:1022A000000EDCEC22F0E40EE66EFD0EE66E000E93
:1022B0002FD0CDC904F0CEC905F0CFC906F0D0C9E2
:1022C00007F02DEC26F026C004F027C005F028C04A
:1022D00006F029C007F0040E1F0B42EC2CF003E0BF
:1022E00085EC25F0FDE1050E2CEC24F0C50EE66E24
:1022F000FD0EE66E000EFFEC29F0086E090EE15EA1
:10230000085068EC2CF0E00EE66EFD0EE66E000E56
:10231000A3EC28F0020EE15C02E2E16AE552E16E14
:1023200010EF23F00BEC23F0FE0EDB500FE0060164
:10233000F3B50CD0ADEC29F003E07EEC23F008E11E
:10234000BEEC28F003E07EEC23F002E1000E05D0A5
:102350000601006BA5DE06EC2DF010EF23F00BEC70
:1023600023F0D5EC29F09CDE3FEC2EF0010E10EFAF
:1023700023F066EC2AF08BEC2CF003E078EC26F0EE
:1023800003D0C90E006E016A0BEC2AF00601F15170
:102390005EEC2AF038EC29F0B2EC27F002E1010EF5
:1023A00002D0FE0EDB50DBEC27F002E2E16AE552E0
:1023B000E16E005010EF23F00BEC23F0E15024EC21
:1023C0002BF0CA0EEE1815E1ED5013E1ECEC2AF0FB
:1023D00009E08CEC25F0EF5005E0F1EC29F032EC4F
:1023E00028F002D00601F16BF1EC29F01C0E93EC01
:1023F00025F0FE0EDB5006E081EC25F0BADFE55259
:10240000E552E552010E10EF23F022EC2CF028E00B
:10241000ADEC29F003E07EEC23F006E1BEEC28F001
:102420001FE07EEC23F01CE0ECEC2AF016E0050E39
:102430006BEC2BF012E0E8EC2AF008E07DEC25F0E4
:1024400005E0FFEC24F032EC28F002D00601F16B3D
:10245000FFEC24F01C0E93EC25F00601F3A502D04E
:10246000000E31D093EC23F0B30EE66EFD0EE66E57
:10247000000E04EC29F00601F1510AE1AD0EE66E02
:10248000FD0EE66E000E4EEC2CF046EC22F016D05F
:10249000F151CDEC2AF0D7EC27F006E1E40E006E06
:1024A000FD0E016E000E05D0E00E006EFD0E016EF9
:1024B000000E026E72EC23F0E6EC26F068EC2CF0D5
:1024C00082EC29F0010EDBEC27F002E2E16AE55232
:1024D000E16E005010EF23F00BEC23F0080EE12624
:1024E000020EDB6A39EC28F0060158EC26F026ECE7
:1024F0002CF00601F151000807E2F151E66ED950C7
:10250000060F76EC25F02AD00901055106110AE0E4
:102510000751081107E0C6EC22F0EFEC26F0D3ECEF
:102520002AF004D0060EDB6A070EDB6AD7EC27F030
:1025300015E171EC26F0033402E2C4EC27F003E36A
:10254000006A016A09D09AEC23F0A8EC29F092EC19
:1025500026F0FDE197EC26F029EC27F0D950060F84
:102560002AEC2AF00FE0060EDBCF08F0070EDBCFD7
:1025700009F00A6A0B6A09AE02D00A680B6843ECDC
:1025800023F002D0006A016A68EC24F08BEC2CF096
:1025900003E078EC26F003D0CB0E006E016A0BEC62
:1025A0002AF00601F0515EEC2AF038EC29F0060121
:1025B000EF51DDEC2DF0040EDBCFE6FF050EDBCF97
:1025C000E6FF4BEC2CF033EC24F04BEC2CF0CDEC94
:1025D00023F09DEC28F0D6EC22F0B2EC27F002E1DB
:1025E000010E02D0FE0EDB50006E080EE15C02E22E
:1025F000E16AE552E16E005010EF23F00BEC23F09E
:10260000040ECAEC26F0CC0EEE1845E1ED5043E185
:10261000DE6ADD6A07EC2CF0ECEC2AF016E08CECBC
:1026200025F0EF5012E09DEC28F0E66EF1EC29F079
:1026300040EC28F068EC2CF09DEC28F0E66E94EC71
:102640002BF040EC28F026EC2CF093EC2CF0EE5024
:10265000ED1005E0ECEC2DF0BAEC25F002D0006AAC
:10266000016A00C0F0F6D950020F2AEC2AF005E00A
:1026700033EC24F0BAEC25F002D0006A016A00C005
:10268000EFF6ECEC2DF01B0E93EC25F033EC24F080
:102690001A0E93EC25F0FE0EDB5006E081EC25F0DF
:1026A0001BDFE552E552E552010E006E040EE15CBF
:1026B00002E2E16AE552E16E005010EF23F00BEC0C
:1026C00023F0100EE126FE0EDB5068E0ADEC29F0A1
:1026D00003E07EEC23F006E1BEEC28F05FE07EEC48
:1026E00023F05CE0ECEC2AF056E0020E6BEC2BF0F1
:1026F00052E0060EDB6A44EC28F00601EF6BF06B4B
:10270000E8EC2AF03EE07DEC25F03BE0FFEC24F025
:102710007EEC92F0E552E55226EC2CF0FFEC24F032
:1027200040EC9FF026EC2AF00006000E015AF80E4D
:10273000DB500024E96EF90EDB500120EA6E040E36
:10274000EFCFDBFFDB50250808E14BEC28F0D3ECA2
:102750002AF0020EDBCFEFF607D04BEC28F052EC5C
:1027600028F0020EDBCFF0F6FFEC24F092EC5BF0E9
:10277000E552E552F80EF3CFDBFFF90EF4CFDBFFA5
:10278000BFD7BDEC2BF01A0E93EC25F0DAEC2AF053
:102790001B0E93EC25F00601F3A502D0000EFED02F
:1027A00093EC23F09E0EE66EFD0EE66E000E04EC3A
:1027B00029F00601EF5108E1F05106E19A0EE66EAC
:1027C000FD0EE66E000EDCD00AEC2BF0EF51000897
:1027D00013E258EC26F00A0EF3CFDBFF0B0EF4CF1A
:1027E000DBFF0601EF51CDEC2AF0370EE66EFF0E4F
:1027F000E66E000EA3EC28F00601F051000801E39C
:1028000084D0F151000807E2F151E66ED9500E0F65
:1028100076EC25F03AD00901055106110EE007517A
:1028200008110BE0C6EC22F0EFEC26F00E0E28C0EB
:10283000DBFF0F0E29C0DBFF04D00E0EDB6A0F0E8C
:10284000DB6AD7EC27F021E10E0EDBCF02F00F0E92
:10285000DBCF03F0033402E2C4EC27F003E3006AA9
:10286000016A0DD00E0EDBCF00F00F0EDBCF01F0B2
:10287000A8EC29F092EC26F0FDE197EC26F00E0E84
:1028800000C0DBFF0F0E01C0DBFFD9500E0F2AEC9A
:102890002AF00FE00E0EDBCF08F00F0EDBCF09F0B1
:1028A0000A6A0B6A09AE02D00A680B6843EC23F08F
:1028B00002D0006A016A0C0E00C0DBFF0D0E01C0E1
:1028C000DBFF0601EF51000807E2950EE66EFD0EF4
:1028D000E66E000EA3EC28F00601F051CDEC2AF0D4
:1028E000D7EC27F006E1E40E006EFD0E016E000E3F
:1028F00005D0E00E006EFD0E016E000E026E72EC51
:1029000023F0E6EC26F068EC2CF024EC28F00134FF
:1029100020E28DEC26F01DE2D9500A0F2AEC2AF0B5
:1029200013E008EC28F00A0EDBCF04F00B0EDBCF2F
:1029300005F003500518E8AE02D0053404D0045069
:10294000025C0550035805E20C0EDBCFE6FF0D0ECE
:102950000BD00FEC28F0013411E28DEC26F00EE2E2
:102960000A0EDBCFE6FF0B0EDBCFE6FF8C0EE66E2A
:10297000FD0EE66E000EE66EEEEC21F0B8EC27F0F0
:10298000A3EC28F0CDEC23F07C0EE66EFD0EE66E97
:10299000000E7DEC2DF082EC29F0010E006E100E81
:1029A000E15C02E2E16AE552E16E005010EF23F0D3
:1029B0000BEC23F0E652090117AD02D0010E14D042
:1029C0000B0EDF6E3F0E0001FE5D08E0DF500008D9
:1029D00005E2010EC9EC27F0DF06F4D73F0EFE5DDD
:1029E00002E0000E01D0010EE55210EF23F066EC7C
:1029F0002AF0DEDFDE6ADD6A6BEC2AF002E62BEC01
:102A00002CF02EE24AEC22F0030EE2EC22F0FDE183
:102A100086EC2CF0E2EC22F0FDE114EC23F0040E45
:102A20009AEC24F04AEC22F0030EE2EC22F0FDE1F5
:102A300086EC2CF0E2EC22F0FDE1D9EC2DF09AECE2
:102A400024F04AEC22F0030EE2EC22F0FDE1E8EC87
:102A50002CF083EC26F0DF2A010ECEE3DB2ACCD764
:102A6000DE6ADD6A6BEC2AF002E644EC2BF013E23E
:102A700013EC2DF0F5EC26F013EC2DF09DEC27F087
:102A80000EEC29F067EC2DF057EC27F0DF2A010E51
:102A9000E9E3DB2AE7D7DE6ADD6A6BEC2AF002E6BF
:102AA0006EEC28F029E2FAEC2DF0020E9AEC24F0FC
:102AB000FAEC2DF0040E9AEC24F00AEC29F00F0E3B
:102AC000C0EC2DF0110E32EC2DF00C0E32EC2DF08E
:102AD0000D0E32EC2DF0060EC0EC2DF0080EC0EC01
:102AE0002DF00E0E32EC2DF00A0E83EC26F0DF2ACC
:102AF000010ED3E3DB2AD1D70001FE6B020EE15CAD
:102B000002E2E16AE552E16E10EF23F00BEC23F0F4
:102B1000180EE1263F0E0001FE5D01E0E6D3D1EC88
:102B200025F095EC24F0070E12EC26F001E397D087
:102B30004AEC22F0020EE2EC22F0FDE1D2EC28F0A9
:102B4000EF5001E18CD04AEC22F0020EE2EC22F0D0
:102B5000FDE17FEC26F0F00E005C01E380D04AEC52
:102B600022F0020EE2EC22F0FDE1D2EC28F0EE526F
:102B7000EF5014E04AEC22F0020EE2EC22F0FDE10C
:102B80007FEC26F04AEC22F0020EE2EC22F0FDE1AE
:102B9000D2EC28F0EE52EF50005C0DE24AEC22F04D
:102BA000020EE2EC22F0FDE151EC2DF0E2EC22F01D
:102BB000FDE19DEC27F04AEC22F0020EE2EC22F05F
:102BC000FDE1D2EC28F0020EFEEC23F016E04AEC18
:102BD00022F0020EE2EC22F0FDE17FEC26F04AEC5E
:102BE00022F0020EE2EC22F0FDE1D2EC28F0020E1F
:102BF000FEEC23F0D88000540DE24AEC22F0020EE5
:102C0000E2EC22F0FDE151EC2DF0E2EC22F0FDE1EE
:102C1000F5EC26F04AEC22F0020EE2EC22F0FDE1A7
:102C20007FEC26F0016A79EC2AF0020EE2EC22F049
:102C3000FDE159EC28F0096A0A6A0B6A4AEC22F0B5
:102C4000020EE2EC22F0FDE1D2EC28F0EFCF04F02E
:102C5000056A02EC24F001E264D7DB2A62D793EC28
:102C60002CF0070EEE1801E03FD1ED5001E03CD111
:102C70003AEC24F0E00E2E6E400E39EC26F044ECD7
:102C80002AF0BCEC8DF01EEC8BF012EC29F02AEC53
:102C90002BF05EEC8BF0D7EC28F02C6A2D6A200E1E
:102CA0002E6E420E2F6E5DEC8BF0BCEC8DF029C0C9
:102CB000C2F90901780EE26F45EC24F0E00E2E6EA9
:102CC000400E61EC22F005E1010EF36E9CEC26F063
:102CD000DB6A77EC23F000017151026E036A28EC85
:102CE00026F016E2020EDBCF71F0DBCF00F0030E10
:102CF000DBCF01F012EC26F003E3800E6D6F08D0FD
:102D000077EC23F0020E12EC26F002E3800E6C6FDB
:102D1000DE6ADD6A95EC24F0070E12EC26F001E382
:102D2000E3D04AEC22F0020EE2EC22F0FDE159EC95
:102D300028F008C029F01CEC8BF06BEC27F0DBCFFF
:102D400009F0150EDBCF0AF0160EDBCF0BF0170ED5
:102D5000DBCF0CF0E1EC2AF00CC02FF083EC2DF06F
:102D6000020EE2EC22F0FDE1D2EC28F0EFCF15F0FC
:102D700015C029F01CEC8BF027C011F028C012F010
:102D800029C013F02AC014F0140EDBCF16F0150E74
:102D9000DBCF17F0160EDBCF18F0170EDBCF19F0D4
:102DA00016C02CF017C02DF018C02EF019C02FF04F
:102DB00049EC8EF0010A05E00D6A0E6A0F6A3F0EBB
:102DC00004D00D6A0E6A0F6ABF0E106E0DC02CF093
:102DD0000EC02DF00FC02EF0DFEC24F003E0C4ECA9
:102DE0002BF002D09AEC23F068EC24F0800E000166
:102DF0006D150CE030EC2BF009E3010EDF5211E011
:102E0000DFCFF3FF00EC28F0FDE10BD030EC2BF02E
:102E10000BE3010EDF5205E0DFCFF3FF00EC28F0FB
:102E2000FDE100016D131FD0800E6C150FE0F5EC75
:102E300022F0020E12EC26F009E3010EDF5211E03F
:102E4000DFCFF3FF00EC28F0FDE10BD0CBEC2BF053
:102E50000AE2010EDF5205E0DFCFF3FF00EC28F0BD
:102E6000FDE100016C13F5EC22F04AEC22F0020EB9
:102E7000E2EC22F0FDE167EC2DF0BEEC29F0EFCFA3
:102E800004F004340DE34AEC22F0020EE2EC22F0EE
:102E9000FDE167EC2DF0FEEC23F0FF0DF3500AD0BE
:102EA0004AEC22F0020EE2EC22F0FDE167EC2DF09C
:102EB000FEEC23F0026E036A02BE036828EC26F0E3
:102EC0000DE24AEC22F0020EE2EC22F0FDE167ECAA
:102ED0002DF0BEEC29F0060EDBCFEFFFDF2A010E4E
:102EE00001E218D7DB2A16D700016251631105E011
:102EF0006251605D6351615904E260C062F061C07B
:102F000063F06451651105E06051645D615165597C
:102F100004E260C064F061C065F0D1EC25F095EC8E
:102F200024F00E0E12EC26F001E399D04AEC22F0C8
:102F3000030EE2EC22F0FDE114EC23F0EE50ED1074
:102F400001E18DD04AEC22F0030EE2EC22F0FDE12B
:102F5000F7EC28F0000E005C0F0E015801E37FD063
:102F60004AEC22F0030EE2EC22F0FDE1D9EC2DF068
:102F7000C4EC25F012E04AEC22F0030EE2EC22F061
:102F8000FDE186EC2CF0E2EC22F0FDE1D9EC2DF035
:102F900001EC26F0CEEC27F00FE24AEC22F0030E13
:102FA000E2EC22F0FDE186EC2CF0E2EC22F0FDE117
:102FB000D9EC2DF09AEC24F04AEC22F0030EE2EC6E
:102FC00022F0FDE114EC23F0040EC4EC25F013E034
:102FD0004AEC22F0030EE2EC22F0FDE186EC2CF04C
:102FE000E2EC22F0FDE114EC23F0040E01EC26F0FB
:102FF00028EC26F010E24AEC22F0030EE2EC22F07C
:10300000FDE186EC2CF0E2EC22F0FDE114EC23F083
:10301000040E9AEC24F04AEC22F0030EE2EC22F0CB
:10302000FDE1F7EC28F079EC2AF0030EE2EC22F057
:10303000FDE1D1EC2BF00A6A0B6A4AEC22F0030E98
:10304000E2EC22F0FDE114EC23F0EECF04F0EFCF40
:1030500005F002EC24F001E262D7DB2A60D793ECA2
:103060002CF00E0EEE1801E031D1ED5001E02ED122
:103070003AEC24F0600E2E6E410E39EC26F045EC51
:1030800024F0600E2E6E410E61EC22F005E1010E7F
:10309000F36E9CEC26F0DB6A77EC23F00001005025
:1030A0006F5D0150705918E2020EDBCF6FF0030E16
:1030B000DBCF70F077EC23F0050E12EC26F004E382
:1030C000686B800E696F08D077EC23F012EC26F065
:1030D00003E3666B800E676FDE6ADD6A95EC24F0B1
:1030E0000E0E12EC26F001E3F1D04AEC22F0030EB2
:1030F000E2EC22F0FDE1D1EC2BF008C028F009C091
:1031000029F02DEC8BF06BEC27F0DBCF0AF0150EDD
:10311000DBCF0BF0160EDBCF0CF0170EDBCF0DF074
:103120000AC02CF00BC02DF00CC02EF00DC02FF0FB
:1031300083EC2DF0030EE2EC22F0FDE114EC23F021
:10314000EECF16F0EFCF17F016C028F017C029F019
:103150002DEC8BF027C012F028C013F029C014F01A
:103160002AC015F0140EDBCF18F0150EDBCF19F0C6
:10317000160EDBCF1AF0170EDBCF1BF018C02CF0A9
:1031800019C02DF01AC02EF01BC02FF049EC8EF0A4
:10319000010A05E00E6A0F6A106A3F0E04D00E6A3B
:1031A0000F6A106ABF0E116E0EC02CF00FC02DF00A
:1031B00010C02EF0DFEC24F003E0C4EC2BF002D0C2
:1031C0009AEC23F068EC24F000016951800B0CE0CC
:1031D000F5EC22F012EC26F007E307EC26F010E005
:1031E00085EC25F0FDE10CD0F5EC22F0060E12EC9A
:1031F00026F00CE307EC26F003E085EC25F0FDE17A
:10320000005000016813015069131BD06751800BF7
:103210000AE030EC2BF007E307EC26F00DE085EC3C
:1032200025F0FDE109D0CBEC2BF00BE207EC26F00A
:1032300003E085EC25F0FDE100500001661301502C
:103240006713F5EC22F04AEC22F0030EE2EC22F0D8
:10325000FDE1E8EC2CF0BEEC29F0EECF04F0EFCF6E
:1032600005F00001800E05140EE04AEC22F0030E7A
:10327000E2EC22F0FDE1E8EC2CF001EC26F0026C2F
:10328000031E03220AD04AEC22F0030EE2EC22F0E5
:10329000FDE1E8EC2CF001EC26F028EC26F010E241
:1032A0004AEC22F0030EE2EC22F0FDE1E8EC2CF017
:1032B000BEEC29F0060EDBCFEEFF070EDBCFEDFFF5
:1032C000DF2A010E01E20AD7DB2A08D700016A5182
:1032D000681906E16B51691903E16E516D5D03E0F8
:1032E000110E090118130001FE6B180EE15C02E2D9
:1032F000E16AE552E16E10EF23F00BEC23F0080ECB
:10330000E126D950FB0FBFEC22F002E0A00E01D065
:10331000C70E006E016A68EC24F01FEC2BF004EC81
:1033200023F0740EE66EFD0EE66E000ECCEC28F077
:10333000A8EC28F00F0E2EEC2AF0A8EC28F0080ECE
:1033400046EC2BF003E05CEC25F008D0A8EC28F06C
:10335000060E46EC2BF004E062EC25F0CCEC28F0F5
:1033600033EC24F082EC2AF089EC2DF0A8EC28F064
:10337000080EC4EC25F00EE1A8EC28F0060EC4EC13
:1033800025F008E1640EE66EFD0EE66E000ECCEC54
:1033900028F05CD0DE6ADD6A6BEC2AF002E62BECEA
:1033A0002CF054E22DEC2CF00C0EBEEC27F0E8AE25
:1033B00002D0033402D0CEEC27F001E399D0A8EC80
:1033C00028F0080E70EC2AF0DF501F0B03E0F1EC40
:1033D00024F0FDE186EC23F003E05CEC25F010D056
:1033E000A8EC28F0060E70EC2AF0DF501F0B03E06B
:1033F000F1EC24F0FDE186EC23F023E062EC25F013
:10340000CCEC28F04AEC22F0030EE2EC22F0FDE1D5
:10341000E8EC2CF02EEC2AF0D8EC2BF05E0EE66EE9
:10342000FD0EE66E000E8FEC2DF005E133EC24F07E
:103430000CEC27F004D033EC24F087EC26F089EC78
:103440002DF0DF2A010EA8E3DB2AA6D72DEC2CF005
:10345000140EBEEC27F0E8AE02D0033402D0CEEC5E
:1034600027F046E2510EE66EFD0EE66E000ECCEC45
:1034700028F0A8EC28F0110EFEEC23F0E66ED950EF
:10348000020F76EC25F02DEC2DF0800B03E05CECC8
:1034900025F006D0C4EC2DF0800B04E062EC25F0A2
:1034A000CCEC28F033EC24F082EC2AF095EC2DF0F3
:1034B0002DEC2DF009E1C4EC2DF006E1640EE66E72
:1034C000FD0EE66E000E19D0DE6ADD6A6BEC2AF0A6
:1034D00002E644EC2BF05AE22DEC2CF0080EBEEC88
:1034E00027F0E8AE02D0033402D0CEEC27F008E398
:1034F000600EE66EFD0EE66E000ECCEC28F046D0B7
:10350000010EDF5205E0DFCFF3FF00EC28F0FDE114
:10351000006E2DEC2DF0001403E05CEC25F00FD0D4
:10352000010EDF5205E0DFCFF3FF00EC28F0FDE1F4
:10353000006EC4EC2DF0001424E062EC25F0CCEC1D
:1035400028F00EEC29F067EC2DF0C8EC25F0016AAC
:1035500000BE016863EC26F0D8EC2BF04C0EE66E52
:10356000FD0EE66E000E8FEC2DF005E133EC24F03D
:103570000CEC27F004D033EC24F087EC26F095EC2B
:103580002DF0DF2A010EA2E3DB2AA0D7080EE15CB2
:1035900002E2E16AE552E16E10EF23F00BEC23F05A
:1035A0000A0EE126D8EC14F0000905E1FE0EDB500E
:1035B000000801E2AED1D95024EC2BF0CD0EEE186C
:1035C00030E1ED502EE1DF6A010EDF5C01E3A1D1B5
:1035D0004FEC22F0080EC4EC25F003E135EC2BF0A3
:1035E00013E0D5EC29F094EC2BF0DFCFE6FFF3EC01
:1035F00027F0016ADF34FE0B0136006E6E0E0026E6
:10360000090E3AEC2BF00BD0EA6ADF34FE0BEA36F7
:10361000E96E6E0EE926090EEA22EE6AED6ADF2AED
:10362000D3D7020EDB6839EC28F0010EDB6A070EF7
:103630005DEC28F02DE2F0EC2AF0EF50006E016A0C
:10364000D950040FF9EC27F0F0EC2AF0EE52EFCF4E
:1036500000F0020EDB50005C06E2F0EC2AF0EE52C5
:10366000020EEFCFDBFFF0EC2AF0020EC8EC25F0E3
:10367000030EDB50D880005408E2F0EC2AF0020E72
:10368000BEEC29F0030EEFCFDBFF010EDB2ACFD714
:10369000040EDBCF28F0050E18EC24F0040E28C031
:1036A000DBFF050E29C0DBFFDF6A010EDF5C01E3F3
:1036B00030D14FEC22F0080EC4EC25F002E0030EEE
:1036C00009D04FEC22F0060EC4EC25F002E0020E09
:1036D00001D0010EF36E060EF3CFDBFF35EC2BF0BD
:1036E00002E0030E08D04FEC22F03FEC2CF002E099
:1036F000020E01D0010E86EC29F0DF28E66EE66AA4
:10370000340EE66EFD0EE66E000E3FEC22F00E0E5D
:10371000FDEC2AF0010EE66EE66A83EC2CF0E1EC9B
:103720002DF080EC28F083EC2CF085EC28F083EC75
:103730002CF08AEC28F083EC2CF04FEC22F0B5EC66
:103740002CF014EC2AF0B5EC2CF020EC29F04FEC26
:1037500022F0020EAFEC22F014EC2AF0020EAFECD5
:1037600022F020EC29F04FEC22F0040EAFEC22F016
:1037700014EC2AF0040EAFEC22F020EC29F0F5EC6A
:1037800022F0DEEC2BF0E5EC21F0020E88EC2AF0C2
:10379000E5EC21F0030E88EC2AF0C8EC2DF00F0EBA
:1037A0001BEC29F0C8EC2DF0110EFEEC23F0E66EB8
:1037B000E66A83EC2CF0016ADF34FE0B0136006E02
:1037C000700E0026090E3AEC2BF0010EDB6A0E0E8D
:1037D0005DEC28F001E39BD04FEC22F0080E70EC7A
:1037E0002AF0DB501F0B03E0F1EC24F0FDE186EC46
:1037F00023F002E0030E11D04FEC22F0060E70EC25
:103800002AF0DB501F0B03E0F1EC24F0FDE186EC25
:1038100023F002E0020E01D0010EF36E060EF3CF8C
:10382000DBFF04EC28F0016E010E015204E0E846D3
:10383000FE0B0106FCE1006E35EC2BF0001402E0FB
:10384000030E14D004EC28F0016E010E015204E0C6
:10385000E846FE0B0106FCE1006E4FEC22F03FEC67
:103860002CF0001402E0020E01D0010E86EC29F0CB
:10387000010EDB28E66EE66A230EE66EFD0EE66EAE
:10388000000E3FEC22F0DF28FDEC2AF0E1EC2DF0F9
:10389000010EDB50080DBAEC2CF0F7EC28F0050E09
:1038A000CCEC2DF09AEC29F0020E1BEC29F09AECEE
:1038B00029F0040E1BEC29F09AEC29F0060E1BEC03
:1038C00029F09BEC2DF0EF50DEEC29F0EE52EF509A
:1038D000DEEC29F0020EFEEC23F0DEEC29F0030E04
:1038E000C8EC25F0016A00BE016872EC23F0E5EC3B
:1038F00021F0010E016ADB34FE0B0136006E720E00
:103900000026090E3AEC2BF0010EDB2A60D7DF2AE5
:10391000CCD6FE0EDB50006E0A0EE15C02E2E16ADC
:10392000E552E16E005010EF23F022EC2CF019E08C
:1039300081EC25F033DE8DEC2AF0ADEC29F003E0CC
:1039400078EC26F003D0CE0E006E016A72EC23F004
:103950000CEC2DF07BEC29F068EC2CF0F4EC2CF066
:1039600009D089EC27F01ADE8DEC2AF0020802E07B
:103970002FEC2EF0010EDBEC27F002E2E16AE552BB
:10398000E16E005010EF23F00BEC23F00D0EE1265A
:10399000FE0EDB500FE00601F3B50CD0ADEC29F0C4
:1039A00003E07EEC23F008E1BEEC28F003E07EECBF
:1039B00023F002E1000E03D2D8EC14F093EC23F0D4
:1039C000E8EC2AF004E07DEC25F0200901D0000E9F
:1039D00069EC28F0DB5009E0010EE76EE4EC2BF017
:1039E000E750FEEC23F0200901D0000EE76E050E33
:1039F000E7CFDBFF040EDB50760A01E1F4D0020AC8
:103A00000FE0060A01E0C7D1F7EC14F005010C0E37
:103A1000FD6FFD0EFE6F000EFF6FFEEC3EF0CED18F
:103A2000060EDB6844EC28F007EC2CF031EC2CF0AF
:103A300002E644EC2BF030E2B9EC22F0EF50006EDD
:103A4000016AD950080FF9EC27F0B9EC22F0EE52D8
:103A5000EFCF00F0060EDB50005C06E2B9EC22F07E
:103A6000EE52060EEFCFDBFFB9EC22F0020EC8ECEF
:103A700025F0070EDB50D880005408E2B9EC22F0A4
:103A8000020EBEEC29F0070EEFCFDBFF020EDB2AA1
:103A9000030ECCE3DB2ACAD7080EDBCF28F0090ED1
:103AA00018EC24F052EC28F01FEC26F0050EDB5049
:103AB00064081CE100016DAF03D05CEC25F004D07C
:103AC0006CAF04D062EC25F036EC2DF000017151A2
:103AD000E66EE66A82EC2AF0E66EA3EC2CF078EC57
:103AE0002CF031EC29F012EC27F024D0EBEC2BF089
:103AF000DEEC2BF0090EE66EFD0EE66E000E98EC85
:103B00002BF0060E88EC2AF0050EE66EFD0EE66E32
:103B1000000E98EC2BF0070E88EC2AF0010EE66EF2
:103B2000FD0EE66E000E98EC2BF0FD0EE66EFC0E20
:103B3000E66E000E3AEC2DF0DB6A030EDB6A31EC28
:103B40002CF002E644EC2BF001E322D1010EF36EDF
:103B5000020EDB5004E0D890F336E806FCE1F350A7
:103B600000016D1503E05CEC25F00FD0010EF36E43
:103B7000020EDB5004E0D890F336E806FCE1F35087
:103B800000016C1504E062EC25F036EC2DF0C2EC7F
:103B900029F015E13FEC2BF000340AE23FEC2BF06A
:103BA000016A00BE016872EC23F00CEC27F010D023
:103BB0003FEC2BF0016A00AE07D0016805D0B9ECEC
:103BC00022F0EF506FEC24F072EC23F087EC26F03B
:103BD00098EC2BF012EC27F03AEC2DF0DB2A030ED8
:103BE000AEE3DB2AACD71FEC26F0DE6ADD6A6BECB5
:103BF0002AF002E66EEC28F001E3CAD0050EDB5095
:103C000064081FE10AEC29F0080E46EC2BF003E0F3
:103C10005CEC25F008D00AEC29F0060E46EC2BF0FF
:103C200004E062EC25F036EC2DF00AEC29F00F0EE2
:103C30001BEC29F082EC2AF098EC2BF006EC27F034
:103C400011D0020EE66EE66A0AEC29F0B5EC2CF013
:103C50000A0E13EC2BF0090EE66EFD0EE66E000E5A
:103C600025EC25F03AEC2DF0DB6A030EDB6A31EC33
:103C70002CF002E62BEC2CF001E384D00B0EDBCF12
:103C800000F00C0EDBCF01F0A00E026E060E036EEC
:103C90000D0E025E000E035A28EC26F009E282ECBB
:103CA00029F041EC5AF01E0E15EC2CF01FEC26F01A
:103CB0000AEC29F0080E70EC2AF0020EDB501F0B04
:103CC00003E0F1EC24F0FDE186EC23F003E05CEC92
:103CD00025F011D00AEC29F0060E70EC2AF0020E45
:103CE000DB501F0B03E0F1EC24F0FDE186EC23F048
:103CF00004E062EC25F036EC2DF0C2EC29F029E16D
:103D0000F8EC29F0E2EC22F0FDE1E8EC2CF0AFEC6D
:103D100022F00001800E01140CE1F8EC29F0E2EC35
:103D200022F0FDE1E8EC2CF01BEC29F00CEC27F084
:103D30000BD0F8EC29F0E2EC22F0FDE1E8EC2CF0FD
:103D40001BEC29F087EC26F098EC2BF006EC27F022
:103D500011D0030EE66EE66AF8EC29F0E2EC22F0F0
:103D6000FDE1F7EC28F0050E13EC2BF087EC26F0C4
:103D700025EC25F03AEC2DF0DB2A030E01E277D793
:103D8000DB2A75D7DF2A010E01E231D7DB2A2FD7D4
:103D900082EC29F013D00601006B010EE66EE66A94
:103DA000000EE66EF3EC27F019EC2CF082EC29F013
:103DB00068C06AF069C06BF06DC06EF0010E006EF5
:103DC0000D0EE15C02E2E16AE552E16E005010EF97
:103DD00023F00BEC23F0FC0EDBCF28F0FD0EDBCF45
:103DE00029F0CF0E281801E1295040E0D00E281804
:103DF00001E129503BE0CD0E281801E1295033E0C4
:103E0000CE0E281801E129502EE0CB0E281801E132
:103E1000295025E0CC0E281801E1295020E0C90ED8
:103E2000281801E1295017E0CA0E281801E129508D
:103E300012E0C80E281801E1295009E0060E2818E2
:103E40001BE1295019E1C9DBAFEC11F012D0C5DB41
:103E50003CEC0FF00ED0C1DBDCEC11F00AD0BDDB86
:103E6000FEEC12F006D0B9DB60DD03D0B6DB7FECF0
:103E70000EF074EC2AF001D0000ED2D3CCDB030E8E
:103E8000E126DE6ADD6A76EC24F004BE0568040EE5
:103E900018EC27F0FDE188EC24F001E1E4D0200EDD
:103EA000066E500E076E010E086EDECF09F0DDCFF4
:103EB0000AF00B6A0ABE0B68040ED89009360A365F
:103EC0000B36E806FAE106500924036E07500A2073
:103ED000046E08500B20056E03C0E6FF04C0E6FF29
:103EE000E66E4EEC9FF08DEC2AF0A1EC2DF0000672
:103EF000000E015A025A72EC23F0200E0F6E500E83
:103F0000106E010E116EDECF12F0DDCF13F0146AC9
:103F100013BE1468040ED890123613361436E80611
:103F2000FAE10F5012240C6E105013200D6E115038
:103F300014200E6E0C2A000E0D220E220CC0E6FF7D
:103F40000DC0E6FF0EC0E6FFF90EDBCFE6FFFA0E6E
:103F5000DBCFE6FF2EEC9EF0156E070EE15E1550EE
:103F6000000901E07AD0FE0EDB5030E0F70EDBCF27
:103F7000E6FFF80EDBCFE6FF4BEC5BF0E552E552D7
:103F8000F70EF3CFDBFFF80EDFEC27F0F70FE66E4E
:103F9000FF0EDA20E66EFB0EDBCFE6FFFC0EDBCF7A
:103FA000E6FF76EC24F004BE0568040E18EC27F05A
:103FB000FDE188EC24F0E66E52EC62F0066E050E30
:103FC000E15E0650000902E1000E4ED0DECFE9FFAF
:103FD000DDCFEAFF030EEA02F3CFEAFFE902F3CFF7
:103FE000E9FFF450EA26EA0EE9260A0EEA22EECFAD
:103FF00000F0EECF01F0EFCF02F0F70EDBCFE6FFDF
:10400000F80EDBCFE6FFF90EDBCFE6FFFA0EDBCFD3
:10401000E6FFFB0EDBCFE6FFFC0EDBCFE6FFFD0E7F
:10402000DBCFE6FF06D002C0FBFF01C0FAFF005065
:10403000F96EF9DF036E070EE15E0350E76E020EC4
:10404000E7CFDBFFFD0EDB5005E0020EDB5002E0A8
:1040500041EC5AF0020EDB5007D0DF2A010E01E2DC
:1040600012D7DB2A10D7000E006E030EE15C02E2CD
:10407000E16AE552E16E0050D3D2CDDAFFEC24F0D4
:10408000ACDAE66A7BEF2BF0C6DAF90EDBCFE6FF9F
:10409000A4DA010EE66EE66E7BEF2BF022EC2CF03C
:1040A00003E10601F3A502D0000E3DD00501E70EA5
:1040B000FD6FFC0EFE6F000EFF6FFEEC3EF0DE6A41
:1040C000DD6A76EC24F004BE0568040E18EC27F0D7
:1040D000FDE188EC24F026E00501E50EFD6FFC0E05
:1040E000FE6F000EFF6FFEEC3EF076EC24F004BE97
:1040F0000568040E18EC27F0FDE1005003240501CB
:10410000FD6F01500420FE6F02500520FF6FFD2B54
:10411000000EFE23FF23FEEC3EF0DF2A010ED1E36A
:10412000DB2ACFD7010EDBEC27F002E2E16AE55291
:10413000E16E005075D26FDAE652520E0601C85D8C
:1041400006E1540EC95D03E1CA5101E178D0520E77
:10415000C86F540EC96FCA6BCB6BCC6B0901400E94
:10416000176F880E036F130E046F100E056F270E66
:10417000066F096B0A6B0901320EA06F0901006B13
:104180000B6F0C6B640E076F086B016B026B0D6B92
:104190000E6B156B166B0F6B106B116B126B136B39
:1041A000146B120EA1EC26F0600EE66E000E8BDB97
:1041B0000001E80E626F030E636F1C0EA1EC26F087
:1041C000720EE66E000E7FDBDF6A070EDF5C0BE22D
:1041D000DF5015DA280EEF6EDF5011DAEE52F00ED6
:1041E000EF6EDF2AF2D7700EA1EC26F08E0EE66E8F
:1041F000000E69DBDF6A0E0EDF5C0EE2DF50080D99
:10420000BAEC2CF0D9EC2DF0BEEC29F0D00EEE6E0D
:10421000070EED6EDF2AEFD791EC2AF03E6B3F6B75
:104220009BEC2AF0B1EC25F0186B0901A56BA66B8D
:10423000A76BA86B0901A96BAA6BAB6BAC6B0001F8
:10424000FE6B900E6F6E6EAEFED7606A0F0118693E
:10425000E00E196F2A0E006FA00E016F046B056B44
:10426000506BFE0E1C6F1D6BB20E086F096BD20EE9
:104270000C6F0D6BAA0E106F116BBA0E146F156BCD
:10428000706ABF0E716E020E726E200E736E0601A2
:10429000F451000802E26F6A02D0600E6F6E0701EF
:1042A0002A0ECC6F4E0ECD6F010ECE6F0701300E71
:1042B000CF6F4E0ED06F010ED16F0701340ED56F48
:1042C000040ED66F000ED76F0701C40ED86F060E0E
:1042D000D96F000EDA6F0701080EF06F0F0EF16F45
:1042E000000EF26F07010C0EDB6F0F0EDC6F000E7D
:1042F000DD6F0701F00EDE6F130EDF6F000EE06F53
:104300000701140EE16F140EE26F000EE36F080157
:104310007A0EF36F400EF46F000EF56F0801880EF1
:10432000F66F400EF76F000EF86F0801D20EF06FB7
:104330003D0EF16F000EF26F0501EE81EE83EE850A
:10434000010EE5526DD1F20E00262B0EF9EC2BF08A
:10435000E40E2B6E570E2C6EB0EC28F0B0EF2CF064
:1043600060EC2CF0D4EC74F0086E090E1BEC2BF012
:1043700051EC2AF09CEC2CF004C026F06DEC29F0F6
:10438000040EDBCF2BF0050EDBCF2CF0060EDBCFBF
:104390002DF0070EDBCF2EF0E8EC2DF01DEC2CF00D
:1043A00059EC2DF0390EE66EFF0EE66E000E60EC55
:1043B0002CF0C2EC74F0086E070E1BEC2BF0370EDD
:1043C000E66EFF0EE66E000E12009DEC28F0E66E23
:1043D000DAEC2AF07BEC29F083EF2BF0ECEC2DF0FB
:1043E00071EF2DF0120EEA02F3CFEAFFE902F3CFEC
:1043F000E9FFF450EA26600EE926000EEA221200D8
:104400009DEC28F0FFEC29F0DBEF2CF0040EDBCF65
:1044100004F0050EDBCF05F0060EDBCF06F0070E2D
:10442000DBCF07F0D950080FBFEC2CF0EE50045C46
:10443000006EEE500558016EEE500658026EEE50BA
:104440000758036E110E00C0DBFF120E01C0DBFF28
:10445000130E02C0DBFF140E03C0DBFFD950040FA4
:10446000E96E94EF29F060EC2CF0E5EC74F0046E4A
:10447000090E06EF2BF0BAEC28F0DCEF28F0E66E20
:10448000DAEC2AF078EC2CF083EF2BF08CEC74F063
:1044900074EF2AF0DECFE9FFDDCFEAFF1200DF5034
:1044A000120DBAEC2CF0600EE926000EEA22120082
:1044B0000102F3CF01F00002F3CF00F0F450012627
:1044C00012002F6ED0EC2DF044EC2AF0140EDBCF4E
:1044D0002CF0150EDBCF2DF0160EDBCF2EF0170EC5
:1044E000DBCF2FF047EC8CF060EC29F05DEC8BF02B
:1044F000100E27C0DBFF110E28C0DBFF120E29C0F3
:10450000DBFF130E2AC0DBFFD950100FBFEC2CF0DD
:10451000EECFE6FFEECFE6FFEECFE6FFEFCFE6FF12
:1045200043ECA0F08DEC2AF0E55242EC2CF02AECA2
:104530002BF026C027F0B6EC2AF0020E28C0DBFFD5
:10454000030E29C0DBFFD950020F2AEF2AF04EECF0
:104550002CF02DEC75F0006E070E2DEF29F0BEEC5F
:1045600029F0B5EF2CF0A3EC2CF07BEC29F031EF27
:1045700029F0F8EC29F0A8EC2DF0D2EF28F0E96E44
:10458000FF0EDA20EA6EEE50ED10120007C928F097
:1045900008C929F02DEC8BF012EC29F005C928F0A0
:1045A00006C929F042EC29F0D0EF2DF04EEC2CF0AA
:1045B0007BEC29F068EF2CF0FFEC29F0046E090E7B
:1045C000C2EF2AF0D890E936EA36E8061200BEECCF
:1045D000B1F022C000F0F2EF2BF0F1EC29F0EAECA0
:1045E00029F0FE0EDBCFE6FF1200040EDBCF00F059
:1045F000050EDBCF01F01200E66EBDEF2BF0040DCF
:10460000BAEC2CF0D2EF28F0060EF3CFDBFF070E4A
:10461000F4CFDBFF1200D9CFE6FFE1CFD9FF1200C4
:10462000E552E7CFD9FF12008E0EE926000EEA22EE
:104630001200B6EC2BF02FEC8BF012EC29F00CEC06
:104640002CF042EC29F047EC8CF0D7EC28F084EC0D
:104650002BF0F4EC8BF0E3EC8DF028C0A1F929C02D
:10466000A2F91200B1EC29F053ECB2F0050E2626A7
:10467000000E2722282229225EEF2BF0000EE66E84
:10468000060EE66E1200F0C604F0056A066A076AB6
:10469000100E2B6E270E2C6E2D6A2E6AF0C626F099
:1046A0006DEC29F008C02BF0E1EC2AF0F4EC8CF072
:1046B00026C002F027C003F0BBEC2DF052EC00F056
:1046C00026EF2AF0D950150FE96E94EF29F03BEC54
:1046D0002AF0C7EC2CF0020EF626000EF722F82284
:1046E0000800120000C0E6FF01C0E6FF1200020E43
:1046F000DBCF00F0030EDBCF01F01200FC0EDBCFAE
:10470000E9FFFD0EDBCFEAFFEF5012000450001668
:1047100005500116065002160750031600500110EE
:10472000021003101200EAEC29F01AEC5AF0E552DC
:10473000E5521200060EDBCF00F0070EDBCF01F0D2
:104740001200E3EC2CF007C027F008C028F009C0E5
:1047500029F073EC8DF024C007F025C008F026C0C6
:1047600009F004502424F36E05502520F46E065001
:104770002620A2EC29F00800F5CF02F002C003F0D9
:10478000026A3C0E0A6E4E0E0B6E010E0C6EE8CAEB
:104790000DF0E9CA0EF00F6A1200100EE66E270E39
:1047A000E66E52EC00F026EC2AF036EF2CF001C059
:1047B00029F0ABECB2F028C000F029C001F01200E3
:1047C000E3EC2CF00DC027F00EC028F00FC029F04C
:1047D00073EC8DF024C00DF025C00EF026C00FF054
:1047E0000A502424F36E0B502520F46E0C50262022
:1047F000A2EC29F09BEC2BF0C6EF2AF0BEEC29F0DE
:10480000EF501200066A076A98EC2CF008C02BF0F3
:10481000E1EC2AF0BEECB1F0F2EC2BF0D9500C0F29
:10482000BFEC2CF022508CEC2BF0DF2A010E120092
:10483000DBCF29F02FEC8BF012EC29F02C6A2D6ADB
:10484000E00E2E6E400E2F6ED0EC2DF02AEC2BF0E9
:104850005EEC8BF0E3EF8DF00026000E012259ECA8
:104860002DF0B0EF2CF0020EDBCFE6FF030EDBCF16
:10487000E6FF120051EC2AF098EC2CF042EC8BF0A1
:10488000D7EC28F02C6A2D6A12000C0EDBCF08F052
:104890000D0EDBCF09F00E0EDBCF0AF00F0EDBCFD3
:1048A0000BF008C026F0A2EC2BF042EC8BF012ECDF
:1048B00029F02C6A2D6A120042EC2DF0E76EFE0EF4
:1048C000E7CFDBFF1200E66E78EC9EF074EF2AF083
:1048D000040E00C0DBFF050E01C0DBFF1200006EFE
:1048E000016A280E005E000E015A1200200E006EB2
:1048F000500E016E010E026EDECF03F0DDCF04F02C
:10490000056A12004EEC2CF0B6EC2DF0C2EF2AF046
:1049100000500324F36E01500420F46E0250052071
:10492000A2EC29F00800F5501200DECF00F0DDCF38
:1049300001F01200BEEC29F000C0EEFF01C0EDFF57
:104940001200026A036A010E046E056A066A076AAB
:10495000120003C0DBFF290EE96E090EEA6E1D513D
:10496000EE24006E1E51EE20016E1F51EE20026EED
:104970002051EE20036E3551002636510122375169
:10498000022238510322120003C0DBFF2D0EE96E14
:10499000090EEA6E2151EE24006E2251EE20016EC6
:1049A0002351EE20026E2451EE20036E3951002671
:1049B0003A5101223B5102223C51032212002F6E38
:1049C00000C027F0B6EC2AF0D3EC2AF0060E070E52
:1049D000DBCF03F00001800E0314120000508CEFB7
:1049E0002BF0D8900436053606360736E806120056
:1049F000E66EE66AE3EC3FF0E552E5521200F80E8F
:104A0000DBCFE6FFF90EDBCFE6FF1200F3CFE6FFC8
:104A100001C0E6FF1200250EE96E090EEA6E0901DB
:104A20001951EE24006E1A51EE20016E1B51EE203A
:104A3000026E1C51EE20036E3151002632510122CC
:104A400033510222345103221200E66EA3EC2CF003
:104A5000B6EC2DF0E15E045031EC29F0FA0EE66E72
:104A6000FC0EE66E000E120002C0E6FF03C0E6FF79
:104A700012002C6E6DEC2CF0F4EC8CF027C001F0E1
:104A800093EC2CF02650EE260150ED221200DBCFE5
:104A90000AF0030E0926000E0A220B6A00500924B0
:104AA000F36E01500A20F46E02500B20A2EC29F0A4
:104AB0000800F550E66E1200720EE66EFD0EE66E10
:104AC000000E1200700EE66EFD0EE66E000E120075
:104AD000C6EC2AF0A9EC2BF0D950010FBFEC2CF05A
:104AE000000ED880EE54000EED541200BFEC2CF0F6
:104AF000E552E750EE6EED6A1200E4EC2BF0EF5059
:104B00001200EAEC29F0E66A1200D890003601366D
:104B100002360336E8061200FA0EDBCFE9FFFB0E81
:104B2000DBCFEAFF1200E66E98ECA8F08DEF2AF0DA
:104B30004DEC3FF0E552E5521200E3EC2CF006C0DC
:104B400027F007C028F008C029F073EC8DF003505F
:104B50002424006E04502520016E05502620026E8C
:104B60001200626B636B646B656B666B676B686B83
:104B7000696B12007EEC92F026EF2AF0050E005EC3
:104B8000000E015A040E1200F9DBEE50ED10120077
:104B9000F5DBEFCF00F01200D89000360136E804C4
:104BA0001200080EDB6A090EDB6A0AEC2BF00E0E0F
:104BB000DB6A0F0EDB6ADE6ADD6A12003D510C0D06
:104BC000BAEC2CF0190EE926090EEA221200000EAA
:104BD000005E060E015ABBEF2AF0FD0EDBCF00F09F
:104BE000FE0EDBCF01F012004EEC2CF0CCEC9FF06F
:104BF000026E050EE15E0250D4EC2DF0F350F4107D
:104C00001200BCDBEECF02F0EFCF03F01200010E7A
:104C1000006E016A026A036ADF501F0B120021DB7B
:104C2000020E12003EEF2DF0DBEC2CF0D5C9E6FFB2
:104C3000D6C9E6FFD7C9E6FFD8C9E6FF1200D950AA
:104C40000B0FBFEC2CF0000EEE6E060EED6E120098
:104C50000050025C015003581200AAEC2CF0CDC9A0
:104C600026F0CEC927F0CFC928F0D0C929F053EFDC
:104C7000B2F02F6EF4EC8BF0140E27C0DBFF150E94
:104C800028C0DBFF160E29C0DBFF170E2AC0DBFF92
:104C90001200FD0EDBCF28F0FE0EDBCF29F0035112
:104CA000285C006E04512958016E026A036A1200E2
:104CB000EF51640DD4EC2DF036EC2CF052EC00F0FA
:104CC000E552E5521200020E00C0DBFF030E01C0E8
:104CD000DBFF12003C0E006E4E0E016E010E026EE6
:104CE0001200060EDBCF02F0070EDBCF03F012003E
:104CF000FC0EDBCF00F0FD0EDBCF01F0120052DA2C
:104D0000EFCF00F012003ADBEE6AED6A1200590EA6
:104D1000E66EFD0EE66E000E120000500008000E5A
:104D200001541200D89001320032E8041200010E42
:104D30000026000E01221200020EF3CFDBFF030E4D
:104D40001200E66EE66AE66A1200DBEC2CF0DBC9C4
:104D5000E6FFDCC9E6FF12000FC95CF910C95DF976
:104D600011C95EF912C95FF9DBC960F9DCC961F9E3
:104D70001200EBEC2BF00A0EDBCF02F00B0EDBCFB8
:104D800003F0120009015C6B5D6B5E6B5F6B606B27
:104D9000616B1200E126D95024EF2BF03C0E046E1B
:104DA0004E0E056E010E066EE8CA07F0E9CA08F05D
:104DB000096A12003C0E036E4E0E046E010E056E63
:104DC000E8CA06F0E9CA07F0086A12004EEC2CF0B7
:104DD0008CEC74F0036E050EE15E0350120084EC5F
:104DE0002BF047EC8CF0E3EF8DF0DCD9020EC6DA45
:104DF0003BEF2CF0DB503F0B006E3D0E005C1200D1
:104E0000000ED8800B55000E0C551200680EE66E91
:104E1000FD0EE66E000E12005B0EE66EFD0EE66EF7
:104E2000000E12004E0EE66EFD0EE66E000E120033
:104E3000D890033604360536E806120015C900F08E
:104E400016C901F0006C011E000E0122026A036AFD
:104E50001200060E00C0DBFF070E01C0DBFF1200D0
:104E600015C900F016C901F0026A036A1200010EAA
:104E7000DBCF00F0020EDBCF01F012000F0E0801B5
:104E8000E915016E006AEA5112000F0E0801EC15D7
:104E9000016E006AED511200020EDBCF02F0030E2C
:104EA000DBCF03F0120027EC9FF074EF2AF066DAF4
:104EB000EF6A1200DBCFEAFFE80EE926080EEA22CD
:104EC0003BEF2CF094EC2BF0E66EE66AE66EE66AB9
:104ED000010EE66E1200A6D9140E1200D1C9E6FF2B
:104EE000D2C9E6FFD3C9E6FFD4C9E6FF120003C961
:104EF00005F904C906F90BC907F90CC908F912002C
:104F00000FC926F010C927F011C928F012C929F0DD
:104F1000120060DA020EE66E12000FC9E6FF10C939
:104F2000E6FF11C9E6FF12C9E6FF120036EC2CF0CD
:104F30006AEC01F0E552E552120034D9EE523BEF33
:104F40002CF00801EB51006E016A040E1200CCDA5D
:104F50000901120092EC0DF08DEF2AF0D2EC9EF0D8
:104F60008DEF2AF03FEC2EF0FE0EDB50020812000F
:104F7000130EE66EFE0EE66E000E1200025E000ECE
:104F8000035A01500318120002500008000E035487
:104F90001200E66E62EC72F0E55212000250005C04
:104FA00003500158120051ECA8F0E55212004D0ECA
:104FB0000701CB5D1200006E020EE15C1200F4CF1F
:104FC000DBFFD9501200010EDBCF03F0020EDBCF66
:104FD00004F0056A1200010E09010024A36F000EFF
:104FE0000120A46F1200E66A7DEC19F096DAE55212
:104FF0001200BFEC2CF00050EE260150ED22120002
:10500000E846FE0BF3061200010EDB407F0B120098
:105010000C0EDBCF02F00D0EDBCF03F012000A0EF8
:10502000DBCF00F00B0EDBCF01F01200030EF3CF4D
:10503000DBFF040EF4CFDBFF120013C900F014C92C
:1050400001F0026A036A12000C0EDBCF00F00D0EB5
:10505000DBCF01F01200D89003320232013200326D
:10506000E80612007EEC92F0E552E552F3CFF1F63D
:105070001200030EDB6A040EDB6A050EDB6A120007
:1050800018ECAEF074EF2AF0070EDB6A080EDB6A4C
:10509000090EDB6A1200F80EDBCF28F0F90EDBCF29
:1050A00029F01200080E28C0DBFF090E29C0DBFF23
:1050B000120078D8EFCF08F01200F36E010EDBCFAC
:1050C000F4FFF350F45C1200E851006E016A040E24
:1050D0001200E76E040EE7CFDBFF1200010E3EEF79
:1050E0002DF044C9E6FF45C9E6FF120052C9E6FFAC
:1050F00053C9E6FF120076EC74F0E552E552120057
:1051000003C9E6FF04C9E6FF120005C9E6FF06C9A8
:10511000E6FF120009C9E6FF0AC9E6FF1200000E09
:10512000DE6E060EDD6E1200020EE126FE0EDB5074
:105130001200090EDB503F081200BD0EE66EFF0E96
:10514000E66E000E1200AADB46EC22F068EF2CF0AF
:10515000FD0EDBCFE9FFFE0EDBCFEAFFF2EF21F021
:10516000BCDBE8EC2DF0BBEF2DF0AADB46EC22F027
:105170007CEF2CF0A5DBBCDB7CEF2CF0E66A13DFC8
:10518000FC0EF3CFDBFFFD0E1ADFFC0FBFEF22F0AA
:10519000E66ED9DB46EF22F0FCEC22F046EC22F082
:1051A00004EF23F0720EE926000EEA221200A1ECB1
:1051B0002DF02AC003F01200110EDBCF04F0120E06
:1051C000DBCF05F0130EDBCF06F0140EDBCF07F0BC
:1051D000AFDB150EDBCF2BF0160EDBCF2CF0170E4E
:1051E000DBCF2DF0180EDBCF2EF0E8EF2DF014EC16
:1051F00023F0B5EF2CF0A3EC21F0980EE66EFF0E35
:10520000E66E000E33EF22F0F7EC2DF046EC22F0C4
:1052100068EF2CF04AEC22F0F2EF21F04AEC22F099
:10522000A8EF2DF027C004F028C005F029C006F033
:105230002AC007F01200AFEC22F0050ECCEF2DF0E3
:105240000A0E58EC22F00E0E2D6E2E6AF3CF28F0C7
:10525000D7EC23F085DBE5EF21F0E15E005068EF4D
:105260002CF00B0EF3CFDBFF0C0EF4CFDBFF1200A4
:10527000E66EEEEF21F02C6E2D6A2E6AE7EC22F03E
:10528000A3EF21F02DEC8BF027C008F028C009F027
:1052900029C00AF02AC00BF0CEDB04C027F005C0FD
:1052A00028F006C029F007C02AF012002B6E2C6AE5
:1052B00014DBE7EF22F0FCEC22F01ADB04EF23F022
:1052C00027C00CF028C00DF029C00EF02AC00FF046
:1052D000B2DB00C027F0AFEF2DF0FFEC2DF0BEECFD
:1052E000B1F022C004F023C005F024C006F025C0B0
:1052F00007F024EF2DF0C2EC74F0026E070EE15EB1
:10530000025012003EEC23F098EF25F0F36E070EEA
:10531000F3CFDBFF450EE66EFD0EE66E000EF7ECFA
:105320002DF046EC22F0CCD3DACFEAFFD880000E85
:1053300049EF2DF0E5EC21F0010EDB50080D1ADBF2
:1053400014EF23F0F86EF4CFF7FFF3CFF6FF12005F
:105350000A0E58EC22F0BEEF25F0D950FC0FBFEF3B
:1053600022F072DBDFCF2BF0010EDBCF2CF0020E30
:10537000DBCF2DF0030EDBCF2EF01200E926000E5E
:10538000EA221200010EE76E77EC23F0E7500026C8
:10539000000E012272EC23F0E66AE66AE66AB3ECDC
:1053A00022F0050EDB5064081200D60EE66EFE0EEB
:1053B000E66E000EF7EC2DF053EF27F06FEC24F0C3
:1053C00072EC23F09BEF2DF02D6E2E6A00C028F0BA
:1053D000D7EF23F0FC0EDBCFE6FFFD0EDBCFE6FFC1
:1053E0001200FA0EDBCFE6FFFB0EDBCFE6FF12006A
:1053F000020EDBCFE9FF030EDBCFEAFF12004EDA2D
:10540000E5EF74F0A3EC21F07F0EE66EFF0EE66E82
:10541000000E33EF22F072EC23F0CE0EE66EFE0E9D
:10542000E66E000ED6EF22F00A0EB6DBC8EF2DF0C6
:10543000F5EC22F056DCA3EC21F09B0EE66EFF0E9D
:10544000E66E000E33EC22F0B9EF26F0E552E5529D
:10545000D4EF2DF094DAEE50ED101200AFEC22F004
:10546000050E0102F3CF01F00002F450012664DCC6
:1054700001C0DBFF1200A7DA03C027F004C028F048
:1054800005C029F073EF8DF0140EDBCF27F0150E59
:10549000DBCF28F0160EDBCF29F0170EDBCF2AF07A
:1054A0001200080EDBCF04F0090EDBCF05F00A0E68
:1054B000DBCF06F00B0EDBCF07F01200E66EE66ADC
:1054C000CA0EE66EFE0EE66E000E12000BEC23F026
:1054D000020EE126120095EC24F0D8900150120043
:1054E000AFEC22F0A1EF24F0006E050EE15E00505B
:1054F0001200026A036AD950080F41DAEEEC24F078
:105500004AEF22F06C0EE66EFD0EE66E000E120003
:10551000DB506FEC24F072EF23F0E552E552E552D8
:105520001200240E0EDC190EE66E090E63EC24F058
:1055300009013D6B12001C0E04DC400EE66E090EE4
:1055400063EC24F0C2EF26F044C900F045C901F035
:10555000026A036AC6DD34EF25F052C900F053C970
:1055600001F0026A036AC2DD34EF25F0F8DA5EEC7E
:105570008BF0E3EF8DF0040EDBCF02F0050EDBCFF6
:1055800003F01200E15E045068EF2CF000010224E9
:10559000006E000E0320016E1200A1EC26F0E66AF8
:1055A000E66AEEEF21F0060E28C0DBFF070E29C0E9
:1055B000DBFF1200080EDBCFE6FF090EDBCFE6FFB4
:1055C000120009C02CF00AC02DF00BC02EF0120002
:1055D000D950F80FBFEF22F0D950FA0FBFEF22F0E9
:1055E000010EDB50FFEF22F0A3EC21F05A0EE66E25
:1055F000FF0EE66E000E33EF22F0E66EE66ABF0E97
:10560000E66EFF0EE66E000E3FEF22F0E15E045004
:105610007CEF2CF00A0EDB6A0B0EDB6A0C0EDB6AE9
:105620000D0EDB6A120058EC22F0026A036A06ECE7
:1056300025F034EF25F0E15E08507CEF2CF0E66AAF
:105640003EEC23F0AEEF27F0FC0FE96EFF0EDA2000
:10565000EA6E12002C6A2D6A2E6A3F0E2F6E12001F
:10566000F5EC22F0030E12EF26F04FEC22F00D0EB7
:10567000FEEF23F0012272EC23F05CEF24F0B9EC92
:1056800022F0030EC8EF25F0070EF8D1AFEC22F0A0
:105690000150800B1200EDEC25F009010050035D74
:1056A000015004591200FAD892EF76F06AEC26F015
:1056B000E8CA03F0E9CA04F0056A12004BD953EFB7
:1056C000B2F0100EE66EFF0EE66E000EB0EF21F0A7
:1056D000E5D87EEF75F0E76E8CEC25F0E750FEEC38
:1056E00023F03F08120004EC23F077EC23F00001D4
:1056F000800E011412003EEC1FF0006E080EE15EF9
:10570000005010EF23F0DCD12C6A400E2D6E1C0EE1
:105710002E6E460E2F6E1200EE260150EE22025023
:10572000EE220350EE221200000EE66EE66A120030
:10573000E66EB3EF22F0F62A000EF722F8220800F8
:10574000F550120009C027F00AC028F00BC029F05C
:105750001200010E00C0DBFF020E01C0DBFF1200D1
:10576000A1EC26F095EC1CF0A7EF27F0040EDBCFA0
:1057700028F0050EDBCF29F01200060EDBCFE6FF86
:10578000070EDBCFE6FF12009AEC23F0006C011E3F
:10579000000E01221200F5EC22F04CEC27F028EF6D
:1057A00026F014EC23F0EECF08F0EFCF09F0120052
:1057B00095EC24F097EC26F072EF23F0280E005EB3
:1057C000000E015A72EF23F0F80EDBCFE9FFF90E5D
:1057D000DBCFEAFF1200080EDBCF00F0090EDBCFB3
:1057E00001F0120023C001F024C002F025C003F034
:1057F00012000122000E02220322120072EC23F09A
:1058000034EF25F00BEC23F0050EE1261200020E1A
:10581000DB6A030EDB6A120003C928F004C929F011
:105820001200E7EC22F032EF23F0C9EC27F093EFFF
:1058300023F03EEC23F07BEF28F0050E0026000E4F
:10584000012212000BEC23F094EF28F09CEC26F0E0
:10585000F4CFDBFF12000E0E11D19AEC23F0E7EF2C
:1058600025F077EC23F0D89001501200F3CFE6FF3B
:10587000F4CFE6FF1200E552E750EF6E12000C0E77
:10588000FEEF23F026C000F027C001F028C002F090
:1058900029C003F0120051DC38EF29F0E66EECEF7E
:1058A0002DF03BEC22F0100E2B6E270EE4DC2B0EBD
:1058B000E66EFF0EE66E000EB0EC21F0B5EF28F0BC
:1058C000E66E0F0EDBCFE6FF100EDBCFE6FF120019
:1058D000F3CFDEFFF4CFDDFF12002D6A2E6A00C089
:1058E00026F001C027F002C028F003C029F0120002
:1058F000C2EC74F006EF2EF00F0EF3CFDBFF100EAC
:10590000F4CFDBFF120019DC3FEF22F070DC4AEC31
:1059100022F0030E1200D00EE66EFE0EE66E000EB2
:1059200073DCADEF29F0D9CFE9FFDACFEAFF12003F
:1059300004C026F0FFEF2DF0E80E2B6E030E2C6E48
:105940002D6A2E6A12000B0EDBCFE6FF0C0EDBCFAA
:10595000E6FF12000A0E2B6E2C6A2D6A2E6A1200C8
:1059600028C0E6FF29C0E6FF1200EECF00F0EFCF1F
:1059700001F01200F3CFE9FFF4CFEAFF1200E96E65
:10598000DACFEAFF1200DBCFE6FFE66A1200005032
:105990002424F36E01502520F46E02502620A2EF3D
:1059A00029F0320E0901016A0D25006E0E51012207
:1059B000640EE4EF29F0006E090E2DEF29F09DEC46
:1059C00028F0DCEF22F00B0E2C6E2D6A2E6A1200EE
:1059D00014EC23F0060E12003BEC22F0E80E2B6EC6
:1059E000030E49DC61EF2BF0DE0EE66EFE0EE66E76
:1059F000000EA3EC28F03FEF2EF021C900F022C9E1
:105A000001F023C902F024C903F0120012DF020ED4
:105A10000CDF78DC010E1200E10EE66EFE0EE66E83
:105A2000000EF7EF2DF00EEC29F0D2EC28F0EF503D
:105A3000E66E0EEF29F027C02CF028C02DF029C00B
:105A40002EF02AC02FF0120022C026F023C027F02B
:105A500024C028F025C029F01200A8EC28F00D0E73
:105A6000FEEF23F057EC27F00AEF29F0C8EC28F0FE
:105A700031EF29F0C8EC28F00FEF26F0005C000EA3
:105A800001581200FE0EDBCFE6FF39EC2FF08DEF50
:105A90002AF0EE54000EEE54000EEE54000EEE54BA
:105AA0001200D2EC28F0EF50E66E4AEC22F0020E23
:105AB0001200022203220A0E2B6E2C6AB0EF28F08D
:105AC000080EF3CFDBFF090EF4CFDBFF1200D2ECA0
:105AD00028F0030E12000BC900F00CC901F0A8EF6A
:105AE00029F0C2EC74F0006E070E2DEF29F0E66E7F
:105AF000E66A9DEC28F0A7EF22F0D6EC22F0B8EC95
:105B000027F0A3EF28F05DEC8BF0D7EC28F04AEFFC
:105B100022F05BEC29F006EC27F0CCEF28F0FCEC4F
:105B200022F07BEC29F073EF2BF05BEC29F012EC08
:105B300027F0CCEF28F0E5EC21F004EC28F0FFEFA3
:105B400022F027C000F028C001F029C002F01200A6
:105B5000D890E936EA36D890E936EA36120001C024
:105B600028F002C029F003C02AF01200C8EC75F03A
:105B7000046E0B0E120026C0E6FF27C0E6FF1200DF
:105B800083EC26F00AEF29F0A8EC28F03FEF2CF088
:105B9000E5EC21F04FEF22F058EC22F006EF25F073
:105BA000F4EC8BF0D7EF28F0F3CF00F0F4CF01F056
:105BB000120014EC23F0020E1200E66EE66A4BEFC0
:105BC0002CF0060EE0DE9FDE070EDDDE83EF2CF00C
:105BD00053ECB2F042EF2CF0DECFE6FFDDCFE6FF74
:105BE00012002BDE0A0EE4EC29F0B0EF2CF0E66E8A
:105BF0003EEF23F00AEC29F0B8DE0AEF29F005C0E9
:105C000027F006C028F007C029F01200006E070E2A
:065C1000E15E00501200ED
:0A5C16000A01A46BA56B12000A013D
:105C2000636B12007F0E0501C85D08E10501CC0E13
:105C3000FD6FF70EFE6F000E5BEF3BF00A01010EE9
:105C4000646F050E81EC3CF00501C00EFD6FF70E90
:105C5000FE6F000E5BEC3BF00A0E81EF3CF07F0E16
:105C60000501C85D04E105019CEC3BF006D005018F
:105C7000BB0EFD6FF70EFE6F000E5BEF3BF044ECCA
:105C80003DF07F0E0501C85D05E139EC3CF04DECBF
:105C90003FF05AD00A01930549E1450E0601055D22
:105CA00045E0410E055D42E0610E055D3FE0670E97
:105CB000055D3CE0500E055D39E0020E05C6DBFFD8
:105CC000060EE66E060EE66E000EE66E050EBBECE8
:105CD0003BF089EC3AF0CBEC3AF002E6A2EC3BF078
:105CE00005E2A5EC3CF0F7E3DB2AF5D7000EE66E03
:105CF000050EE66E96EC3DF0000EE66E050E08EC25
:105D00003AF0B30EE66EF70EE66E000EFBEC39F0DD
:105D1000020EDBCF07F6080EE66E060EB4EC3DF081
:105D2000000EE66E050EE66ED8EC3BF039EC3CF06A
:105D300096EC3DF0BEEC3AF024EC3CF039EC3CF053
:105D400076EC99F0E552E552E552E55205019CECFE
:105D50003BF05BEC3BF0030EE15C02E2E16AE552F2
:105D6000E16E04EF3AF0FFEC39F0050EE126D65073
:105D7000016E006A030E00C0DBFF040E01C0DBFFF2
:105D8000D75043EC3BF0DF6A080EDF5C0BE2DF50DC
:105D9000EA6AE80FE96E080EEA22EF5043EC3BF0A6
:105DA000DF2AF2D7030EDBCFE6FF040EDBCFE6FFE0
:105DB0000DEC95F0E552E552DF6A160EDF5C11E25C
:105DC0000AEC3AF004BE0568F0EC3AF0DF50EA6AFB
:105DD000650FE96E0A0EEA22E552E750EF6EDF2A00
:105DE000ECD70A017B6B090EFBEC3CF07AEC3AF045
:105DF000D80EE66E040EE66E7EEC3AF0A3EC3DF0B3
:105E00007EEC3AF0160EE66EE66AA7EC3BF0FFEC8D
:105E1000ABF0026E0A0EE15E02500501AB0EFD6FA3
:105E2000F70EFE6F000E5BEC3BF0A7EC3BF030ECA6
:105E30003BF012EC3DF0E8EC3AF076EC99F000EC37
:105E40003DF0050112EC3DF0080EFBEC3CF07AEC65
:105E50003AF07EEC3AF030EC3BF09CEC3BF05BEC43
:105E60003BF0050EE15C02E2E16AE552E16E04EF0F
:105E70003AF06BEC3CF039EC3CF0A3EC3DF039EC43
:105E80003CF024EC74F0E552E55276EC3AF0FE0E6C
:105E9000DB50020A11E0030A03E0010A1EE109D007
:105EA00029EC3BF0DFEC3BF003E1DE52DD50011862
:105EB00014E0DCEC3CF011D029EC3BF0DFEC3BF0E3
:105EC00003E1DE52DD50011808E0ACDEDCEC3CF012
:105ED000010EF36EFE0EF3CFDBFFFE0EDB50006E05
:105EE000020EE15C02E2E16AE552E16E005004EF6D
:105EF0003AF048EC3DF0020EFBEC3CF030EC3CF0AC
:105F0000ACEC3BF0A20EE66EF70EE66E000EDEEC99
:105F100039F03EEC3CF024EC3CF01EEC3CF0E66E3C
:105F2000A6EC3DF086EC3BF03EEC3CF08EC9E6FF83
:105F30008FC9E6FFB4EC39F009019051A1EC3CF0B7
:105F4000090194510F0A20E0020A18E0090A10E042
:105F5000060A08E0030A1EE1960EE66EF70EE66EEC
:105F6000000E1DD08E0EE66EF70EE66E000E17D0F8
:105F7000880EE66EF70EE66E000E11D07F0EE66E0E
:105F8000F70EE66E000E0BD0760EE66EF70EE66E9E
:105F9000000E05D06D0EE66EF70EE66E000EAFEC4D
:105FA0003AF009019651040A18E0070A10E0020AC3
:105FB00008E0010A18E1630EE66EF70EE66E000EC9
:105FC00014D05A0EE66EF70EE66E000E0ED0530E8B
:105FD000E66EF70EE66E000E08D0460EE66EF70E81
:105FE000E66E000E02D01EEC3CF0AFEC3AF0A9ECED
:105FF0003AF04D080FE1A1C9E6FFA2C9E6FFB4ECF3
:1060000039F0A3C9E6FFA4C9E6FF6CEC3DF045EC0E
:106010003CF016D0A1C900F0A2C901F0040EB1EC09
:106020003BF0FDE1ADEC3CF03EEC3CF0A3C900F0F0
:10603000A4C901F0040EB1EC3BF0FDE1ADEC3CF085
:106040003EEC3CF009019151A1EC3CF092C9E6FF15
:1060500093C9E6FFB4EC39F009019751A1EC3CF08B
:1060600009019851A1EC3CF009019551A1EC3CF0DB
:1060700009019451A1EC3CF009019651A1EC3CF0CE
:10608000DDC900F0016A00BE01689BEC3DF0DEC98D
:10609000E6FFDFC9E6FFB4EC39F0E5C900F0016ABC
:1060A00000BE01689BEC3DF0DAEC3AF06CEC3DF0A0
:1060B000B8EC3CF03EEC3CF0F7C9E6FFF8C9E6FF6F
:1060C000B4EC39F0940EE66E0A0EEBEC39F0040EE7
:1060D000E15C02E2E16AE552E16E005004EF3AF061
:1060E0006BEC3CF08AEC3BF03F0EE66EF70EE66E92
:1060F000000E79EC3DF035EC3AF056EC3DF000BE88
:106100000168CCEC39F0960EE66E0A0E4CEC3DF0D0
:1061100002E2E16AE552E16E005004EF3AF0FFEC72
:1061200039F0070EE126380EE66EF70EE66E000E29
:10613000A3EC3AF07AEC3AF0DF6A040EDF5C6EE230
:10614000E6EC3BF0EFCF00F0000EE76E0018E8AE93
:1061500002D0003403D0E750D880005451E2DF5021
:10616000EA6AC70FE96E090EEA22EFCF04F004C015
:1061700029F01CEC8BF027C000F028C001F029C0EA
:1061800002F02AC003F0560E2C6E0E0E2D6E8D0EF0
:106190002E6E3E0E2F6EF4EC8BF012EC8EF0030E92
:1061A00026C0DBFF040E27C0DBFF050E28C0DBFF87
:1061B000060E29C0DBFFB7EC3DF0D950030FA6EC6B
:1061C0003AF0E66AE66AE66A7EEC3AF0C8EC75F008
:1061D000006E0B0EE15E00507AEC3AF0E6EC3BF01C
:1061E000EF50D80F006E016A00BE016886EC3CF0EB
:1061F0001EEC3CF0E66E9FEC3DF01EEC3CF005D052
:10620000330EE66EF70EE66E000EE66E7EEC3AF0AA
:106210005DEC3CF07AEC3AF0DF2A8FD7E4C900F06D
:10622000016A00BE016886EC3CF0E66AE66AE66A4E
:106230009FEC3DF0980EE66E0A0EEBEC39F0070E7F
:10624000E15C02E2E16AE552E16E005004EF3AF0EF
:1062500044EC3DF0010EF36E020EF3CFDBFFF36E64
:10626000DB6E5EEC3BF02C0EE66EF70EE66E000E7B
:106270008EEC3DF00F0EF66E000EF76E000E85EC04
:106280003AF0100EF66E000EF76E000E85EC3AF046
:10629000B4EC3AF024EC3CF0EDEC3BF030EC3CF0AC
:1062A000020EE4EC3CF0B4EC3DF0ABEC3DF0AE0E95
:1062B000E66E090E30EC3AF00901E95159EC3CF078
:1062C0000601F45159EC3CF0C80EE66E060E30ECB7
:1062D0003AF0EC0EE66E090E30EC3AF09A0EE66EED
:1062E0000A0EEBEC39F0030EE15C02E2E16AE552E2
:1062F000E16E005004EF3AF0FFEC39F0060EE126B3
:106300000901A951AA11AB11AC1109E1020EDB6A16
:10631000030EDB6A040EDB6A050EDB6A1DD0A90ED4
:10632000E96E090EEA6EEE500901A55D006EEE50B1
:10633000A659016EEE50A759026EEE50A859036E91
:10634000020E00C0DBFF030E01C0DBFF040E02C023
:10635000DBFF050E03C0DBFF09019951E66EE66A1B
:106360001E0EE66EF70EE66E000E8EEC3DF0090195
:106370009A5159EC3CF009019E5159EC3CF0C0C9CE
:1063800000F0016A00BE0168CCEC39F00901C1518E
:1063900059EC3CF0C2C900F0016A00BE0168CCECC7
:1063A00039F0CBC9E6FFCCC9E6FFB1EC39F0CDC975
:1063B000E6FFCEC9E6FFCFC9E6FFD0C9E6FF45EC50
:1063C0003AF009019F5159EC3CF0D950020FA6EC6C
:1063D0003AF045EC3AF0ADC900F0016A00BE016840
:1063E000CCEC39F009019B5159EC3CF0E2C900F0CA
:1063F000016A00BE0168CCEC39F0E1C900F0016A25
:1064000000BE0168CCEC39F057EC3AF01EEC3CF0E1
:1064100065EC3AF009019C5159EC3CF001EC3BF081
:106420001EEC3CF065EC3AF009019D5159EC3CF052
:106430009C0EE66E0A0EEBEC39F0060EE15C02E211
:10644000E16AE552E16E005004EF3AF06BEC3CF08B
:10645000170EE66EF70EE66E000EA3EC3AF030EC87
:106460003CF00701CF51D011D11116E0CFC7F6FF94
:10647000D0C7F7FFD1C7F8FF0800F5500DE0CFC730
:10648000E6FFD0C7E6FFD1C7E6FFE7EC39F01EEC28
:106490003CF0E66EE7EC39F0070EE66EF70EE66EBE
:1064A000000EE66EE7EC39F0A20EE66E0A0E4CEC3A
:1064B0003DF002E2E16AE552E16E005004EF3AF08D
:1064C0006BEC3CF0F4EC3BF0000EE66EF70EE66E83
:1064D000000E0CEC3BF0ACEC3BF0B1EC39F00901F8
:1064E0009F5159EC3CF056EC3DF000BE0168CCECFD
:1064F00039F08AEC3BF053EC3DF035EC3AF0FD0E10
:10650000DB0404E19E0EE66E0A0E03D0A00EE66EDA
:106510000A0E4CEC3DF002E2E16AE552E16E0050F9
:1065200004EF3AF0FFEC39F0090EE126010EB6EC6B
:106530003BF0020EB6EC3BF069EC3BF0EE50ED1098
:1065400001E138D1FD0EDBCFDEFFDBCFDDFFA9ECB3
:106550003AF009E0A9EC3AF0200805E0DF2A010E44
:10656000F6E3DB2AF4D7A9EC3AF0200801E022D1C7
:10657000FBEC3BF001E3DB2AEF6A29EC3CF0A7ECF3
:106580003BF0C0EC3BF001E115D1090EE66E94EC56
:106590003AF0D80EE66E040EF6EC39F029EC3CF039
:1065A00099EC3AF029EC3CF070EC3BF039EC3CF023
:1065B000E8EC3AF0D8EC3BF039EC3CF024EC3CF061
:1065C000C0EC3BF001E0F6D029EC3CF0000EE66EAA
:1065D000060EBBEC3BF0A7EC3BF071EC3AF0D80EAA
:1065E000E66E040EF6EC39F039EC3CF099EC3AF03A
:1065F00039EC3CF070EC3BF0E8EC3AF019EC3DF093
:106600004DEC3BF020EC3BF002E6A2EC3BF00AE262
:1066100085EC3DF0C1EC3AF0060EDB2A070EF2E302
:10662000DB2AF0D7E8EC3AF021EC3DF04DEC3BF002
:1066300020EC3BF002E6A2EC3BF00AE285EC3DF0F8
:10664000BEEC3AF0060EDB2A070EF2E3DB2AF0D7A7
:106650000A01010E636F0A0EE66E94EC3AF0E1EC6B
:1066600039F050084EE10A01935127E1060EDB6A2A
:10667000070EDB6A20EC3BF004E6160E005C000E11
:10668000015819E20AEC3AF004BE0568F0EC3AF061
:10669000060EDBCFE9FF070EDBCFEAFF7C0EE92613
:1066A0000A0EEA22E552E750EF6E060EDB2A070ECD
:1066B000E1E3DB2ADFD70A01926B936BF80EE66EFB
:1066C000F60EE66E000EFBEC39F010EC3CF071ECCF
:1066D0003AF012EC2EF0D1EC3CF00A01010E936F6F
:1066E000E66E94EC3AF0E80EE66E040EF6EC39F045
:1066F00010EC3CF099EC3AF010EC3CF070EC3BF014
:1067000002D00A01936B0601F69F5EEC3BF0D60EB9
:10671000E66EF60EE66E000EAEEC3DF00F0EF66E77
:10672000000EF76E000E6FEC3CF0D5EC39F0100E59
:10673000F66E000EF76E000E6FEC3CF0D5EC39F003
:10674000B4EC3AF093EC3CF0EDEC3BF049EC3CF06F
:106750000701CC51CD11CE110CE0CCC7E6FFCDC75F
:10676000E6FFCEC7E6FF93EC3CF05DEC3CF049EC75
:106770003CF0080EE4EC3CF0D5EC39F00601F551A4
:1067800067EC3DF00601F651E66EE66A1EEC3CF061
:10679000E66E93EC3CF02DEC75F091EC3DF049EC9D
:1067A0003CF00601F75167EC3DF0140E62EC3AF054
:1067B000D1EC3CF0090EE15C02E2E16AE552E16EE7
:1067C00004EF3AF044EC3DF00A0163511AE1070E80
:1067D000E66EE66ACE0EE66EF60EE66E000EB1ECE2
:1067E0003DF0C5EC3BF001E0B9D0070E69EC3AF0A2
:1067F00099DEE552E5520501060ED06F0E0ED16FFF
:10680000ADD0C4EC3AF039EC3CF029EC3CF03EEC75
:106810003DF024EC3CF0C1EC3AF0050EE66EE66A81
:10682000C80EE66EF60EE66E000E79EC3DF0C5EC95
:106830003BF006E0400EE66E98EC40F0E5528ED05C
:10684000D950FD0F3AEC3DF0050EEE6E060EED6EE2
:10685000CFEC3AF0EF50450835E129EC3DF04D081A
:1068600031E169EC3BF0020EEE26000EED22C4ECA5
:106870003AF0010EE66E050EE66E010E69EC3AF096
:106880003EEC3DF089EC3AF0CBEC3AF002E6A2ECBB
:106890003BF005E2A5EC3CF0F7E3DB2AF5D724EC6E
:1068A0003CF0010EE66E050E08EC3AF0CFEC3AF043
:1068B000EFCF00F5D950FD0F3AEC3DF0000EEE6E33
:1068C000050EED6E0601F6BF03D00601150EF76F3B
:1068D000CFEC3AF0EF50430A37E0190A11E01B0AF7
:1068E0003DE1C10EE66EF60EE66E000EFBEC39F0F1
:1068F0000A01645133E112EC2EF03FEC2EF01ED071
:1069000029EC3DF030081DE00901010EE86F0A0195
:10691000645124E112EC2EF0E66A79EC2FF0E55296
:10692000E66A70EC30F0E552E66A8FEC30F0E55242
:10693000E66A8EDCE552E66ADFDCE5522FEC2EF0EB
:106940000DD00901E86B0AD0010E69EC3AF00ED8BF
:10695000E552E5520A01645101E1D8D9030EE15C28
:1069600002E2E16AE552E16E04EF3AF048EC3DF0F4
:10697000FD0EDBCFDEFFDBCFDDFFA9EC3AF009E057
:10698000A9EC3AF02C0805E0DF2A010EF6E3DB2A39
:10699000F4D7A9EC3AF02C0805E1FBEC3BF001E35D
:1069A000DB2AEF6AFD0EDBCFE6FFFE0E02EC3CF0C9
:1069B000F3CFA4FAF4CFA5FADECFA6FADDCFA7FA7B
:1069C000040EE15C02E2E16AE552E16E04EF3AF0A6
:1069D000FFEC39F0060EE126020E81EC3CF0310EA0
:1069E0000A01A41901E1A55101E170D1290EA419F0
:1069F00001E1A55101E158D1280EA41901E1A551E9
:106A000001E126D1060EA41901E1A55101E11CD135
:106A1000050EA41901E1A55101E10DD1040EA4193F
:106A200001E1A55101E1BED0030EA41901E1A55178
:106A300001E180D0020EA41901E1A5512AE0010E66
:106A4000A41901E1A55102E0000E57D1DE6ADD6A0A
:106A5000CBEC3AF004E6100E005C000E015801E3A6
:106A60004BD124EC3CF0B60EE66EF60EE66E000E50
:106A7000AEEC3DF0100E67EC3DF093EC3BF0EF50C8
:106A800067EC3DF03FEC2EF0DF2A010EE1E3DB2A5C
:106A9000DFD777EC3BF0E1EC39F008E00FEC3DF0AC
:106AA00005E01AEC3CF0F7E3DB2AF5D70FEC3DF0FC
:106AB00001E0BAD036EC3BF001E3DB2AD5EC3CF048
:106AC00001E0ACD009EC3CF004E6100E025C000ED4
:106AD000035801E3A3D0A6EC3DF002EC3CF0F350E8
:106AE000E66E93EC3BF0E552E750EF6ECBEC3AF0FC
:106AF00004E6080E005C000E015810E335EC3CF093
:106B00000AEC3DF0080E005E000E015A180E00243B
:106B1000E66E98ECA8F0E552E552E5523EEC3BF00B
:106B20000F0EEE1804E1ED5002E1A7EC9BF055ECDE
:106B30003BF07FD0DE6ADD6ACBEC3AF004E6200E53
:106B4000005C000E015801E3D7D0DFCFE6FF94ECE4
:106B50003AF03EEC3BF0090EEE1804E1ED5002E194
:106B6000CFEC3BF024EC3CF0AB0EE66EF60EE66E9E
:106B7000000EAEEC3DF0200E67EC3DF035EC3CF045
:106B80001EEC3CF0E66E040EDBCFE6FF050E86EC55
:106B90003BF049EC3CF03FEC2EF0DF2A010ECCE359
:106BA000DB2ACAD777EC3BF0E1EC39F008E00FECD8
:106BB0003DF005E01AEC3CF0F7E3DB2AF5D70FECEB
:106BC0003DF032E136EC3BF001E3DB2AD5EC3CF062
:106BD00025E109EC3CF004E6180E025C000E0358B7
:106BE0001DE235EC3CF0DFCFE6FF98ECA8F0E55273
:106BF000E552E55255EC3BF0BBDB3EEC3BF0020EC0
:106C0000EE1801E1ED5007E03EEC3BF00E0EEE1801
:106C10001CE1ED501AE1A7EC9BF017D0D90EE66EFF
:106C2000610EE66E010E05D0AD0EE66E610EE66EEB
:106C3000010E9EDB0AD055EC3BF050EC3DF0040E0B
:106C4000E66E98EC40F057D0F2DA3FEC2EF054D0DC
:106C500077EC3BF0B6DB08E00FEC3DF005E01AEC1A
:106C60003CF0F8E3DB2AF6D70FEC3DF015E136EC0B
:106C70003BF001E3DB2AEF6A7EEC3BF01AEC5AF0C2
:106C8000E552E55235EC3CF030EC3BF0BB0EFD6FCD
:106C9000F70EFE6F000E23D012EC2EF0AD0EE66E56
:106CA000610EE66E010E21D005019F0EFD6FF60EFE
:106CB000FE6F000E5BEC3BF07EEC3BF030EC3BF00B
:106CC000990EFD6FF60EFE6F000E09D07EEC3BF0C4
:106CD00030EC3BF0970EFD6FF60EFE6F000E5BEC96
:106CE0003BF0050EEFDB55EC3BF050EC3DF0020EB7
:106CF000E66E62EC72F0E552010E006E060EE15C8B
:106D000002E2E16AE552E16E00507ED30601F6BF71
:106D100003D00601160EF76F020E81EC3CF0280E30
:106D20000A01A5AF02D0D89003D0A45D000EA559EA
:106D300007E3A53507E2A4513108000EA55502E28C
:106D400012EC2EF00801F051F111F21119E0A6CA6F
:106D5000E6FFA7CAE6FFA4CAE6FFA5CAE6FF010E42
:106D6000E66E07D0F2C8FBFFF1C8FAFF0801F05148
:106D7000F96EF8DF006E050EE15E005000090AE1D1
:106D800027DE000907E1480EE66E620EE66E010E90
:106D900050EC3DF02FEC2EF00A01A46BA56BA6CAB7
:106DA000E9FFA7CAEAFFEF6A120029DB0A01635173
:106DB0002CE06451000829E3020E84DB8F0EE66E9E
:106DC000F60EE66E000E17DB840EE66EF60EE66E2D
:106DD000000E53EC3BF029EC3CF083DB7B0EE66EBF
:106DE000F60EE66E000E53EC3BF0AA0EE76EFB0EBD
:106DF000DBCFE9FFFC0EDBCFEAFF15EC3CF0EF6ADE
:106E0000F4EC3BF06EDBD1EC3CF0FED248EC3DF014
:106E1000020EDB6A030EDB6A0A01635101E194D0C2
:106E200069EC3BF0EE50ED1001E18ED0FC0EDB5032
:106E300001E18AD0FC0EDBCFE6FFE66A220EB1EC60
:106E40003DF010EC9EF0026E050EE15E02503EEC4D
:106E50003CF0F3CF00F0F4CF01F0F350F41036E043
:106E60001AEC3CF001E3DB2ADBDBDBCFE7FF005071
:106E7000E75EFC0EE7CFDBFF020EDBCF28F0030E50
:106E8000DBCF29F0FD0E28C0DBFFFE0E29C0DBFFA3
:106E900098DA1AE096DA220817E0C2DBDB5000012C
:106EA00001AE02D0D89003D0005C000E01580CE275
:106EB0000FEC3DF004E1BFEC3CF02E0EEF6E1AEC4F
:106EC0003CF0E6E3DB2AE4D7CFEC3BF0290EE66E9C
:106ED000E66ACF0EE66EF70EE66E000E8EEC3DF023
:106EE000D2EC3BF00EE029EC3CF0770EE66EF60EAD
:106EF000E66E000EB4EC3DF0BAEC74F0006E070ED6
:106F00000BD0600EE66EF60EE66E000EB4EC3DF0B1
:106F10008CEC74F0006E050EE15E005030EC3CF03D
:106F20000A016451000805E2140E81EC3CF0DE6AAF
:106F3000DD6A12EC2EF0D1EC3CF0A0DBEE50ED104F
:106F400003E1140E81EC3CF0040EE15C02E2E16A24
:106F5000E552E16E59D253DA0C0EE126A3C9DEFFE9
:106F6000A4C9DDFF020EA1C9DBFF030EA2C9DBFF2E
:106F7000040ECDC9DBFF050ECEC9DBFF060ECFC95F
:106F8000DBFF070ED0C9DBFF5C0EF0DBF60EF36E05
:106F9000090EF3CFDBFF000EF36E0A0EF3CFDBFF1B
:106FA0004B0E0701CB5D59E10AEC3DF0040ED9DB35
:106FB000FEE170DA28C0DEFF29C0DDFF020EDBCF64
:106FC00000F0030EDBCF01F0040ECBDBFEE162DA52
:106FD00029C001F0020E28C0DBFF030E29C0DBFF31
:106FE000040E006ED950040F3AEC3DF000501F0B18
:106FF000EECF26F0EECF27F0EECF28F0EECF29F03F
:1070000007E0D8902636273628362936E806F9E1F3
:10701000050E2626000E2722282229220A0E2B6E74
:107020002C6A2D6A2E6A53ECB2F0040E26C0DBFFE8
:10703000050E27C0DBFF060E28C0DBFF070E29C0A8
:10704000DBFF580E93DBF60EF36E090EF3CFDBFF7A
:10705000000EF36E0A0EF3CFDBFF090199A58FD066
:10706000010EF36E0B0EF3CFDBFF09019651040AFC
:1070700018E0070A10E0020A08E0010A19E14C0EC4
:10708000E66EF60EE66E000E11D0410EE66EF60EBE
:10709000E66E000E0BD0380EE66EF60EE66E000EB3
:1070A00005D0290EE66EF60EE66E000EE66E79D974
:1070B000090194510F0A20E0020A18E0090A10E0C1
:1070C000060A08E0030A20E1200EE66EF60EE66EE0
:1070D000000E17D00A0EE66EF60EE66E000E11D008
:1070E000FC0EE66EF50EE66E000E13D0F20EE66EA6
:1070F000F50EE66E000E05D0E00EE66EF50EE66EBD
:10710000000EE66E4ED909D0CF0EE66EF50EE66E95
:10711000000EE66E46D90B0EDB6A0B0EDB5036E036
:107120008EC9E6FF8FC9E6FFCC0EE66EF50EE66E61
:10713000000E40D909019051E66EE66AC90EE66E6E
:10714000F50EE66E000E36D9C70EE66EF50EE66E4B
:10715000000EE66E26D90901800EF81517E1F7C971
:10716000E6FFF8C9E6FFBC0EE66EF50EE66E000E11
:1071700021D9B60EE66EF50EE66E000E05D0A90E0C
:10718000E66EF50EE66E000EE66E0BD9E5DAA10EA0
:10719000E66EF50EE66E000E0DD99F0EE66EF50E4C
:1071A000E66E000EE66EFDD8FDDA08E05EDB8F0EBF
:1071B000E66EF50EE66E000EFDD882DB5FDAEE506D
:1071C000ED1008E041DB800EE66EF50EE66E000E77
:1071D000F1D876DBB7EC3DF0D950040FB7D9780E73
:1071E000E66EF50EE66E000E8EDA006E0B0EE15EB8
:1071F0000050A0DB65DB0901F551F6110CE0DAD98E
:10720000700EE66EF50EE66E000E7DDA046E0B0E65
:10721000E15E04508FDBBADB00C0F3FF01C0F4FF76
:107220000C0EE15C02E2E16AE552E16EEDD053DB67
:1072300068DB8F0EE66EF60EE66E000E84D910DB6C
:1072400003DB89DEE552E552020EE15C02E2E16A0F
:10725000E552E16ED9D076EC3DF04E0EE66EF50EBD
:10726000E66E000EC8D8A2D902E2E16AE552E16EEC
:10727000CBD076EC3DF0230EE66EF50EE66E000EFA
:10728000BAD894D902E2E16AE552E16EBDD076EC5B
:107290003DF062DAF30EE66EF40EE66E000E8EEC52
:1072A0003DF0EC0EE66EF40EE66E000EE66E8FD844
:1072B0007DD902E2E16AE552E16EA6D076EC3DF0BE
:1072C0000701CAA307D0F3D8C50EE66EF40EE66E2A
:1072D000000E06D0ECD8AD0EE66EF40EE66E000E93
:1072E00079EC3DF045DBBCDA8CD9A50EE66EF40EE8
:1072F000E66E000EEAD8A20EE66EF40EE66E000E02
:10730000E66E65D853D902E2E16AE552E16E7CD0BF
:10731000EDDBC80EE66E060EE66E9A0EE66EF40E15
:10732000E66E000E79D932DB026A036AEFDA02C038
:10733000E6FF03C0E6FFB7DBE5EC74F0046E090E70
:10734000E15E04508DDAD950F90FE96EFF0EDA20B4
:10735000EA6E43DB9AD82AD902E2E16AE552E16E8D
:1073600053D0A1DBABEF3DF0B7DB8FDA3EEF3CF063
:10737000E66EA4CAE6FFA5CAE6FFA30EE66E610E9E
:10738000E66E010EB6DBB6DA8BDA8CEC74F0036EC7
:10739000050EE15E03501200B9DA85DBABDA30EF9F
:1073A0003CF057DA8ADA9AEF3CF0E66EBCDA6DDA36
:1073B00049EF3CF0D6DB69DA9AEF3CF09ADB45EF17
:1073C0003CF0DDDAEF50120087DB7AEF3CF03CDA7C
:1073D00074DA30EF3CF0E66EFE0EDBCFE6FF39EC00
:1073E0002FF0E552E552E552006E1200E66E3DDAEE
:1073F000AADB35EF3CF07DDB27EC9FF08AD3D9CFB9
:10740000E6FFE1CFD9FF1200E552E7CFD9FF120026
:1074100073DB81D2EA0E006E620E016E010E026E07
:1074200075DAE66E14EC95F0E552E7CF02F0E5521E
:10743000E7CF01F0E552E7CF00F0F3CF03F0F4CF50
:1074400004F0400E2D6E2E6AF3CF28F0F4CF29F011
:10745000CEEC8CF024C003F025C004F0056A1200C5
:10746000E66E21DB9ADA30EF3CF092EC76F038DB16
:10747000D5C9E6FFD6C9E6FFD7C9E6FFD8C9E6FFFA
:1074800012DB92EC76F070EF3DF00DDBE5EC74F082
:1074900070EF3DF0050E0026000E01220A0E2D6E43
:1074A0002E6A00C028F001C029F0ABEFB2F05FDB1C
:1074B000EAC900F0016A026A036AEAC9E6FF01C08C
:1074C000E6FF94D21EDA12EF2EF04EDB51DA30EFE7
:1074D0003CF0E76E5BDAE7500026000E012286EFF3
:1074E0003CF0C7D992EC9EF000EF3DF0E552E5523A
:1074F00030EF3CF0DE52B4D9DD521200010EDBCF8A
:10750000E6FF020EDBCFE6FF1200E9D92DDBABEF81
:107510003DF0100EE66EE66AE80EE66E040EECDA5A
:107520009EDADE6ADD6A120051ECA8F0E5523EEF09
:107530003CF06BDAF3CF02F0F4CF03F0F3CFE6FFC9
:10754000F4CFE6FF1200D5DA5DEF3CF093DAEDEF11
:107550003CF0DECFE9FFDDCFEAFFEF501200E66E30
:1075600084D9ABD93EEF3CF00E0E45DA99D9280EFE
:10757000E66EF70EE66E000EE66E12007AD961DA5C
:10758000CAD177D956DAC7D1BD0EE66EF70EE66ED0
:10759000000EE7DA6CD23EDAD89001501200FD0EF0
:1075A000DBCFE9FFFE0EDBCFEAFF1200FAD9020EB5
:1075B000E15C1200020EE66EE66AF5C900F0F6C95B
:1075C00001F0026A036AF5C9E6FFF6C9E6FF0ED2CA
:1075D000100EE66EE66AD80EE66E040EE66E120037
:1075E00000500324F36E01500420F46E0250052075
:1075F000F86EF4CFF7FFF3CFF6FF0800F550E66E14
:107600001200B5DAEBC900F0016A026A036AEBC93D
:10761000E6FF01C0E6FFEAD16CDABFD930EF3CF0FB
:10762000020EDBCF02F0030EDBCF03F0FD0EDB50CA
:10763000025C006EFE0EDB500358016EFC0E120061
:10764000060EDBCF00F0070EDBCF01F0D890015023
:107650001200FC0EDBCFE9FFFD0EDBCFEAFF1200CC
:107660004DEC3FF0E552E55205011200020EDBCF72
:10767000E9FFDB2A030EDBCFEAFF1200D9CFE9FFD7
:10768000DACFEAFF1200006E016AD950030FF2D977
:107690000050EE260150ED221200E1D9060EDB6A01
:1076A000070EDB6A120025DAE2D1AA0EE66E610E41
:1076B000E66E010E1200FF6FFEEF3EF00E0EF66E4C
:1076C000000EF76E000EF86E0800F550E66EE66AE2
:1076D0001200D950FD0FE96EFF0EDA20EA6E12009B
:1076E000FFECABF0046E0A0EE15E04501200020ED5
:1076F000A6CADBFF030EA7CADBFF1200A6CAE6FF7D
:10770000A7CAE6FF12002DDA1FEF76F0DBCFE6FF07
:10771000CDEF3CF0D1C9E6FFD2C9E6FFD3C9E6FF01
:10772000D4C9E6FF1200DECFE9FFDDCFEAFFE50EA8
:10773000E926060EEA221200BD0EFD6FF70EFE6F5F
:10774000000E1200000E005C040E01581200650EBF
:10775000E66E0A0EE66E12000901A051E66EE66AB8
:107760001200D89000360136E8041200F36E080EBD
:10777000F3CFDBFF1200E66E06EC9FF000EF3DF06A
:10778000E6EC9EF03DD9000912002EEC9EF0C9D91E
:10779000000912003FD90001800E01141200EFD839
:1077A000EF6A1200D950020F65D9EE50ED101200A9
:1077B00021EC99F0006E060EE15E00501200EECF53
:1077C00000F0EFCF01F0DF5000181200DF50EA6A3E
:1077D000C30FE96E090EEA221200BAEC74F0026ED1
:1077E000070EE15E02501200FB0EDBCFE6FFFC0E3F
:1077F000DBCFE6FF1200DFCFE9FFDF2A010EDBCF90
:10780000EAFF1200DBCFE6FF7EEC92F0E552E55294
:107810001200DECF02F0DDCF03F0D890035012004B
:107820007C0EE66E0A0EE66E1200E750E926000EA8
:10783000EA221200020EDB2A030E1200A00EE66EF0
:10784000F70EE66E000E1200DECFE6FFDDCFE6FF9C
:107850001200FD0EDBCFE6FFFE0EDBCFE6FF1200CF
:10786000F3CFDEFFF4CFDDFF120070D9DBCFE6FFF0
:107870001200000EE66E060EE66E1200020EF3CF48
:10788000DBFF030EF4CFDBFF1200C2EC74F091EFCC
:107890003DF0040EF3CFDBFF050EF4CFDBFF12004B
:1078A000F3CF00F0F4CF01F0F3CFE6FFF4CFE6FF23
:1078B0001200E66EE66AB1EF39F08CEC74F029D173
:1078C000080EDBCFE6FF090EDBCFE6FF0A0EDBCFAB
:1078D000E6FFD1EF39F093DD020EE1261200F86EDB
:1078E0000800F550E66EE66A2A0EE66EF70EE66EC2
:1078F000000E1200C2EC74F0026E070EE15E025040
:107900001200E66E62EC72F0E552120000C0E6FF73
:1079100001C0E6FF1200E66E64ECA6F0006E080EF1
:10792000E15E00501200040EDBCFE6FF050EDBCF58
:10793000E6FF1200FD0EF3CFDBFFFE0EF4CFDBFF00
:107940001200E66EE66AB4EF39F0DFD8000EE66E9C
:10795000060E5EDDDF2A010E12009CDD28C000F05D
:1079600029C001F028C0E6FF29C0E6FFE4EF39F0A6
:10797000C8EC75F0046E0B0EE15E04501200020EAE
:10798000DBCFE9FF030EDBCFEAFF1200FD0EDBCFFA
:1079900000F0FE0EDBCF01F01200BAEC74F091EFB4
:1079A0003DF03FEC2EF02FEF2EF0EF6AA7DE7EECDD
:1079B00092F09CDDCAEF3BF03FEC2EF04ADEDECFCA
:1079C000EEFFDDCFEDFF1200DBCFE6FFE66A250E0E
:1079D000E66EF70EE66E000E1200EECFE6FFEECF7B
:1079E000E6FFEECFE6FFEFCFE6FF120002C0E6FFB4
:1079F00003C0E6FF1200E66E51ECA8F0E55212005B
:107A0000E552E552E552E552120040EC9FF0E55296
:107A1000E5521200DECF00F0DDCF01F01200D1DC24
:107A20002C081200A90EFD6FF70EFE6F000E5BEF23
:107A30003BF0000EE66E020EE66EFA0EE66E040EE7
:107A40001200000EE66E010EE66EF80EE66E040EF3
:107A50001200010EE76EA3DDE8DEEF501200E66EC5
:107A6000BBECA5F0006E080EE15E00501200B6EC13
:107A70009EF04FD0E96EDACFEAFF1200DDEC99F00C
:107A8000E552E55276EF3AF0BADC030EE126120039
:107A9000B6DC040EE12612009EDC020EE15C120050
:107AA00067DC3FEF2EF0CADEB4EF3DF0D9C9E6FF48
:107AB000DAC9E6FF56DCDBC9E6FFDCC9E6FF51DCCC
:107AC0000901E051F6DEE3C900F0016A1200E66E3A
:107AD000E66AB4DED5EF39F0B1DEE66E35EF3CF0A4
:107AE000006E090EE15E005030EF3CF0F4DE62EF14
:107AF0003AF0E66E39EF3CF0E66E000EE66E030EED
:107B0000E66EFC0EE66E040E12000601006BB7EF87
:107B10003DF0006E050EE15E005012004FDC30EFCC
:107B20003CF0006E070EE15E0050120040EC9FF04A
:107B3000DDDC24EF3CF0EADE47DC3EEF3CF0DEDC4F
:107B4000D9DE7AEF3AF061DF50EF3CF0020EDBCF86
:107B5000E6FF030E120099DE30EF3CF02FDC49EF18
:107B60003CF0E66E29EF3CF0E66E24EF3CF0010EAF
:067B7000E66EE66A120059
:0A7B7600D8CFE4FFE0CFE4FFE46E97
:107B8000DACFE4FFE2CFDAFFE9CFE4FFEACFE4FFA8
:107B9000F6CFE4FFF7CFE4FFF8CFE4FFF5CFE4FF43
:107BA000F3CFE4FFF4CFE4FFFACFE4FFFBCFE4FF31
:107BB00000EE20F0140EE80403E3EECFE4FFFBD761
:107BC00000EE00F0200EE80403E3EECFE4FFFBD765
:107BD000E652C8ECAAF0F1ECACF0E55200EE1FF072
:107BE000200EE80403E3E5CFEDFFFBD700EE33F012
:107BF000140EE80403E3E5CFEDFFFBD7E5CFFBFF71
:107C0000E5CFFAFFE5CFF4FFE5CFF3FFE5CFF5FFD2
:107C1000E5CFF8FFE5CFF7FFE5CFF6FFE5CFEAFFC9
:107C2000E5CFE9FFE5CFDAFFE550E5CFE0FFE5CFAF
:107C3000D8FF10000801009B1200CEEC4AF0E6527B
:107C4000D9CFE6FFDACFE6FF9EECAAF0E552E55287
:107C5000000901E1D0D0FF0E0501EB5D01E094D0F9
:107C6000C85103E07F0EC85D08E10A0EDF5CE8E062
:107C70000D0EDF5C02E10A0EDF6E0D0EDF5CE0E050
:107C80002EEC4CF077EC4BF003E1015001E1EA07F8
:107C90003A0EDF5C1EE1060EEA5D1BE39DEC4BF045
:107CA00018E1490E015D15E1500E025D12E1440E2E
:107CB000035D0FE10501EA05ADEC4AF0EF6A050E40
:107CC000E66E070EE66E4CEC4BF0FD0EEB6FEA6BCA
:107CD000B7D70A0EDF5CB4E10501EA07EA51ADEC63
:107CE0004AF0EF6A040EEA5D48E39DEC4BF045E193
:107CF000430E015D42E14D0E025D3FE1540E035D16
:107D00003CE1070EDF6EDF50DF2AADEC4AF0EF50AA
:107D1000220804E00501EA51DF5CF5E3DF04ADEC85
:107D20004AF0EF6A0501D66B140EE66EE66A070E9E
:107D3000E66E070EE66ED60EE66E050E20EC4BF0F4
:107D40000501E96BEAC5DFFFDF50DF06ADEC4AF065
:107D5000EF502C0803E0DF500008F6E3DF50016A23
:107D6000000F006E070E0122020E7DEC4BF04CEC72
:107D70004BF0EA6BFE0EEB6F63D7050107EC4BF09F
:107D80000701006B050135D0FE0EEB5D1CE10D0E09
:107D9000DF5C03E00A0EDF5C07E1EA51EA2BADECA1
:107DA0004AF0200EEF6E02D02EEC4CF077EC4BF048
:107DB00003E1015001E1EA07EC07EC5101E040D793
:107DC00092EC4CF016D00D0EDF5C08E02EEC4CF07F
:107DD00077EC4BF003E1015001E1EA07EC070A0EF2
:107DE000DF5C03E1EA0792EC4CF0EC5101E028D7AC
:107DF000EA6BEB6925D7E552D3EF4AF097EC4CF0EC
:107E000038E1DF6AA4EC4AF00A080BE10D0EDF5CF2
:107E100008E0080100B1FDD70D0ED7EC4AF00FE1E4
:107E2000FBD70D0EDF5C0BE1A4EC4AF00A0807E07B
:107E3000080100B1FDD70A0ED7EC4AF0FCE0A4EC33
:107E40004AF028E0080100B1FDD7A4EC4AF0D7ECD5
:107E50004AF0FBE00501FDC5F6FFFD2BFEC5F7FF6F
:107E6000000EFE23FFC5F8FFFF230800F550DF6E6C
:107E7000C9D7A4EC4AF00EE0080100B1FDD7A4EC8C
:107E80004AF0D7EC4AF0FBE00501FD2B000EFE2383
:107E9000FF23EFD7E552D3EF4AF097EC4CF035E1F2
:107EA000DF6AC6EC4AF00A080BE10D0EDF5C08E061
:107EB000080100B1FDD70D0ED7EC4AF00FE1FBD75A
:107EC0000D0EDF5C0BE1C6EC4AF00A0807E0080182
:107ED00000B1FDD70A0ED7EC4AF0FCE0C6EC4AF040
:107EE00025E0080100B1FDD7C6EC4AF0D7EC4AF016
:107EF000FBE0FD0EDBCFE9FFDB2AFE0EDBCFEAFF66
:107F000001E3DB2AEFCFDFFFCCD7C6EC4AF00EE06F
:107F1000080100B1FDD7C6EC4AF0D7EC4AF0FBE00F
:107F2000FD0EDB2AFE0EF1E3DB2AEFD7E552D3EF9D
:107F30004AF0CEEC4AF0080100B1FDD7FE0EDBCFCF
:107F4000E6FF77ECAAF0E5520009F8E0D3EF4AF03B
:107F5000CEEC4AF0E150FD0FE96EFF0EDA20EA6E3A
:107F6000EE50ED1029E0A5EC4BF00501F75100189B
:107F700002E1F85101181CE0080E0601F31518E1A2
:107F8000FD0EDBCFF1F5FE0EDBCFF2F5F90EDBCF08
:107F9000F3F5FA0EDBCFF4F5FB0EDBCFF5F5FC0EB7
:107FA000DBCFF6F5FD0EDBCFF7F5FE0EDBCFF8F5F8
:107FB00005013C0EF96F05D085EC4BF0F76BF86BC3
:107FC000F96BD3EF4AF0CEEC4AF0040EE126030E33
:107FD0000DEC4BF0960EE66EF40EE66E000EEEEC37
:107FE0004AF00AE0A5EC4BF000C001F0006A005036
:107FF0000501FA130150FB13930EE66EF40EE66EC4
:10800000000EEEEC4AF00BE0FD0EDBCF28F0FE0E8A
:10801000DBCF29F028500501FA132950FB13040E79
:10802000E15C02E2E16AE552E16ED3EF4AF0CEECA8
:108030004AF0060EE12617EC4CF0E66EFD0EDBCFA3
:10804000E6FFFE0EDBCFE6FF7AEC4AF069E017ECC4
:108050004CF09DEC4CF064E0C5EC4CF061E0C5ECFC
:108060004CF05EE0ACEC4BF0EF504F0859E1010EE4
:10807000E76EACEC4BF0E750E926000EEA22EF5039
:108080002D084EE18F0EE66EF40EE66E000EE66EE3
:10809000020EE76EDBCF00F0030EDBCF01F0E750FE
:1080A0007DEC4BF00AEC4CF01DEC4CF039E08F0EFF
:1080B000E66EF40EE66E000EB3EC4AF0E4EC4AF025
:1080C000F350C9EC4CF0040EF3CFDBFF050EF4CFF8
:1080D000DBFF28EC4BF00DE1040EDBCFE9FF050ED2
:1080E000DBCFEAFFEF501CE08E0EE66EF40EE66E7C
:1080F00012D0B3EC4BF0040EDBCFE6FF050EDBCF66
:10810000E6FFE6EC9EF0E552E552E552E552000945
:1081100007E0B3EC4BF0E4EC4AF0F350BAEC4BF070
:10812000060EE15C02E2E16AE552E16ED3EF4AF04D
:10813000CEEC4AF0020EE126FE0EDBCFC8F50501BB
:10814000C851240A01E15FD1070A01E152D1010AB5
:1081500001E149D1030A01E115D1010A01E1FCD095
:10816000600A01E1D7D0030A01E1B9D0010A01E1B7
:108170008FD0030A01E178D0530A69E0030A5CE07A
:10818000010A4FE0160A47E0030A3CE0010A33E027
:10819000070A25E0010A21E0030A11E07E0A0CE04B
:1081A0007F0A01E03CD1A9EC4CF000EC4BF005015A
:1081B000010ECD6F0A0E24D105EC80F030D10A0EED
:1081C00045EC4CF00501030ECD6F140ECE6FCF6B56
:1081D0000901E86B0BEC2EF022D1CD6B20D100EC25
:1081E0004BF076EC72F00501020ECD6F30EC4BF0E7
:1081F0000501CC6B14D1050ECD6F0A0E30EC4BF09F
:108200000A0E9ED0060ECD6F020ECE6FCF6BC96BDD
:1082100076EC72F004D1E66A44EC4AF042EC72F07B
:10822000FED0090E45EC4CF056EC4BF0B00EFD6F55
:10823000600EFE6F010ED4D0080E45EC4CF056ECEB
:108240004BF0F70EFD6F600EFE6F010EC9D0070EEA
:1082500045EC4CF00501030ECD6F230ECE6FCF6BB6
:10826000C96BC1EC4BF0BCD0050EE66EB8EC4CF01F
:108270005FEC4BF006E2070EEAEC4AF00501400E17
:1082800005D0080EEAEC4AF00501020ECD6F14D0BD
:10829000050E10EC4BF0750EFD6FF40EFE6F000E28
:1082A00037EC4BF0090EEAEC4AF05FEC4BF002E2DF
:1082B000430E01D0020ECD6FCAC5CEF5CBC5CFF5AA
:1082C0000A0ED880CE57000ECF570F0ECF03F3CF34
:1082D000CFF5CE03F3CFCEF5F450CF27A0D0050EC7
:1082E00045EC4CF014EC4BF00501020ECD6F3C0E4A
:1082F000CE6FCF6B060EC96F0901E86B0FEC2EF045
:10830000B1EC4CF0C8EC4BF037EC4BF00501400EF3
:10831000C86F85D0050E45EC4CF014EC4BF00DEC1D
:108320004BF047EC4BF0EF5014E0FCECB1F00009DF
:1083300010E00501020ECD6F3C0E30EC4BF0020E4A
:10834000C1EC4AF00501820EFD6FF40EFE6F000EC7
:1083500047D00501200EC86F020E45EC4CF00A0113
:10836000646B0501CD6BC96B0901E60507E0050EDD
:10837000E65D04E0780E0501D26F02D00501D26BF4
:10838000D36B4DD0060E45EC4CF0B1EC4CF0050132
:10839000030ECD6FF00ECE6FCF6B0FEC2EF00D0EE7
:1083A0000DEC4BF047EC4BF0EF5007E105015F0E91
:1083B000FD6F610EFE6F010E13D005014F0EFD6FB4
:1083C000F40EFE6F000E37EC4BF03BEC4CF065DD2D
:1083D000E552E5520501450EFD6FF40EFE6F000EED
:1083E00037EC4BF01CD00A0ECE6FCF6B400ECD6F2A
:1083F00016D0060E45EC4CF00501240ECD6F1E0E76
:10840000CE6FCF6B0CD0CC51CC2B006E140E005C19
:1084100002E2020E01D0030EE66E8ADEE552020E83
:10842000E15C02E2E16AE552E16ED3EF4AF0CEECA4
:108430004AF0110EE126FE0E0501EB5D1AE109017D
:10844000E60507E0050EE65D04E014EC4BF0B4EC45
:108450004CF00601F6BF03D006010A0EF76F43EC9D
:108460004BF0D60EE66E050EE66ECFEC4BF0A6EFA7
:1084700046F0FF0EEB5D10E00601F6BF03D00601EB
:10848000140EF76F12EC4CF0E2EC33F0E552E552CB
:10849000E1EC4BF0A6EF46F00601F6BF03D0060173
:1084A0001E0EF76F0501C8517F0A02E19FEF46F0EB
:1084B0005F0A01E117D2600A01E15ED1630A01E1BE
:1084C00041D1020A01E1F7D0330A01E1CAD0030A1F
:1084D00068E0010A2CE0110A17E0010A02E0A6EFA9
:1084E00046F0050EEA5D02E2A6EF46F0F0EC4BF036
:1084F0003F0EE66EF40EE66E000E37EC4AF002E038
:10850000A6EF46F07F0EEAD1020EEA5D02E2A6EF88
:1085100046F0A1EC4BF002E0A6EF46F04B0E015DF9
:1085200002E0A6EF46F0B4EC4CF0100ED7D1040EEA
:10853000EA5D23E39DEC4BF020E1430E015D1DE17C
:10854000530E025D1AE14D0E035D17E112EC4CF083
:1085500040EC9FF0E552E552F3CFE9FFF4CFEAFF9C
:10856000E906000EEA5A000EE926070EEA22EF504D
:10857000310801E1EBD3030E5AD00501C95101E0E6
:10858000E5D3020EEA5D01E2E1D3A1EC4BF001E09C
:10859000DDD34B0E015D01E0D9D3B4EC4CF0110EEC
:1085A0009DD1100EEA5D14E3380E0701005D10E165
:1085B000390E015D0DE1180EE66EE66A12EC4CF024
:1085C000CD0EE66E060E20EC4BF00601E46BBED33A
:1085D000080E0501EA5D16E39DEC4BF013E1430E36
:1085E000015D10E1500E025D0DE1420E035D0AE1F6
:1085F000460E045D07E13A0E055D04E112EC4CF015
:1086000016DD95D1080E0501EA5D17E39DEC4BF0F0
:1086100014E1430E015D11E1500E025D0EE1490EC1
:10862000035D0BE1520E075D01E190D3040EEAEC0D
:108630004AF00501010EC96F89D30501C95101E056
:1086400085D3020EEA5D01E281D3A1EC4BF001E09B
:108650007DD34B0E015D01E079D3B4EC4CF0120EEA
:108660003DD1060EEA5D16E39DEC4BF013E1490E99
:10867000015D10E1500E025D0DE1520E035D0AE155
:10868000390E065D07E00501960EFD6F610EFE6F67
:10869000010E6DD1020E0501EA5D01E257D3A1EC96
:1086A0004BF001E053D34B0E015D01E04FD3B4EC2E
:1086B0004CF0210E13D1020EEA5D0BE3A1EC4BF05E
:1086C00008E14B0E015D05E1E1EC4BF0CC6B220EB5
:1086D00005D1050E0501EA5D07E3450E0701005DC2
:1086E00003E1520E015D05E068EC4CF037EC4AF016
:1086F00002E1230EF3D0F4EC4BF02D0EE66EF40EF7
:10870000E66E000E37EC4AF001E020D317EC4CF097
:10871000E66E12EC4CF07AEC4AF001E117D317EC5C
:108720004CF09DEC4CF001E111D3080EE66EE66AC8
:108730003BEC4CF0EC0EE66E090E20EC4BF0090120
:10874000F46B04D348EC4CF001E000D32C0E07018D
:10875000085D03E1070E091502D0070E0715090190
:10876000E66FE80404E0050EE65D01E0EFD2E1EC1F
:108770004BF0CC6B400EB2D0020EEA5D16E3450E14
:108780000701005D12E1520E015D0FE1020E0501CD
:10879000C95D03E0030EC95D02E1410E9FD0050EE5
:1087A000C95D01E0D3D2030E99D0020E0501EA5D46
:1087B00006E3A1EC4BF003E14B0E015D0BE0530E21
:1087C0000701005D03E1480E015D04E0050E0501AF
:1087D000C95D6DE10501EA6B1E0ECE6FCF6B09011D
:1087E000E76BB1EC4CF00501C92BC951080A5DE0FB
:1087F0000F0A48E0010A43E0030A3AE0010A31E0C7
:10880000070A26E0010A0DE0030A01E09FD20501F4
:10881000130EFD6FF40EFE6F000E37EC4BF0050EDD
:108820000FD00501060EFD6FF40EFE6F000E37EC43
:108830004BF0050E50EC4CF0060E50EC4CF0070ED1
:108840006BEC4AF0100EFD6FF40EFE6F000E8FD031
:10885000040E10EC4BF0F80EFD6FF30EFE6F000EE1
:1088600086D00501EA0EFD6FF30EFE6F000E7FD07D
:108870000501E00EFD6FF30EFE6F000E78D0C8EC20
:108880004BF075D0030E10EC4BF0CC0EFD6FF30ED9
:10889000FE6F000E37EC4BF0040E6BEC4AF0C20E8C
:1088A000FD6FF30EFE6F000E62D0200E17D0070E84
:1088B000EA5D0DE3080EE66EE66AB90EE66EF30EAB
:1088C000E66E000E37EC4AF002E1020E07D071ECC2
:1088D0004CF037EC4AF001E039D2020EE66E98EC2B
:1088E00040F026D048EC4CF025E12C0E0701085D45
:1088F00003E1070E091502D0070E07150901E66FFF
:10890000E80403E0050EE65D05E10501D26BD36BDB
:10891000E66A0AD00501D251D31101E017D2780ED0
:10892000D26FD36B010EE66EE66ABEECACF0E55298
:10893000E5520CD2F0EC4BF0A70EE66EF30EE66EAD
:10894000000E37EC4AF016E10901E60507E0050ED6
:10895000E65D04E014EC4BF0B4EC4CF0010EC1EC1D
:108960004AF00501770EFD6F610EFE6F010E37ECC8
:108970004BF0ECD1020EE66EE66AA40EE66EF30E44
:10898000E66E000E37EC4AF001E0BCD0E6EC4BF0AE
:1089900001E3B8D034EC4CF0020EE66E070EFDECAD
:1089A0004AF03EEC4AF00EE068EC4BF0020E26C0B6
:1089B000DBFF030E27C0DBFF040E28C0DBFF050E24
:1089C00029C0DBFF3EEC4AF005E047EC4BF00A0E15
:1089D000EFCFDBFF3EEC4AF00EE068EC4BF0060E0A
:1089E00026C0DBFF070E27C0DBFF080E28C0DBFF19
:1089F000090E29C0DBFF3EEC4AF005E047EC4BF0E6
:108A00000B0EEFCFDBFF3EEC4AF005E047EC4BF0FE
:108A10000C0EEFCFDBFF3EEC4AF03EEC4AF03EECB2
:108A20004AF008E0E4EC4AF00D0EF3CFDBFF0E0E47
:108A3000F4CFDBFF1DEC4CF001E188D10C0EDB50D4
:108A4000010B0901E06FE8505AE00A0EDB505308B1
:108A500018E1020EDBCF00F0030EDBCF01F0040EB5
:108A6000DBCF02F0050ED3EC4BF0020E00C0DBFFB3
:108A7000030E01C0DBFF040E02C0DBFF050E03C0C6
:108A8000DBFF0B0EDB50570818E1060EDBCF00F0C2
:108A9000070EDBCF01F0080EDBCF02F0090ED3EC9E
:108AA0004BF0060E00C0DBFF070E01C0DBFF080E17
:108AB00002C0DBFF090E03C0DBFF020EDBCFD1F9E2
:108AC000030EDBCFD2F9040EDBCFD3F9050EDBCFDB
:108AD000D4F9060EDBCFD5F9070EDBCFD6F9080E99
:108AE000DBCFD7F9090EDBCFD8F90D0EDBCFDBF9E1
:108AF0000E0EDBCFDCF90901780EE36F27D10901F7
:108B0000E36B24D1030EE66EE66A9E0EE66EF30E6C
:108B1000E66E000E37EC4AF022E1E6EC4BF01FE285
:108B200034EC4CF0030EE66E070EFDEC4AF008E064
:108B3000E4EC4AF00F0EF3CFDBFF100EF4CFDBFFB7
:108B40001DEC4CF001E102D10901E05101E1FED040
:108B50000F0EDBCFD9F9100EDBCFDAF9F7D00A0E02
:108B6000E66EE66A930EE66EF30EE66E000E37ECE6
:108B70004AF004E10901E75125E119D0070EE66E3C
:108B8000E66A8B0EE66EF30EE66E000E37EC4AF0E8
:108B900042E1110EE66EE66A790EE66EF30EE66EBF
:108BA000000E37EC4AF012E10901E7510BE1010E2A
:108BB000E66EE66E00EC4CF012EC2EF0B3EC2EF00C
:108BC0002FEC2EF00901010EE76FC0D0150EE66EF6
:108BD000E66A630EE66EF30EE66E000E37EC4AF0C0
:108BE00001E1B4D0110EE66EE66A510EE66EF30EA8
:108BF000E66E000E37EC4AF058E00901E76B020E12
:108C0000E66EB8EC4CF00901E6056CE0050EE65D99
:108C100001E09CD067D0F0EC4BF04B0EE66EF30E0B
:108C2000E66E000E37EC4AF012E12C0E0701085DEB
:108C300009E1070E0715006E070E06150A0DF35021
:108C4000002402D0070E06150901E96F7FD0070E38
:108C5000E66EE66A430EE66EF30EE66E000E37EC45
:108C60004AF058E00B0EE66EE66A370EE66EF30E3B
:108C7000E66E000E37EC4AF003E10A01646B66D041
:108C8000F4EC4BF0300EE66EF30EE66E000E37ECB1
:108C90004AF00BE00C0EE66EE66A230EE66EF30E6B
:108CA000E66E000EDDEC4AF004E10FEC2EF0420E11
:108CB00034D0090EE66EE66A190EE66EF30EE66E25
:108CC000000ED5DB0FE068EC4CF0DDEC4AF00AE07A
:108CD00071EC4CF0BCEC4CF0026E070EE15E025001
:108CE000000904E10FEC2EF0410E17D0040EE66EE1
:108CF000E66A150EE66EF30EE66E000EB8DB0AE0CD
:108D0000F4EC4BF00E0EE66EF30EE66E000EDDECAC
:108D10004AF007E10FEC2EF0010EE66E98EC40F001
:108D200014D0F4EC4BF0070EE66EF30EE66E000E78
:108D30009EDB0CE143EC4BF006EC37F004D043EC47
:108D40004BF086EC83F0E552E552E552110EE15C02
:108D500002E2E16AE552E16ED3EF4AF0CEEC4AF06E
:108D6000080EE1260501F951000805E2F907F9515D
:108D700002E1F76BF86BC8517F0A01E187D15F0A06
:108D800043E0220A3FE0230A32E0330A2AE0030AE2
:108D90001EE0010A12E0110A01E07AD1050ECE5D53
:108DA000000ECF5903E2020EEAEC4AF00501730E01
:108DB000FD6F610EFE6F010E67D1BADB01E068D175
:108DC0000501B00EFD6F600EFE6F010E5DD1B0DBD0
:108DD00001E05ED10501F70EFD6F600EFE6F010E22
:108DE00053D1A6DB01E054D1C1EC4BF04DD1140EB0
:108DF000CE5D000ECF5901E34BD1F4EC4BF0BEEC4D
:108E0000ACF00BD1E66A23D0FF0EEB5D09E0ED0577
:108E100003E1ED6BEB6910D0ED51010801E2ED07C4
:108E2000000ED880D255000ED35508E2D207000EAE
:108E3000D35BD251D31102E1210E08D0F8EC4BF0F4
:108E400009E2642B64513C0805E2400EE66E98ECA2
:108E500040F0E4D00901E60504E0050EE65D01E01E
:108E600007D10A01A451A51106E00A01630503E137
:108E70000A0164514AE0DAEC4BF020E20A01630592
:108E80001DE10A0164511AE18FEC4CF0DAEC4BF071
:108E900012E2F3C5E6FFF4C5E6FFF5C5E6FFF6C549
:108EA000E6FFF1C5E6FFF2C5E6FF88EC39F0006E9B
:108EB000060EE15E005085EC4BF0EAD0FF0E050196
:108EC00005EC4CF063E20A01630560E10A016451BC
:108ED0005DE18FEC4CF0200E050105EC4CF004E256
:108EE000FA9B2BEC39F0D4D0040E05EC4CF010E2D8
:108EF000FA95FC5101E0CCD0060E0A01A46FA56BD7
:108F0000A6CAE9FFA7CAEAFFEF6A86EC36F0C0D02E
:108F1000080E05EC4CF006E2FA97EEA3B9D05EEC31
:108F200039F0B6D0100E05EC4CF004E2FA9939ECA9
:108F300039F0AED0020E05EC4CF00AE2FA938FEC59
:108F40004CF0020EE66E79EC2FF0E55202081BD0D1
:108F5000010E05EC4CF01AE2FA910901E851000803
:108F600015E2020EDF6E8FEC4CF0DFCFE6FF7CECFB
:108F700031F040EC4CF079EC2FF0E552DF6E020E50
:108F8000DF5C01E185D02FEC2EF082D0000E0501D0
:108F9000FA15006EFF0E24EC4CF050E28FEC4CF012
:108FA0006FDB000E0501FA15006E200E24EC4CF06C
:108FB00005E2FB9BB0DA91EC5AF02FD0FCEC4BF0C1
:108FC000040E24EC4CF012E2FB95FC5161E1020E20
:108FD000E66EF30EE66E000EA0DB27EC9FF083EC4E
:108FE0004CF0040E9ADB97DADADB52D0FCEC4BF053
:108FF000080E24EC4CF007E2FB97EEA349D08BDA85
:10900000DAEC5AF00AD0FCEC4BF0100E24EC4CF0E9
:1090100007E2FB9980DAA6EC5AF0E552E55238D027
:10902000EBDB020E24EC4CF002E2FB9307D0E4DB16
:10903000010E24EC4CF002E2FB912AD009019F5171
:10904000000816E20601ED51000812E20A0164511F
:109050000FE10901E85100080BE2B1EC4CF0020EFF
:10906000E66E70EC30F0E552020802E02FEC2EF0D4
:10907000B2DB02E3EDDB0CE1A9DB0AE20501D20E73
:10908000FD6F600EFE6F010EF2DA02D025EC80F06B
:10909000080EE15C02E2E16AE552E16E84D205016C
:1090A000C851200A01E01200A3DB02E23AEF4BF0C4
:1090B000CFDB14E0B1EC4CF005017C0EFD6F610ECE
:1090C000FE6F010EFF6FFEEC3EF0080141510008FB
:1090D00003E2010E56DAF9D7020E53DA12005EDA15
:1090E000030EE1260901EA511AE101ECB2F026C0B3
:1090F00000F027C001F028C002F029C003F0EEDA2A
:1091000001C028F002C029F003C02AF047EC8CF01F
:10911000BCEC8DF029C0EAF90901EB6B3BD0EA51B8
:10912000026E036AEAC9E6FF03C0E6FF01ECB2F093
:10913000E552E7CF03F0E552E7CF02F026C004F096
:1091400027C005F028C006F029C007F0C7DA05C01F
:1091500028F006C029F007C02AF047EC8CF0E3ECB9
:109160008DF002502824006E03502920016E010E5C
:109170000026000E0122020E2D6E2E6A00C028F07D
:1091800001C029F0CEEC8CF028C000F029C001F01D
:1091900028C0EAF909019DB907D00F0E0901EB5D5E
:1091A00009E2090199AF03D00901EB6B0ED0090167
:1091B000EB2B0BD00F0EEB5D08E109019951800BF1
:1091C00004E1EAC9EBF90701CA930901EB510F0861
:1091D00025E209019951800B21E1020E0701CA1510
:1091E0000AE10F0E0901EB5D0901D880EA5503E39E
:1091F0000701CA830CD0020E0701CA150FE00D0E3D
:109200000901EB5D0901EA5D09E30701CA93080E54
:10921000E66EE66AE3EC3FF0E552E5520501C8511F
:10922000200A1BE1E5DA02E225DA17D00901E70599
:1092300010E10901E85100080CE271DB5BDB01E0A1
:109240005EDB0C0E24D901E089DB2BD902E02FEC88
:109250002EF0010E0501C919C96F030EE15C02E28F
:10926000E16AE552E16E9FD112006DDB0AE0020E69
:10927000945D07E00F0E945D04E0ADDA02E3000EAA
:1092800001D0010E52DA49E1050E0901A05D29E283
:10929000800E0901991525E10501F0510FE1090141
:1092A000E7050DE10A0164510AE10501EEA502D0CE
:1092B00047EC39F00501480EF06F01D0F0070501C9
:1092C000EF510DE1DDD90501EEA505D024D9BBECA8
:1092D0005AF0E552E5520501480EEF6F06D0EF0750
:1092E00004D00501060EEF6FF06F0901E70515E1E7
:1092F0000901E85112E1030EDB500FE079DA02E2D6
:10930000B9D90BD0F7DA01E0FADA0C0EC0D801E0D7
:1093100025DBC7D802E02FEC2EF0040EE15C02E260
:10932000E16AE552E16E3FD10EDB0AE0020E945D88
:1093300007E00F0E945D04E04EDA02E3000E01D068
:10934000010EF3D918E10901E70515E10901E8511A
:1093500012E1030EDB500FE14BDA02E28BD90BD0A6
:10936000C9DA01E0CCDA0C0E92D801E0F7DA99D82C
:1093700002E02FEC2EF0040EE15C02E2E16AE5521D
:10938000E16E11D10501FC51000801E2FC07D02B70
:10939000000ED123CD51000810E2CEC500F0CFC59C
:1093A00001F0CE07000ECF5B0050011006E1CDC5E5
:1093B000E6FF98EC40F0E55201D0D0DC3CD91E0E1F
:1093C0002D6E2E6A83D801E16ADE42DA01E187DE82
:1093D00032D92C0E2D6E010E2E6E78D801E144DFAD
:1093E0002AD9580E2D6E020E2E6E70D801E13DDF87
:1093F00022D9100E2D6E0E0E2E6E68D806E194DF67
:10940000100E0501D05F0E0ED15B0501D407000ED2
:10941000D55BD451D5111EE1E66A36D8050199DA3B
:109420000601EF2BEF51E66EE66AE66AE66AE66A47
:10943000000EE66E060EE66EC2EC74F0006E070ECD
:10944000E15E0050000EE66E060EE66E1A0E92D930
:1094500042EC72F012001200800E946E5BECAAF0E7
:109460000901E66BE66A98EC40F0E552120084DAF6
:10947000006E070EE15E005000091200F5D9000EE3
:10948000E66EE66AC7D944D273DAB4EF4CF0E66E02
:109490000FDA010EDBCFE9FF020EDBCFEAFFEF5060
:1094A0001200DFCFE6FF79EC2FF0EAD970EC30F054
:1094B000E7D98FEC30F0E4D97CEC31F0E1D926EC3F
:1094C00032F0E552DF6E020EDF5C1200D0C528F0EC
:1094D000D1C529F0F4D15DDAF3CF00F0F4CF01F07B
:1094E000F3CFE6FFF4CFE6FF4DEC3FF0E552E55257
:1094F0000501120018ECAEF006DA42DA1DEF4CF06E
:10950000E66EDFCFE6FF60EC32F0E552E552E55261
:10951000E552DF6E1200010EDBCFE6FF020EDBCF5D
:10952000E6FF1200000ED8800054000E0154120015
:10953000CEC500F0CFC501F0030E2D6E2E6ACEC54C
:1095400028F0CFC529F0BBD1FDC5F6FFFEC5F7FF5A
:10955000FFC5F8FF0800F5501200EA6A000FE96E37
:10956000070EEA221200E66E000EE66EE66A18ECBE
:10957000AEF0C9D9020EF3CFDBFF030EF4CFDBFF51
:109580001200E66E62EC72F0E5521200FD0EDBCFC7
:10959000E9FFFE0EDBCFEAFFEF501200D9CFE6FF66
:1095A000E1CFD9FF1200E552E7CFD9FF1200E66EF6
:1095B00077ECAAF0E55200091200DED9016E070E21
:1095C000E15E01500009120056D97EEC92F0E5529E
:1095D000E5521200E66EE66A00EF4CF0E66E4BD9FB
:1095E000CCEC9FF0026E050EE15E0250F3CF00F06E
:1095F000F4CF01F0F350F4101200E66E0BD988D1CD
:10960000E668B6D9E668E66AFBD8E5EFACF0A1D922
:1096100017EC42F00501EA6B1200BBD9C0EF4CF029
:10962000E66EA6D9050112000501D26BD36B0901C4
:10963000050EE66F1200D0C500F0D1C501F0120092
:10964000E66E9EEC9FF0006E060EE15E005012008A
:10965000D950020FE96EDACFEAFFEE50ED1012009A
:10966000CE6FCF6BC96B0901E86B0FEF2EF0FF6F68
:10967000FEEF3EF0050E0501D05F000ED15B12003B
:10968000E66A58EF4CF0EAC5E6FF12EF4CF0DECF89
:10969000E9FFDDCFEAFF12007EEC92F0E552E552E1
:1096A000F3CFECF505013C0EED6F12000501030E42
:1096B000CD6F5F0ECE6FCF6BC96B05011200050138
:1096C000CA07000ECB5BD880CA55000ECB551200DE
:1096D000D2D87BEC73F0E552E55212002C6A2D6A69
:1096E000200E2E6E410E2F6E26C027F01200EA517A
:1096F000006E016AC80E001812000026000E01223A
:1097000000C0E6FF01C0E6FF12000501F16BF26B3D
:10971000F36BF46BF56BF66B1200E66ED950030F2A
:10972000E66E000EDA20E66E1200E76E030EE7CF5B
:10973000DBFF0501C851200A12002B0E0701005D56
:1097400012004F0E0701005D1200FD0EDBCF00F08E
:10975000FE0EDBCF01F01200020EDBCFE9FF030E9D
:10976000DBCFEAFF1200020EDBCFE6FF030EDBCFFA
:10977000E6FF1200E66E98ECA8F0E552E552E552DD
:1097800012000501120EFD6F610EFE6F010E120038
:1097900005015D0EFD6FF40EFE6F000E120076ECFB
:1097A00062F083EF4CF0DBCF03F0001E011E021EBF
:1097B000031E12000501000ED880F155000EF2556F
:1097C00012000A0E0501CA6FCB6B1200010E0501D3
:1097D000EE1500081200800E09019915000812000C
:1097E000050EE66EE66A1200060EE66EE66A1200E6
:1097F0000A01645100081200000EFA15006E1200F2
:10980000BEECACF0E552E5521200FA15006E016AAA
:1098100092EF4AF018ECAEF0026E050EE15E0250D7
:10982000C0EF4CF0000EE66E070EE66E1200910ED1
:10983000E66EF40EE66E000E1200D9CFE9FFDACF25
:10984000EAFFEE50ED101200FB15016E92EF4AF0A8
:10985000F2DE3C0E2D6E2E6A66EF4AF0EA51EA2BDC
:109860007CDEDFCFEFFF1200A20EE66EF30EE66E97
:10987000000EE66E1200DECFE6FFDDCFE6FF12003F
:10988000E552DF6EDFCFE6FF1200E66E44EF4AF0EE
:10989000A7DF270EE66EF40EE66E000E37EF4AF0F5
:1098A0001ADE020EFD6FF40EFE6F000E37EF4BF066
:1098B00051ECA8F0E552DE5263D8DD521200ABEC59
:1098C000B2F024C000F025C001F024502510120091
:1098D0000A0EE66EE66A340EE66EF40EE66E000ED2
:1098E00012000B0EE66EE66AAD0EE66EF30EE66E45
:1098F000000E1200020EDF6E0B0E47EF4AF00BDE79
:10990000010E80EF4AF0006E050EE15E005012007D
:10991000DECF00F0DDCF01F00050011012000A0E82
:10992000C1EF4AF0EA5119DEEF6A07EF4BF036DE7D
:10993000E6527F0E0501C85D1200E66E000EE66E6F
:10994000E66A7AEF4AF02ADE040EE1260901940560
:109950001200080ED46F070ED56F1200DCDD80EF09
:109960004AF0020EC1EF4AF0E66AE66A00EF4CF0F8
:10997000010EE66E00EF4CF0E66E54DF2EEF9EF027
:10998000F3CFDEFFF4CFDDFF120051DFECDD28EF77
:0C9990004BF0E66E51ECA8F0E55212001E
:04999C0088EC59F00A
:1099A000CEEC59F0EE6AEE6AEE6AEE6A01EC59F01E
:1099B000EE6AEE6AEE6AEE6A3DEC56F0010EEE6E6D
:1099C000230EEE6E450EEE6E670EEE6E3DEC56F01B
:1099D000040E7FEC57F0890EEE6EAB0EEE6ECD0EE0
:1099E000EE6EEF0EEE6E3DEC56F0080E7FEC57F08B
:1099F000FE0EEE6EDC0EEE6EBA0EEE6E980EEE6E93
:109A00003DEC56F00C0E7FEC57F0760EEE6E540ED9
:109A1000EE6E320EEE6E100EEE6EE552E7CFD9FF0F
:109A2000120088EC59F0080EE126030E046E01ECDA
:109A300059F0B3EC57F003E0D3EC57F0FDE13F0EE3
:109A400000160DEC58F042EC59F0F90EDBCF04F0A3
:109A5000FA0EDBCF05F0066A076A05AE02D006688B
:109A60000768030E1F0B07E0D8900436053606364C
:109A70000736E806F9E101EC59F00450EF26EECF85
:109A800000F00550EF22EECF01F00650EF22EECFAE
:109A900002F00750EF22EECF03F0F90EDBCF08F013
:109AA000FA0EDBCF09F00A6A0B6A09AE02D00A6827
:109AB0000B68030E1F0B03E0E4EC57F0FDE10850C8
:109AC000005C095001580A5002580B50035806E236
:109AD000CEEC59F0EE2AEE22EE22EE22EBEC57F01D
:109AE000026A036A01AE02D0026803681D0ED3EC5D
:109AF00057F0FDE1CEEC59F07BEC59F0400E046ECE
:109B0000056A066A076AD9CFE9FFB9EC57F0EE504B
:109B10000758060E00C0DBFF070E01C0DBFFEBECB1
:109B200057F0A5EC59F001500318E8AE02D0033409
:109B300004D00250005C035001586AE3060EDBCFEC
:109B4000E6FF070EDBCFE6FFA7EC57F084EC59F0F9
:109B5000E9CF02F0EACF03F0DB50E924006E010EFA
:109B6000DB50EA2003EC58F04DEC9EF0046E060E3C
:109B7000E15E045084EC59F09EEC57F03DEC56F059
:109B8000E9CF02F0EACF03F0C2EC57F0060EDBCFCC
:109B900028F0070EDBCF29F0040E28C0DBFF050EEE
:109BA00029C0DBFF3F0EE76E6BEC59F0E750002653
:109BB000000E012264EC59F001500318E8AE02D007
:109BC000033404D00250005C035001581EE2040E1E
:109BD000DBCF02F0050EDBCF03F0FB0EDB500224DF
:109BE000006EFC0EDB50032003EC58F03DEC56F009
:109BF000E9CF04F0EACF05F0C2EC57F0C1EC59F020
:109C0000400EEE26000EED22CDD7ACEC59F004D07C
:109C1000040EDB6A050EDB6A64EC59F0040EDB50BF
:109C2000025C006E050EDB50035803EC58F0DAECD2
:109C300057F0046EFC0EDB500720056E04C0E6FFF3
:109C4000E66E84EC59F0E9CF0AF0EACF0BF0DB5076
:109C5000E924086E010EDB50EA20096E08C0E6FF19
:109C6000E66E4DEC9EF00C6E060EE15E0C50080E9A
:109C7000E15C02E2E16AE552AEEF57F0F8EC57F032
:109C8000080ECDEC57F0100E7FEC57F09EEC57F01D
:109C9000D9CFE6FFDACFE6FFF2EC57F0030E046E01
:109CA000B3EC59F0100E7FEC57F0B3EC57F003E033
:109CB000D3EC57F0FDE13F0E00160DEC58F0F1EC3F
:109CC00058F0380EEE5C000EEE58000EEE58000E06
:109CD000EE580DE2380E046E056A066A076ACAEC91
:109CE00059F0B9EC57F0026EEE50075813D0780EC9
:109CF000086E096A0A6A0B6ACAEC59F012EC5AF04B
:109D0000085C006EEE500958016EEE500A58026E63
:109D1000EE500B58036E0EEC59F00C0EDBCFE6FF45
:109D20000D0EDBCFE6FF000EE66E0B0EE66EA7EC27
:109D300057F0FCEC57F0080EE66EE66AD9CFE6FF66
:109D4000DACFE6FFA7EC57F0FCEC57F0100ECDECA5
:109D500057F09EEC57F0FD0EDBCFE6FFFE0EDBCF9B
:109D6000E6FFF2EC57F0100EE15C02E2E16AE55228
:109D7000AEEF57F0F8EC57F03DEC56F0EECFDFFFCA
:109D8000010EEECFDBFF020EEECFDBFF030EEECFB8
:109D9000DBFF040EE3EC58F0040EEECFDBFF050E04
:109DA000EECFDBFF060EEECFDBFF070EEECFDBFFC5
:109DB000080EE3EC58F0080EEECFDBFF090EEECFF5
:109DC000DBFF0A0EEECFDBFF0B0EEECFDBFF0C0E40
:109DD000E3EC58F00C0EEECFDBFF0D0EEECFDBFF09
:109DE0000E0EEECFDBFF0F0EEECFDBFF400EE66E6A
:109DF000E66AE66AE66AA7EC57F0A80EE66E0A0E77
:109E0000E66EB3EC54F0006E080EE15E005057ECC5
:109E100058F09EEC56F0780E0026A40E01226A0E31
:109E20000222D70E8DEC59F003E0E3EC55F0FDE192
:109E3000B5EC55F0190ED2EC55F0FDE111EC58F0EF
:109E4000ABEC56F0560E0026B70E0122C70E0222CA
:109E5000E80EFFEC59F003E0E3EC55F0FDE1C5EC52
:109E600055F0140ED2EC55F0FDE12CEC58F0B8ECA6
:109E700056F0DB0E0026700E0122200E0222240E68
:109E8000D2EC59F003E0E3EC55F0FDE1A8EC55F01D
:109E90000F0ED2EC55F0FDE144EC58F0C5EC56F055
:109EA000EE0E0026CE0E0122BD0E0222C10E03ECE4
:109EB0005AF003E0E3EC55F0FDE1B8EC55F00A0E82
:109EC000D2EC55F0FDE107EC5AF0D2EC56F0AF0EB3
:109ED00000260F0E01227C0E0222F50E8DEC59F0A9
:109EE00003E0E3EC55F0FDE1B5EC55F0190ED2ECD2
:109EF00055F0FDE111EC58F0DFEC56F02A0E00268B
:109F0000C60E0122870E0222470EFFEC59F003E035
:109F1000E3EC55F0FDE1C5EC55F0140ED2EC55F034
:109F2000FDE12CEC58F0ECEC56F0130E0026460E3A
:109F30000122300E0222A80ED2EC59F003E0E3EC2D
:109F400055F0FDE1A8EC55F00F0ED2EC55F0FDE117
:109F500044EC58F0F9EC56F0002A950E0122460E1A
:109F60009FEC59F0160E1F0B03E0E3EC55F0FDE1FA
:109F7000B8EC55F00A0ED2EC55F0FDE107EC5AF0C2
:109F800006EC57F0D80E0026980E0122800E022211
:109F9000690E8DEC59F003E0E3EC55F0FDE1B5EC12
:109FA00055F0190ED2EC55F0FDE111EC58F013EC20
:109FB00057F0AF0E0026F70E0122440E02228B0E40
:109FC000FFEC59F003E0E3EC55F0FDE1C5EC55F092
:109FD000140ED2EC55F0FDE12CEC58F020EC57F0CB
:109FE000B10E00265B0E0122FF0E0222D2EC59F0C8
:109FF00003E0E3EC55F0FDE1A8EC55F00F0ED2ECD8
:10A0000055F0FDE144EC58F02DEC57F0BE0E002663
:10A01000D70E01225C0E0222890E03EC5AF003E0F7
:10A02000E3EC55F0FDE1B8EC55F00A0ED2EC55F03A
:10A03000FDE107EC5AF03AEC57F0220E0026110E23
:10A040000122900E02226B0E8DEC59F003E0E3EC3E
:10A0500055F0FDE1B5EC55F0190ED2EC55F0FDE1EF
:10A0600011EC58F047EC57F0930E0026710E0122C8
:10A07000980E08EC58F00C0F82EC55F004EC56F0FA
:10A080000C0E1F0B03E0E3EC55F0FDE1C5EC55F0C1
:10A09000140ED2EC55F0FDE12CEC58F054EC57F0D6
:10A0A0008E0E0026430E0122790E0222A60ED2EC5D
:10A0B00059F003E0E3EC55F0FDE1A8EC55F00F0E8C
:10A0C000D2EC55F0FDE144EC58F061EC57F0210E74
:10A0D0000026080E0122B40E0222490E03EC5AF0AB
:10A0E00003E0E3EC55F0FDE1B8EC55F00A0ED2ECDC
:10A0F00055F0FDE178EC58F0ABEC56F0620E00261E
:10A10000250E01221E0E0222F60E91EC59F003E0FC
:10A11000E3EC55F0FDE1B5EC55F01B0ED2EC55F03B
:10A12000FDE194EC58F0ECEC56F0400E0026B30E36
:10A130000122400E0222C00ED6EC59F003E0E3ECFF
:10A1400055F0FDE1C5EC55F0170ED2EC55F0FDE1F0
:10A150006BEC58F02DEC57F0510E00265A0E0122F0
:10A160005E0E0222260EDAEC59F003E0E3EC55F025
:10A17000FDE1A8EC55F0120ED2EC55F0FDE180ECBB
:10A1800058F09EEC56F0AA0E0026C70E0122B60E1D
:10A190000222E90EDEEC59F003E0E3EC55F0FDE1BC
:10A1A000B8EC55F00C0ED2EC55F0FDE178EC58F01F
:10A1B000DFEC56F05D0E0026100E01222F0E02225B
:10A1C000D60E91EC59F003E0E3EC55F0FDE1B5EC6F
:10A1D00055F01B0ED2EC55F0FDE194EC58F020EC5C
:10A1E00057F0530E0026140E0122440E0222020ED6
:10A1F000D6EC59F003E0E3EC55F0FDE1C5EC55F089
:10A20000170ED2EC55F0FDE16BEC58F061EC57F015
:10A21000810E0026E60E0122A10E0222D80EDAECF3
:10A2200059F003E0E3EC55F0FDE1A8EC55F0120E17
:10A23000D2EC55F0FDE180EC58F0D2EC56F0C80EAF
:10A240000026FB0E0122D30E0222E70EDEEC59F0AF
:10A2500003E0E3EC55F0FDE1B8EC55F00C0ED2EC68
:10A2600055F0FDE178EC58F013EC57F0E60E0026BF
:10A27000CD0E0122E10E0222210E91EC59F003E0F5
:10A28000E3EC55F0FDE1B5EC55F01B0ED2EC55F0CA
:10A29000FDE194EC58F054EC57F0D60E0026070E72
:10A2A0000122370E0222C30ED6EC59F003E0E3EC94
:10A2B00055F0FDE1C5EC55F0170ED2EC55F0FDE17F
:10A2C0006BEC58F0C5EC56F0870E00260D0E0122FF
:10A2D000D50E0222F40EDAEC59F003E0E3EC55F06F
:10A2E000FDE1A8EC55F0120ED2EC55F0FDE180EC4A
:10A2F00058F006EC57F0ED0E0026140E01225A0E0F
:10A300000222450EDEEC59F003E0E3EC55F0FDE1EE
:10A31000B8EC55F00C0ED2EC55F0FDE178EC58F0AD
:10A3200047EC57F0050E0026E90E0122E30E02224B
:10A33000A90E91EC59F003E0E3EC55F0FDE1B5EC2A
:10A3400055F01B0ED2EC55F0FDE194EC58F0B8EC52
:10A3500056F0F80E0026A30E0122EF0E0222FC0E8C
:10A36000D6EC59F003E0E3EC55F0FDE1C5EC55F017
:10A37000170ED2EC55F0FDE16BEC58F0F9EC56F00D
:10A38000D90E0026020E01226F0E0222670EDAECB1
:10A3900059F003E0E3EC55F0FDE1DADB120ED2EC0C
:10A3A00055F0FDE180EC58F03AEC57F08A0E0026AB
:10A3B0004C0E01222A0E02228D0EDEEC59F003E033
:10A3C000E3EC55F0FDE1D4DB0C0EECDBFEE1AFEC91
:10A3D00058F0DFEC56F0420E0026390E0122FA0E3C
:10A3E0000222FF0E95EC59F002E0EDDBFEE1BDDB51
:10A3F0001C0ED8DBFEE1C7EC58F006EC57F0810EDE
:10A400000026F60E0122710E0222870EE2EC59F0B0
:10A4100002E0D9DBFEE1B9DB150EC4DBFEE1B6ECF0
:10A4200058F02DEC57F0220E0026610E01229D0EF1
:10A4300002226D0EE6EC59F002E0C5DBFEE188DB9E
:10A44000100EB0DBFEE1CFEC58F054EC57F00C0EE0
:10A450000026380E0122E50E9FEC59F0170E1F0B57
:10A4600002E0B1DBFEE184DB090E9CDBFEE1AFEC38
:10A4700058F0ABEC56F0440E0026EA0E0122BE0E58
:10A480000222A40E95EC59F002E09DDBFEE16DDBAB
:10A490001C0E88DBFEE1C7EC58F0D2EC56F0A90E9A
:10A4A0000026CF0E0122DE0E02224B0EE2EC59F006
:10A4B00002E089DBFEE169DB150E74DBFEE1B6EC40
:10A4C00058F0F9EC56F0600E00264B0E0122BB0E40
:10A4D0000222F60EE6EC59F002E075DBFEE138DB15
:10A4E000100E60DBFEE1CFEC58F020EC57F0700E60
:10A4F0000026BC0E0122BF0E0222BE0E0BEC5AF04B
:10A5000002E061DBFEE134DB090E4CDBFEE1AFEC87
:10A5100058F047EC57F0C60E00267E0E01229B0E27
:10A520000222280E95EC59F002E04DDBFEE11DDB26
:10A530001C0E38DBFEE1C7EC58F09EEC56F0FA0E2C
:10A540000026270E0122A10E0222EA0EE2EC59F0AB
:10A5500002E039DBFEE119DB150E24DBFEE1B6EC8F
:10A5600058F0C5EC56F0850E0026300E0122EF0E95
:10A570000222D40EE6EC59F002E025DBFEE1E8DA37
:10A58000100E10DBFEE1CFEC58F0ECEC56F0050EAF
:10A5900000261D0E0122880E0222040E0BEC5AF03A
:10A5A00002E011DBFEE1E4DA090EFCDAFEE1AFECD9
:10A5B00058F013EC57F0390E0026D00E0122D40EBD
:10A5C0000222D90E95EC59F002E0FDDAFEE1CDDA77
:10A5D0001C0EE8DAFEE1C7EC58F03AEC57F0E50E55
:10A5E0000026990E0122DB0E0222E60EE2EC59F063
:10A5F00002E0E9DAFEE1C9DA150ED4DAFEE1B6ECE2
:10A6000058F061EC57F0F80E00267C0E0122A20EE5
:10A6100002221F0EE6EC59F002E0D5DAFEE198DAEC
:10A62000100EC0DAFEE1CFEC58F0A2DB650E00267A
:10A63000560E0122AC0E0222C40E0BEC5AF002E0C0
:10A64000C2DAFEE195DA090EADDAFEE19DEC58F0D2
:10A6500075DB440E0026220E0122290E0222F40E82
:10A660009AEC59F002E0AFDAFEE17FDA1A0E9ADADC
:10A67000FEE188EC58F0BDDB970E0026FF0E0122AC
:10A680002A0E0222430EEAEC59F002E09CDAFEE1C7
:10A690007CDA160E87DAFEE1BDEC58F054EC57F088
:10A6A000A70E0026230E0122940E0222AB0EEEEC22
:10A6B00059F002E088DAFEE14BDA110E73DAFEE1BE
:10A6C000A6EC58F07CDB390E0026A00E0122930E7A
:10A6D0000222FC0EF2EC59F002E075DAFEE148DAF3
:10A6E0000B0E60DAFEE19DEC58F0C4DBC30E0026D1
:10A6F000590E01225B0E0222650E9AEC59F002E01F
:10A7000062DAFEE132DA1A0E4DDAFEE188EC58F038
:10A710003CDB920E0026CC0E01220C0E02228F0E84
:10A72000EAEC59F002E04FDAFEE12FDA160E3ADADF
:10A73000FEE1BDEC58F084DB7D0E0026F40E012214
:10A74000EF0E0222FF0EEEEC59F002E03CDAFEE1E1
:10A75000FFD9110E27DAFEE1A6EC58F0FCDAD10E93
:10A7600000265D0E0122840E0222850EF2EC59F0C5
:10A7700002E029DAFEE1FCD90B0E14DAFEE19DECD1
:10A7800058F044DB4F0E00267E0E0122A80E022256
:10A790006F0E9AEC59F002E016DAFEE1E6D91A0ED5
:10A7A00001DAFEE188EC58F08CDBE00E0026E60EC4
:10A7B00001222C0E0222FE0EEAEC59F002E003DA2E
:10A7C000FEE1E3D9160EEED9FEE1BDEC58F004DB54
:10A7D000140E0026430E0122010E0222A30EEEECFF
:10A7E00059F002E0F0D9FEE1B3D9110EDBD9FEE158
:10A7F000A6EC58F04CDBA10E0026110E0122080E2B
:10A8000002224E0EF2EC59F002E0DDD9FEE1B0D9A1
:10A810000B0EC8D9FEE19DEC58F0C4DA820E00267A
:10A820007E0E0122530E0222F70E9AEC59F002E03E
:10A83000CAD9FEE19AD91A0EB5D9FEE188EC58F0D2
:10A840000CDB350E0026F20E01223A0E0222BD0E5E
:10A85000EAEC59F002E0B7D9FEE197D9160EA2D979
:10A86000FEE1BDEC58F084DABB0E0026D20E0122C8
:10A87000D70E02222A0EEEEC59F002E0A4D9FEE136
:10A8800067D9110E8FD9FEE1A6EC58F0CCDA910E03
:10A890000026D30E0122860E0222EB0EF2EC59F0B6
:10A8A00002E091D9FEE164D90B0E7CD9FEE10BD90F
:10A8B000E4D94EEC59F0040EE3EC58F035EC59F0C5
:10A8C000080EE3EC58F028EC59F00C0EE3EC58F0CD
:10A8D0001BEC59F0100EE15C02E2E16AE5523ED356
:10A8E00012DBFCDA3AE2DFCF06F0010EDBCF07F035
:10A8F000D89006360736D89006360736FB0EDB5062
:10A900000624A1EC59F00720EA6EEECF02F00250C7
:10A91000E66E6BEC59F0B8D9080E44D9FEE104504C
:10A92000E66E010ED7EC58F0AFD9100E3BD9FEE120
:10A930000450E66E020ED7EC58F0A6D9180E32D9A4
:10A94000FEE10450E66E030ED7EC58F005EC59F02A
:10A95000E552E750EF6EE4DAC4D7080EE15C02E29C
:10A96000E16AE552FBD2CFDAB9DA01E3A2D022DB09
:10A97000A1EC59F00720EA6EEFCF02F0036A046AF7
:10A98000056A010E0C6E0D6A0E6A0F6AC1EC59F071
:10A99000EE500C26EE500D22EE500E22EE500F22FD
:10A9A000FB0EDB500C24A1EC59F00D20EA6EEFCF2A
:10A9B00008F0096A0A6A0B6A080E1F0B02E004DB42
:10A9C000FEE108500212095003120A5004120B5003
:10A9D0000512020E146E156A166A176AC1EC59F058
:10A9E000EE501426EE501522EE501622EE5017228D
:10A9F000FB0EDB501424A1EC59F01520EA6EEFCFCA
:10AA000010F0116A126A136A100E1F0B07E0D8903B
:10AA10001036113612361336E806F9E110500212DC
:10AA2000115003121250041213500512030E1C6E23
:10AA30001D6A1E6A1F6AC1EC59F0EE501C26EE50CA
:10AA40001D22EE501E22EE501F22FB0EDB501C2456
:10AA5000A1EC59F01D20EA6EEFCF18F0196A1A6ABE
:10AA60001B6A180E1F0B07E0D890183619361A36D5
:10AA70001B36E806F9E118500212195003121A5059
:10AA800004121B500512DFCF00F0010EDBCF01F0E6
:10AA9000D89000360136D89000360136B6DB02C0B9
:10AAA000EEFF03C0EEFF04C0EEFF05C0EEFF38DA94
:10AAB0005BD7080EE15C02E2E16AE5524FD288DB27
:10AAC00090DB1BEF59F084DB040E00C0DBFF050EAA
:10AAD00001C0DBFF060E02C0DBFF070E03C0DBFF79
:10AAE000C1EC59F028EF59F073DB98DBF6EC59F024
:10AAF000DACFEAFF4EEF59F06BDBC4DBC5EC59F05F
:10AB000035EF59F0E96EDACFEAFF7BEF59F0DACF93
:10AB1000EAFF0C50EE14086E0D50EE14096E0E5044
:10AB2000EE140A6E0F50EE140B6EC4D303220050C5
:10AB3000DE260150DE220250DE220350DD22DD52ED
:10AB4000DD52C5EC59F0BAEC59F0EFCF03F012002A
:10AB5000080EDBCF04F0090EDBCF05F00A0EDBCFC9
:10AB600006F00B0EDBCF07F01200C5EC59F0BAD39C
:10AB7000040EDBCF04F0050EDBCF05F0060EDBCFB5
:10AB800006F0070EDBCF07F012000C0EDBCF04F04F
:10AB90000D0EDBCF05F00E0EDBCF06F00F0EDBCF78
:10ABA00007F01200D8900732063205320432E80668
:10ABB000120012EC5AF00816EE500916EE500A1662
:10ABC000EE500B1677D3D890003601360236033696
:10ABD000E806120012EC5AF00416EE500516EE507C
:10ABE0000616EE5007161200DACFEAFF0850EE18EC
:10ABF000046E0950EE18056E0A50EE18066E0B50E2
:10AC0000EE18076E045012000C0EDBCF00F00D0E94
:10AC1000DBCF01F00E0EDBCF02F00F0EDBCF03F027
:10AC20001200080EDBCF00F0090EDBCF01F00A0E98
:10AC3000DBCF02F00B0EDBCF03F012004CDBA5EFF5
:10AC400059F0F0DB041AEE50051AEE50061AEE50D9
:10AC5000071A04501200E6DB081AEE50091AEE50EB
:10AC60000A1AEE500B1A1200DDDB0412EE50051228
:10AC7000EE500612EE5007121200FD0EDBCFE9FF78
:10AC8000FE0EDBCFEAFF1200C0DAE552E750EF6EAE
:10AC9000DFCF08F0010EDBCF09F0D8900836093677
:10ACA000D89008360936FB0EDB5008244ADB092011
:10ACB000EA6E18D30C0EDBCF08F00D0EDBCF09F0D7
:10ACC0000E0EDBCF0AF00F0EDBCF0BF01200080EDA
:10ACD000DBCF08F0090EDBCF09F00A0EDBCF0AF05C
:10ACE0000B0EDBCF0BF01200040EDBCF08F0050ECD
:10ACF000DBCF09F0060EDBCF0AF0070EDBCF0BF03F
:10AD0000120043DBEECF08F0EECF09F0EECF0AF0F1
:10AD1000EFCF0BF01200DBCF0FF00C1E0D1E0E1E3E
:10AD20000F1E1200081E091E0A1E0B1ED95012000B
:10AD3000041E051E061E071ED95012000A01A82572
:10AD4000006E0550A921016E0650AA21026E07501F
:10AD5000AB21036E12000A01AC25006E0550AD2137
:10AD6000016E0650AE21026E0750AF21036E120035
:10AD70000A01B025006E0550B121016E0650B221C6
:10AD8000026E0750B321036E12000A01B425006E53
:10AD90000550B521016E0650B621026E0750B7214D
:10ADA000036E12000A01B825006E0550B921016E2C
:10ADB0000650BA21026E0750BB21036E12000A0131
:10ADC000BC25006E0550BD21016E0650BE21026EED
:10ADD0000750BF21036E12000A01C025006E055006
:10ADE000C121016E0650C221026E0750C321036EBD
:10ADF00012000A01C425006E0550C521016E0650DF
:10AE0000C621026E0750C721036E12000A01C82531
:10AE1000006E0550C921016E0650CA21026E07500E
:10AE2000CB21036E12000A01CC25006E0550CD2106
:10AE3000016E0650CE21026E0750CF21036E120024
:10AE40000A01D025006E0550D121016E0650D22195
:10AE5000026E0750D321036E12000A01D425006E42
:10AE60000550D521016E0650D621026E0750D7211C
:10AE7000036E12000A01D825006E0550D921016E1B
:10AE80000650DA21026E0750DB21036E12000A0120
:10AE9000DC25006E0550DD21016E0650DE21026EBC
:10AEA0000750DF21036E12000A01E025006E0550F5
:10AEB000E121016E0650E221026E0750E321036E8C
:10AEC00012000A01E425006E0550E521016E0650CE
:10AED000E621026E0750E721036E1200F70EDBCF6A
:10AEE00000F0F80EDBCF01F0EFD94BDA0050EE5C4A
:10AEF0000150EE580250EE580350EE581200E92669
:10AF0000000EEA22120004DA080EE12625DA040E09
:10AF1000DB6A050EDB6A060EDB6A070EDB6A1200CF
:10AF200034DAEE2A000EEE22EE22EE222ADA040EA7
:10AF3000EE26000EEE22EE22EE221200E9CF00F005
:10AF4000EACF01F0E9CFE6FFEACFE6FF1200FB0E01
:10AF5000DBCFE6FFFC0EDBCFE6FF1200E16EE55231
:10AF6000E7CFD9FF120004501F0B04DAEECF03F035
:10AF7000120058DA045C006EEE500558016EEE5077
:10AF800006581200E9CFE6FFEACFE6FFBAEC4EF032
:10AF9000E552E552E552E5521200E66EE66AE66ACF
:10AFA000E66AB3EF59F0D890033202320132003230
:10AFB000E8061200040EDBCF06F0050EDBCF07F02B
:10AFC000FB0EDB5006241200D890083609360A36EC
:10AFD0000B36E8061200F90EDBCF00F0FA0EDBCFDD
:10AFE00001F012007DDC026E080EE15E02501200DC
:10AFF0008FD9100EE126120011EC4DF0006E060EF6
:10B00000E15E00501200016E00C0E6FFE66E120025
:10B010000222FD0E0322D9501200016A026A036A5D
:10B0200012006ADDA5DDD9CFE9FFD4DDAED9EECFC0
:10B030000CF0EECF0DF0EECF0EF0EFCF0FF00C1EB8
:10B040000D1E0E1E0F1EA6D987EF55F00322D950F4
:10B05000080F58DD11EF56F047DD87DDC7D9BADD9F
:10B060000C0EDBCF0CF00D0EDBCF0DF00E0EDBCF98
:10B070000EF00F0E50DEDAD987EF55F00322D950CB
:10B080000C0F40DD04EF56F01ADD7FDD83D9A2DD21
:10B09000080EDBCF0CF0090EDBCF0DF00A0EDBCF74
:10B0A0000EF00B0E38DED9CFE9FF87EF55F050DDFB
:10B0B000BDD990DD040EDBCF0CF0050EDBCF0DF01B
:10B0C000060EDBCF0EF0070E26DE90D987EF55F087
:10B0D0000322D9508FD108DD4BDD88D97BDD04DE1A
:10B0E000081E091E0A1E0B1ED9CFE9FFD9EF55F025
:10B0F000EADC4BDD9BD96EDDDDDD14DE080F8FD180
:10B10000DEDC33DD47D966DDFCDD0CDE0C0F87D1DC
:10B11000F3DC1EDD041E051E061E071ED9CFE9FF47
:10B12000A3DD84D921EF56F0E7DC12DDD9CFE9FFAA
:10B1300051DDCDDDF7DD040F72D1C5DC26DDF8DD94
:10B14000040FE96E91DD26D921EF56F0B8DC0DDD54
:10B15000EFDD080FE96E88DD49D921EF56F0B3DC49
:10B16000B6DD64D978DD42D9F4EF55F0BDDCC9DD38
:10B170003DD971DD5BD9F4EF55F0B6DCF9DCD8DDF3
:10B180000C0FE96E71DDD9CFE9FF21EF56F0B4DC89
:10B19000ABDDD9CFE9FF5FDDFDD8F4EF55F08FDCF3
:10B1A00089DDF8D858DDD9CFE9FFF4EF55F0006E0E
:10B1B00034DFE7D8EE500026EE500122EE50022296
:10B1C000EE5003221200E76E58DDE7507FEF57F094
:10B1D00004500012055001120650021207500312CB
:10B1E0001200080E00C0DBFF090E01C0DBFF0A0ED3
:10B1F00002C0DBFF0B0E03C0DBFFCCD8DACFEAFFC7
:10B2000012003BDD100E7FEF57F0FD0EDB500024E7
:10B21000E96EFE0EDB500120EA6E12000C0E00C03B
:10B22000DBFF0D0E01C0DBFF0E0E02C0DBFF0F0EB9
:10B2300003C0DBFF12000C0EDB50EE260D0EDB50C0
:10B24000EE220E0EDB50EE220F0EDB50EE2212002D
:10B25000080EDB50EE26090EDB50EE220A0EDB5004
:10B26000EE220B0EDB50EE221200040EDB50EE2617
:10B27000050EDB50EE22060EDB50EE22070EDB50F1
:10B28000EE22120000C0DFFF010E01C0DBFF020E44
:10B2900002C0DBFF030E03C0DBFF1200DF50EE260F
:10B2A000010EDB50EE22020EDB50EE22030EDB50CD
:10B2B000EE22120008500412095005120A5006121C
:10B2C0000B50071204501200F90EDBCF02F0FA0EF9
:10B2D000DBCF03F01200040EDBCF00F0050EDBCF56
:10B2E00001F01200EECF04F0EECF05F0EECF06F045
:10B2F000EFCF07F012000050EE260150EE22025070
:10B30000EE220350EE221200B8DC180E7FEF57F049
:10B31000D9CFE6FFE1CFD9FF120008DC070E1F0BE3
:10B32000120004DC050E1F0B120096EC55F0040E03
:10B330001F0B120096EC55F0060E1F0B120068DE74
:10B3400059D0E96EFC0EDB501200060EDBCF02F086
:10B35000070EDBCF03F01200DE6ADE6ADE6ADD6A0A
:10B36000DD52DD521200FB0EDBCFE9FFFC0EDBCF1E
:10B37000EAFF1200EECF00F0EECF01F0EECF02F0C8
:10B38000120054D8DACFEAFF1200D9CFE9FFDACFA2
:10B39000EAFF1200D950080FE96E120032DF040EE6
:10B3A0007FEF57F053DE110E1F0B120067DE090E00
:10B3B0001F0B12004BDE0E0E1F0B120089DE140E47
:10B3C0001F0B12005BDE0B0E1F0B12003FDE100E78
:10B3D0001F0B120053DE0A0E1F0B120037DE0F0E7A
:10B3E0001F0B120075DE150E1F0B1200D9500C0F2B
:10B3F000E96E1200040F82EC55F01EEF56F03EDEAF
:10B400000C0E1F0B120064DE160E1F0B120063ECF5
:10B4100055F057EF58F05CDE170E1F0B1200E96E67
:10B42000D9EF55F0DACFEAFFEE501200D950040FF1
:04B43000E96E1200AF
:0CB4340048EC64F021EC66F009E1050131
:10B44000880EFD6FFA0EFE6F000EA3EC64F017D0AD
:10B4500005017E0EFD6FFA0EFE6F000EA3EC64F088
:10B460007CEC65F007EC66F005017A0EFD6FFA0ED4
:10B47000FE6F000EA3EC64F0020EB8EC64F04DEF2A
:10B4800064F021EC66F003E160EC65F006D00501A4
:10B49000750EFD6FFA0EFE6F000EA3EF64F048EC20
:10B4A00064F00601F3B50BD032EC64F0FBC8FDF597
:10B4B000FCC8FEF5FDC8FFF5FEEC3EF0E2DF4DEF07
:10B4C00064F048EC64F00601F3B509D032EC64F0A6
:10B4D000FEC8E6FFFFC8E6FF07EC66F0D2DF4DEFDF
:10B4E00064F0A4EC65F0F3A502D0000E11D06EEC70
:10B4F00066F04CEC66F0ABEC37F0E552E5524CEC04
:10B5000066F076EC74F0E552E55251EC64F0010E11
:10B51000E9EC64F002E2E16AE552E16E00504DEFC1
:10B5200064F0A4EC65F0F3B509D090EC66F0170E6A
:10B53000FD6F460EFE6F010E3DEC66F0020EE15C03
:10B5400002E2E16AE552E16E4DEF64F0A4EC65F0D1
:10B55000F3B509D090EC66F0320EFD6F460EFE6F2B
:10B56000010E3DEC66F0020EE15C02E2E16AE5529A
:10B57000E16E4DEF64F0AAEC65F00A0E6EEC66F039
:10B580000901A051E66EE66A4C0EE66EFA0EE66E12
:10B59000000EB9EC65F078EC64F0450EE66EFA0E3C
:10B5A000E66E000EBCEC65F002E2E16AE552E16E87
:10B5B0004DEF64F0AAEC65F00A0E6EEC66F0070140
:10B5C000CAA308D085EC64F01E0EE66EFA0EE66E95
:10B5D000000E07D085EC64F0060EE66EFA0EE66EFD
:10B5E000000E96EC66F066EC66F0D4EC64F0FE0EAD
:10B5F000E66EF90EE66E000E90EC64F0FB0EE66E61
:10B60000F90EE66E000EBCEC65F002E2E16AE5526E
:10B61000E16E4DEF64F0AAEC65F0E66AB3EC64F01D
:10B62000DFEC64F0FD0EDBCFE6FFFE0EFBEC64F01A
:10B6300002E1010E06D00601F3B302D0BDEC64F0C6
:10B64000000EE9EC64F002E2E16AE552E16E0050BE
:10B650004DEF64F07DEC66F0D950FB0F51EC66F0D5
:10B660000BE0DFEC64F0FB0EDBCFE6FFFC0EFBEC47
:10B6700064F002E1010E06D00601F3B302D0BDEC86
:10B6800064F0000EE9EC64F002E2E16AE552E16E7A
:10B6900000504DEF64F048EC64F02BEC65F021E0D5
:10B6A00028EC66F040EC66F07CEC65F040EC9FF036
:10B6B00079EC66F0E7CF01F0E552E7CF00F00050FB
:10B6C000F3240801F96F0150F420FA6FF9C800F073
:10B6D000016EFD0EDB50001807E1FE0EDB50011875
:10B6E00003E1F36AF46A16D0FD0E6CEC65F025EC0C
:10B6F00066F008E082EC64F005E0DF2A010EF7E373
:10B70000DB2AF5D725EC66F003E1EAEC65F0EF6A99
:10B7100031EC65F0020EE15C02E2E16AE552E16EB5
:10B720004DEF64F048EC64F02BEC65F016E0FD0E94
:10B730006CEC65F082EC64F005E0DF2A010EFAE3C0
:10B74000DB2AF8D7DECF00F0DDCF01F00801F95198
:10B75000001806E1FA51011803E1F36AF46A21D0F6
:10B76000DF2A010E01E3DB2AD9CFE9FFDACFEAFFB6
:10B77000FD0EEECFDBFFFE0EEDCFDBFF25EC66F01E
:10B7800008E082EC64F005E0DF2A010EF7E3DB2A33
:10B79000F5D725EC66F003E1EAEC65F0EF6A31ECF1
:10B7A00065F0020EE15C02E2E16AE552E16E4DEF06
:10B7B00064F0AAEC65F0E66AB3EC64F00601F3A568
:10B7C00002D0000E0BD032EC64F083EC65F0E70E93
:10B7D000E66EF90EE66E000E88EC65F0E9EC64F0BA
:10B7E00002E2E16AE552E16E00504DEF64F048EC90
:10B7F00064F07CEC65F0E66A67EC65F0F3A502D0D6
:10B80000000E0AD0A7EC65F0DA0EFD6F440EFE6F55
:10B81000010EA3EC64F0010E4DEF64F07DEC66F0D8
:10B820000601F3A502D0000E0BD032EC64F083ECDD
:10B8300065F0D50EE66EF90EE66E000E88EC65F04A
:10B84000E9EC64F002E2E16AE552E16E00504DEF8E
:10B8500064F048EC64F071EC65F0010EE66E67ECA4
:10B8600065F0F3A502D0000E0AD0A7EC65F0070E34
:10B87000FD6F450EFE6F010EA3EC64F0010E4DEF5F
:10B8800064F0A4EC65F0F3A502D0000E27D06EECB6
:10B8900066F0D1C9E6FFD2C9E6FFD3C9E6FFD4C935
:10B8A000E6FF560EE66E460EE66E010E96EC66F06C
:10B8B00037EC65F0D5C9E6FFD6C9E6FFD7C9E6FF84
:10B8C000D8C9E6FFD30EE66EF90EE66E000E93ECD5
:10B8D00066F037EC65F051EC64F0010EE9EC64F0D1
:10B8E00002E2E16AE552E16E00504DEF64F048EC8F
:10B8F00064F07CEC65F0F5DDE552E5524DEF64F067
:10B9000048EC64F0070EE1260601F3A502D0000E14
:10B9100070D0A7EC65F00CEC66F0070EF36E020E2B
:10B92000F3CFDBFFDF6A200EDF5C62E2DFCFE6FFF2
:10B9300051ECA8F0E552030EF3CFDBFF040EF4CF79
:10B94000DBFF030EDBCFE9FF040EDBCFEAFFEF5096
:10B950004DE0DFCFE6FFE66AC90EE66EF90EE66E51
:10B96000000EB9EC65F03FEC65F0030EDBCFE6FFAF
:10B97000040EDBCFE6FFC70EE66EF90EE66E000E94
:10B98000E66E050EDBCFE6FF060EDBCFE6FFBAEC78
:10B9900074F03FEC65F0050EDBCF00F0060EDBCF58
:10B9A00001F0000E005E060E015A010E00C0DBFF22
:10B9B000DBCFE6FF020EDB50E552E724006E016AA2
:10B9C000013412E20050A008000E01540DE259DDCE
:10B9D000140E90EC66F00CEC66F0010EDB50070FD5
:10B9E000E76E020EE7CFDBFF51EC64F0DF2A9BD756
:10B9F000010E006E070EE15C02E2E16AE552E16EC3
:10BA000000504DEF64F048EC64F0E652020EDF6E39
:10BA1000200EDF5C11E278EC65F00EE0EFEC65F0F3
:10BA200006E1AEEC65F003E163EC64F002D071EC8A
:10BA300065F0A6EC64F0ECD7A7EC65F0290EFD6F7D
:10BA4000450EFE6F010E3DEC66F0A7EC9BF021EC7D
:10BA500066F002E0CEEC64F0000EE5524DEF64F0CB
:10BA600045EC66F0DF6A010EE66E51ECA8F0E55297
:10BA700062EC66F0200EDF5C11E278EC65F00EE01F
:10BA8000EFEC65F006E1AEEC65F003E163EC64F029
:10BA900002D071EC65F0A6EC64F0ECD721EC66F016
:10BAA00004E0E66A98EC40F0E552000E006E030EEA
:10BAB000E15C02E2E16AE552E16E00504DEF64F0B4
:10BAC000A4EC65F0F3A502D0000E31D032EC64F0A6
:10BAD000BF0EE66EF90EE66E000E58EC64F0080E2E
:10BAE00044EC64F0B10EE66EF90EE66E000E40EC2A
:10BAF00064F00E0E44EC64F0A10EE66EF90EE66EF4
:10BB0000000E40EC64F0020E44EC64F0970EE66E1A
:10BB1000F90EE66E000E40EC64F0030E44EC64F0A7
:10BB2000850EE66EF90EE66E000E03EC66F0E9ECAB
:10BB300064F002E2E16AE552E16E00504DEF64F01C
:10BB400049EC66F0080E38EC64F00EE071EC65F03C
:10BB5000020E38EC64F008E071EC65F0030E38EC8E
:10BB600064F002E006EC65F054EC64F0A9DF42EC0E
:10BB700065F002E0CEEC64F0DF50E5524DEF64F08A
:10BB8000A4EC65F0F3A502D0000E13D032EC64F003
:10BB90007C0EE66EF90EE66E000E58EC64F00E0EAA
:10BBA00044EC64F06B0EE66EF90EE66E000E03ECEC
:10BBB00066F0E9EC64F002E2E16AE552E16E005001
:10BBC0004DEF64F048EC64F0E652EFEC65F003E111
:10BBD0007BEC64F0EF6A06EC65F054EC64F0D0DFC7
:10BBE00042EC65F002E0CEEC64F0DF50E5524DEF40
:10BBF00064F0A4EC65F0F3A502D0000E56D032EC50
:10BC000064F0650EE66EF90EE66E000E58EC64F018
:10BC1000050E44EC64F05D0EE66EF90EE66E000E65
:10BC200040EC64F0060E44EC64F0540EE66EF90E3F
:10BC3000E66E000E40EC64F0070EF3EC65F0EC0EDF
:10BC4000E66E090EE66E3F0EE66EF90EE66E000E2B
:10BC500093EC66F0BAEC74F078EC64F00A0163518E
:10BC600006E01C0EE66EF90EE66E000E19D0200EF0
:10BC70000501C85D06E1F90EE66EF80EE66E000EEF
:10BC80000FD0C851E66EE66ADA0EE66EF80EE66E82
:10BC9000000E74EC66F0D80EE66EF80EE66E000E3E
:10BCA0003CEC64F051EC64F0010EE9EC64F002E26B
:10BCB000E16AE552E16E00504DEF64F049EC66F048
:10BCC000050E38EC64F01DE0EFEC65F006E1AEEC3B
:10BCD00065F003E163EC64F002D071EC65F0060EF0
:10BCE00038EC64F00EE0EFEC65F006E1AEEC65F0E8
:10BCF00003E163EC64F002D071EC65F0070E9AEC9E
:10BD000065F054EC64F075DFEDEC64F002E0CEEC2D
:10BD100064F0DF50E5524DEF64F0A4EC65F0F3A55C
:10BD200002D0000E2AD0A7EC65F0CE0EFD6FF80E03
:10BD3000FE6F000EA3EC64F00D0EE66EB3EC64F043
:10BD400082EC64F007E10501C50EFD6FF80EFE6F91
:10BD5000000E06D083EC65F007EC66F060EC65F051
:10BD6000A3EC64F0EC0EE66E090EE66EBB0EE66E1A
:10BD7000F80EE66E000E88EC65F0E9EC64F002E285
:10BD8000E16AE552E16E00504DEF64F0AAEC65F017
:10BD900078EC65F009E1010EDB6AD950010FE66E1F
:10BDA000000EDA20E66E02D071EC65F00D0E9AEC12
:10BDB00065F054EC64F0B1DFEDEC64F002E0CEEC41
:10BDC00064F0DF50E9EC64F002E2E16AE552E16E12
:10BDD00000504DEF64F0A4EC65F0F3A502D0000E26
:10BDE00020D032EC64F0B30EE66EF80EE66E000E74
:10BDF00058EC64F0040E44EC64F0AC0EE66EF80E01
:10BE0000E66E000E40EC64F0090EF3EC65F00A0EED
:10BE100044EC64F09F0EE66EF80EE66E000E03EC46
:10BE200066F0E9EC64F002E2E16AE552E16E00508E
:10BE30004DEF64F049EC66F0040E38EC64F00BE072
:10BE400071EC65F0090E38EC64F005E071EC65F01A
:10BE50000A0E9AEC65F054EC64F0BDDFEDEC64F092
:10BE600002E0CEEC64F0DF50E5524DEF64F0A4EC5C
:10BE700065F0F3A502D0000E9ED032EC64F0990E6E
:10BE8000E66EF80EE66E000E58EC64F00901F9510A
:10BE9000E66EE66A8E0EE66EF80EE66E000E58EC62
:10BEA00066F00901FA51E66EE66A830EE66EF80E58
:10BEB000E66E000E58EC66F00501C851E66EE66AC3
:10BEC000740EE66EF80EE66E000E74EC66F0090174
:10BED000EA51000812E285EC64F0680EE66EF80E96
:10BEE000E66E000E90EC64F0D4EC64F0620EE66E48
:10BEF000F80EE66E000E90EC64F00601F551E66E69
:10BF0000E66A570EE66EF80EE66E000E58EC66F026
:10BF10000601F6514DE04D0EE66EF80EE66E000E8F
:10BF20003CEC64F00601F6A107D0480EE66EF80E70
:10BF3000E66E000E3CEC64F00601F6A307D0430E5B
:10BF4000E66EF80EE66E000E3CEC64F00601F6A517
:10BF500007D03F0EE66EF80EE66E000E3CEC64F085
:10BF60000601F6A707D03B0EE66EF80EE66E000E51
:10BF70003CEC64F00601F6A907D0370EE66EF80E29
:10BF8000E66E000E3CEC64F00601F6AB07D02F0E17
:10BF9000E66EF80EE66E000E3CEC64F00601F6ADBF
:10BFA00007D0270EE66EF80EE66E000E3CEC64F04D
:10BFB00051EC64F0010EE9EC64F002E2E16AE55252
:10BFC000E16E00504DEF64F045EC66F00601F3A51C
:10BFD00002D0000E2CD0A7EC65F01D0EFD6FF80E00
:10BFE000FE6F000EA3EC64F0DF6A100EDF5C1EE251
:10BFF0004BEC65F0EF5018E0DFCFE6FFE66A190E74
:10C00000E66EF80EE66E000ECAEC64F04BEC65F0DE
:10C01000EF50E66EE66AC70EE66EF90EE66E000EAB
:10C020005CEC64F051EC64F0DF2ADFD7010E006EA7
:10C03000030EE15C02E2E16AE552E16E00504DEF71
:10C0400064F048EC64F0E65278EC65F002E1000E32
:10C0500031D011EC65F0DF6E71EC66F0000EDF5C44
:10C0600028E3100EDF5C25E278EC65F022E011ECAD
:10C0700065F0E66E4BEC65F0E552E750EF6E080EAA
:10C08000DF5C07E371EC65F0080EDF5C180F9AECDB
:10C0900065F00F0EDF5C02E1A7EC9BF0A7EC65F00A
:10C0A000430EFD6F450EFE6F010EA3EC64F0010E12
:10C0B00001D0000EE552F1D3B3EC65F017E0F90EB4
:10C0C000DBCFE6FFFA0EDBCFE6FF180EE66EE66A80
:10C0D000E66A07D0F2C8FBFFF1C8FAFF0801F05189
:10C0E000F96EF8DF006E050EE15E0050A7EC65F01A
:10C0F000590EFD6F450EFE6F010EB6EF65F0B3EC05
:10C1000065F017E0F90EDBCFE6FFFA0EDBCFE6FFB6
:10C11000140EE66EE66AE66A07D0F2C8FBFFF1C8C5
:10C12000FAFF0801F051F96EF8DF006E050EE15ECE
:10C130000050A7EC65F06C0EFD6F450EFE6F010E12
:10C14000B6EF65F0B3EC65F017E0F90EDBCFE6FF74
:10C15000FA0EDBCFE6FF160EE66EE66AE66A07D059
:10C16000F2C8FBFFF1C8FAFF0801F051F96EF8DFE1
:10C17000006E050EE15E0050A7EC65F0830EFD6FCA
:10C18000450EFE6F010EB6EF65F0B3EC65F017E0FB
:10C19000F90EDBCFE6FFFA0EDBCFE6FF150EE66EFB
:10C1A000E66AE66A07D0F2C8FBFFF1C8FAFF0801A9
:10C1B000F051F96EF8DF006E050EE15E0050A7EC5D
:10C1C00065F09C0EFD6F450EFE6F010EB6EF65F03B
:10C1D000B3EC65F017E0F90EDBCFE6FFFA0EDBCF2C
:10C1E000E6FF170EE66EE66AE66A07D0F2C8FBFFC6
:10C1F000F1C8FAFF0801F051F96EF8DF006E050E84
:10C20000E15E0050A7EC65F0B10EFD6F450EFE6FCC
:10C21000010EB6EF65F03CDBE150F90F51EC66F032
:10C2200001E18BD071EC65F02EECA0F0E552E55207
:10C23000CBDB01E190D0030EE66EE66A150EE66EEA
:10C24000F80EE66E000E4DDB12E1130EE66EF80EF0
:10C25000E66E0A0EE66EE66AE66A07D0F2C8FBFFF3
:10C26000F1C8FAFF0801F051F96EF8DF53D0030E60
:10C27000E66EE66A0F0EE66EF80EE66E000E31DB35
:10C2800012E10D0EE66EF80EE66E0A0EE66EE66A36
:10C29000E66A07D0F2C8FBFFF1C8FAFF0801F051C7
:10C2A000F96EF8DF37D0030EE66EE66A090EE66E29
:10C2B000F80EE66E000E15DB12E1070EE66EF80EC4
:10C2C000E66E0A0EE66EE66AE66A07D0F2C8FBFF83
:10C2D000F1C8FAFF0801F051F96EF8DF1BD0030E28
:10C2E000E66EE66A030EE66EF80EE66E000EF9DA0A
:10C2F00024E1010EE66EF80EE66E0A0EE66EE66AC0
:10C30000E66A07D0F2C8FBFFF1C8FAFF0801F05156
:10C31000F96EF8DF006E050EE15E005071EC66F01C
:10C32000E7DB19E0F90EDBCFE6FFFA0EDBCFE6FF25
:10C330000F0EE66EE66AE66A09D0000E15D0F2C866
:10C34000FBFFF1C8FAFF0801F051F96EF8DF006E4B
:10C35000050EE15E0050A7EC65F0CD0EFD6F450EB9
:10C36000FE6F010EF0DA010E98D2B3EC65F014E026
:10C37000000EE66EE66A0B0EE66EE66AE66A07D027
:10C38000F2C8FBFFF1C8FAFF0801F051F96EF8DFBF
:10C39000006E050EE15E00500501FC6BD8DBEA0E75
:10C3A000FD6F450EFE6F010EE1D3DDDB14E0000EE4
:10C3B000E66EE66A0C0EE66EE66AE66A07D0F2C83A
:10C3C000FBFFF1C8FAFF0801F051F96EF8DF006ECB
:10C3D000050EE15E005005011E0EFC6FB8DB010E7C
:10C3E000FD6F460EFE6F010EC1D345EC66F0010EE7
:10C3F000DF6E020EDF6E0E0EF66E000EF76E000E92
:10C4000051DBE90EE66EF70EE66E000EC3DA0F0E94
:10C41000F66E000EF76E000EEEDB100EF66E000EDE
:10C42000F76E000EE8DB0E0E2FDAE50EE66EF70E65
:10C43000E66E000EE66EB9DB2FEC66F062EC66F09D
:10C440000701CC51CD11CE110AE0CCC7E6FFCDC714
:10C45000E6FFCEC7E6FFA9DBAFDB62EC66F0DFCF1D
:10C46000E6FFE66AE20EE66EF70EE66E000E24DAEE
:10C47000F9D917DA010E006E030EE15C02E2E16AFF
:10C48000E552E16E005009D265DB030EE66E98ECD2
:10C4900040F0E552000E9DDA02E2E16AE552E16EFB
:10C4A0000050FBD1F5D9FE0EDB50330A0AE0010A39
:10C4B00005E0030A19E14FDA08E009D0B9DA14E11E
:10C4C00004D0B6DA11E147DA02E1000E0ED05DDBEE
:10C4D00092EC5BF0E552E552F4CF01F082EC66F0AD
:10C4E000F3CFEEFF01C0EDFF010ED7D1D1D9070E7A
:10C4F000E126FB0EF1DA06DA17E0A7DB15E002DA37
:10C5000060080DE267DBEFCF00F07B0E005C07E216
:10C51000F9D9E00FE66E5EDBE552E750EF6EDF2AF9
:10C52000010EE9E3DB2AE7D790DB04E1DF2A010E05
:10C5300001E3DB2A020EDB6A030EDB6A55DAB8DAA6
:10C5400004BE0568040E81DAFEE1EDD901E119D1DE
:10C55000850E066E460E076E010E086E020EDBCFCC
:10C5600009F0030EDBCF0AF00B6A0ABE0B68040E5B
:10C57000D89009360A360B36E806FAE10650092447
:10C58000036E07500A20046E08500B20056E03C08E
:10C59000E6FF04C0E6FFE66E4EEC9FF0AADB27C084
:10C5A00000F028C001F029C002F00006000E015A78
:10C5B000025A66DB850E0F6E460E106E010E116E6E
:10C5C000020EDBCF12F0030EDBCF13F0146A13BEA2
:10C5D0001468040ED890123613361436E806FAE1C1
:10C5E0000F5012240C6E105013200D6E1150142099
:10C5F0000E6E0C2A000E0D220E220CC0E6FF0DC09E
:10C60000E6FF0EC0E6FFDFDA2EEC9EF0156E070E99
:10C61000E15E1550000901E0ADD0040EDB6A73DA6B
:10C620004BEC5BF0E552E55221DBD950050FE66E8D
:10C63000000EDA20E66E60DAD7D93ADA04BE056871
:10C64000040E03DAFEE16FD9E66E2CDF066E050EEE
:10C65000E15E0650000901E1BED00801F351F4117A
:10C66000F51124E0050EDBCFE6FF060EDBCFE6FF7B
:10C67000FB0EDBCFE6FFFC0EDBCFE6FFFD0EDBCFD4
:10C68000E6FFFE0EDBCFE6FF010EE66E07D0F5C833
:10C69000FBFFF4C8FAFF0801F351F96EF8DF006EF2
:10C6A000070EE15E0050000901E095D0020EDBCFDD
:10C6B000E9FF030EDBCFEAFFEA02F3CFEAFFE9026C
:10C6C000F3CFE9FFF450EA26000EE9260A0EEA222B
:10C6D000EECF00F0EECF01F0EFCF02F0050EDBCF92
:10C6E000E6FF060EDBCFE6FFFB0EDBCFE6FFFC0E20
:10C6F000DBCFE6FFFD0EDBCFE6FFFE0EDBCFE6FF76
:10C7000006D002C0FBFF01C0FAFF0050F96EF9DF4E
:10C71000036E060EE15E0350E76E040EE7CFDBFF0B
:10C72000DB5059E00801F351F411F51120E0050E3A
:10C73000DBCFE6FF060EDBCFE6FFFB0EDBCFE6FF2F
:10C74000FC0EDBCFE6FFFD0EDBCFE6FFFE0EDBCF00
:10C75000E6FFE66A07D0F5C8FBFFF4C8FAFF080158
:10C76000F351F96EF8DF006E070EE15E005041EC08
:10C770005AF031D0020EDB2A030E01E2DFD6DB2AAB
:10C78000DDD60801F651F711F8111FE0DECFE6FF04
:10C79000DDCFE6FFFB0EDBCFE6FFFC0EDBCFE6FFD7
:10C7A000FD0EDBCFE6FFFE0EDBCFE6FF07D0F8C8BD
:10C7B000FBFFF7C8FAFF0801F651F96EF8DF006ECB
:10C7C000060EE15E0050000906E1FDD995D9D5ECD1
:10C7D00036F08FDAE552070EE15C02E2E16AE552DB
:10C7E000E16E5BD0B1D9F3A502D0000E34D0AFD941
:10C7F000D80EFD6FF70EFE6F000EA5D8DE6ADD6A5B
:10C8000012DA04BE0568040E20D9FEE18CD822E0BD
:10C810000501D60EFD6FF70EFE6F000E94D803DAF9
:10C8200004BE0568040E11D9FEE100500324050181
:10C83000FD6F01500420FE6F02500520FF6FFD2B9D
:10C84000000EFE23FF23FEEC3EF0DF2A010ED8E3AC
:10C85000DB2AD6D7010EBDD802E2E16AE552E16ECD
:10C8600000501BD049D91AEC5AF0E552E55212009B
:10C8700061D937DA78EF65F056DA9ED99FEF65F027
:10C8800052DAEDD99FEF65F0E66E51ECA8F083D156
:10C89000D9CFE6FFE1CFD9FF1200E552E7CFD9FFAC
:10C8A0001200FAD907EF66F01CD98DD97CEF65F03C
:10C8B0003DDA82D99FEF65F0E66E77D9C2EC74F06D
:10C8C000FCD962EF66F0010EE76EF90EDBCF00F0E7
:10C8D000FA0EDBCF01F0E7500026000E012240EFF8
:10C8E00066F0E66EFED82EEC9EF0E7D90009120045
:10C8F000E4D99FEF65F0F90EDBCFE9FFFA0EDBCF4D
:10C90000EAFF120067D9EF501200010EE66EE66AE8
:10C91000EAC900F0016A026A036AEAC9E6FF8AD13D
:10C9200002DA66EF66F000500324F36E0150042033
:10C93000F46E02500520F86EF4CFF7FFF3CFF6FF48
:10C940000800F5501200FF6FFEEF3EF0DF50DF2AC7
:10C95000F1D871EF66F019D9DCD92AEC5BF0C9D9AE
:10C96000E5520009120051ECA8F0E5529FEF65F086
:10C97000E66E62EC72F0E55212000801C80EFB6F21
:10C98000440EFC6F010EFD6FB7D84FEC5AF0E55224
:10C99000E5521200EED891D962EF66F0400EE66ED5
:10C9A00098EC40F0E5521200010EE66EE66AEBC923
:10C9B00000F0016A026A036AEBC9E6FF3BD1A3D823
:10C9C00040EC9FF0E552E7D00801F051F111F2116F
:10C9D0001200006E020EE15C1200006E060EE15EB7
:10C9E0000050DF6E21EF66F0850E006E460E016E80
:10C9F000010E026E1200DBCFE6FF85D873EC9FF0CC
:10CA0000026E060EE15E0250000912006AD80E0E98
:10CA10009AEF65F0E65271EF65F0020EE12606012D
:10CA200012005FD87EEC92F0E552E552F35012000E
:10CA300070D90BEC5BF0E552E55200091200E750AB
:10CA4000E926000EEA22EF501200D8900336043691
:10CA50000536E8061200020EE126D950FD0F51EF0F
:10CA600066F0F6D800C0F3FF01C0F4FF120092ECAC
:10CA700076F0006E090EE15E00509FEF65F01DD963
:10CA800036EF66F0006E060EE15E0050DF6EA7EC3A
:10CA90009BF021EF66F0DF50EA6AE50FE96E060EC3
:10CAA000EA221200F86E0800F550E66EE66A1200FF
:10CAB000020EDBCF03F0030EDBCF04F0056A120099
:10CAC0000501770EFD6FFA0EFE6F000E120098EC56
:10CAD000A8F00FD906011200DBCFDEFFDBCFDDFFB0
:10CAE0001200F90EDBCFE6FFFA0EDBCFE6FF1200F5
:10CAF000D950F90F51EF66F0FD0EDBCFE6FFFE0EC9
:10CB0000DBCFE6FF1200DECFE6FFDDCFE6FF12004F
:10CB10000DD9BAEC74F0D1D8C4DE010E120092EC3B
:10CB20005BF0E552E552F90EF3CFDBFFFA0EF4CFDE
:10CB3000DBFF1200E66E98ECA8F079EF66F0F3CF19
:10CB4000DEFFF4CFDDFF1200A3DE0DEF65F08ADE1D
:10CB5000050112009DDE020EE1261200010EE76EB5
:10CB6000CADE1FEF65F094DEE4EF64F0ECDE010E48
:10CB700094D6DCD8C2EF74F07FDE93DE41EC5AF03D
:10CB8000050EF6DE020EE15C1200BCD8EECFE6FF29
:10CB9000EFCFE6FF1200E552F3CF00F0F4CF01F043
:10CBA000F3CFE6FFF4CFE6FF1200010EDBCFE6FF86
:10CBB000020EDBCFE6FF12008CEC74F0006E050E67
:10CBC000E15E00501200FB0EDBCFE6FFFC0EDBCF78
:10CBD000E6FF1200DECFE9FFDDCFEAFF12008BDEB9
:10CBE000EF502D08120050DE470EE66EF90EE66E8D
:10CBF000000E40EF64F056DFE70EE66EF70EE66ECD
:10CC0000000E5CEF64F03CDE4CDE010E12004DECD9
:10CC10003FF0E552E5521200CB0EFD6FF90EFE6FAC
:10CC2000000EA3EF64F0E0DEDECF03F0DDCF04F012
:10CC3000056A120001C0E6FF02C0E6FF03C0E6FF7E
:10CC400012007F0E0501C85D12005CDE2008120094
:10CC5000FD0EDBCF00F0FE0EDBCF01F01200BAECD0
:10CC600074F0026E070EE15E02501200050EF3CF63
:10CC7000DBFF060EF4CFDBFF120065DE41EF5AF05A
:10CC800000C0E6FF01C0E6FF120002DE030EE1264F
:10CC90001200FEDD0AEF65F0000EE66E060EE66E8F
:10CCA0001200E96EFF0EDA20EA6EEE50ED1012006F
:10CCB0003AD8C2EC74F078EF64F0006E070EE15ED3
:10CCC00000501200DE523BDFDD521200C8EC75F05E
:10CCD000046E0B0EE15E04509FEF65F049DE32EF0B
:10CCE00064F0FFDE8FEF65F01ED82DEC75F078EF65
:10CCF00064F0E552E552E55212002CDF010EE66EBB
:10CD0000B3EF64F0FA0EDBCFE9FFFB0EDBCFEAFFF7
:10CD10001200FC0EDBCFE6FFFD0EDBCFE6FF1200BC
:10CD200027DEA7EF65F0E66E83EF65F0E66E4CEF69
:02CD300066F0AB
:0ECD3200B9EC70F0080EE126E00E6214DF6E20
:10CD40000F0E65140801E76F66CFE8F867CFE9F8C2
:10CD500068CFEAF869CFEBF86ACFECF86BCFEDF863
:10CD60006CCFEEF86DCFEFF8609EDF5001E0D4D2CB
:10CD70000801E851A60A01E1C8D2030A01E19CD2E8
:10CD8000010A01E18FD2070A01E182D23D0A01E1E5
:10CD90005ED2080A01E1E5D1030A01E1A6D1060A43
:10CDA00001E120D11A0A01E1FAD0010A01E1E8D03B
:10CDB0000D0A01E1B4D0010A01E191D0070A6FE048
:10CDC000010A67E0030A45E0010A18E0860A01E06B
:10CDD000B0D21B0EE95D03E1ECC8DDF90BD01A0EF1
:10CDE000E95D01E0A6D2EC51000EF350ED250901FA
:10CDF000DE6FDF6B0901010EE56F9BD2E9C8A0F978
:10CE0000EBC801F0006AEA5109010024A16F000E8D
:10CE10000120A26FEFC801F0006A0801EE5109017C
:10CE20000024A36F000E0120A46F0901700ED880AA
:10CE3000A155170EA25502E2A16BA26B0901700E5B
:10CE4000D880A355170EA45501E373D2A36BA46B2E
:10CE500070D29BEC70F003E0C1EC70F0FDE130ECBF
:10CE600072F003E0C8EC70F0FDE17DEC70F003E0DF
:10CE700050EC71F0FDE100500C240901A56F015048
:10CE80000D20A66F02500E20A76F03500F20A86F31
:10CE900050D2E9C8ADF90901780EE16F4AD29BEC96
:10CEA00070F003E0C1EC70F0FDE130EC72F003E0F3
:10CEB000C8EC70F0FDE17DEC70F003E050EC71F037
:10CEC000FDE100500C240901D16F01500D20D26FFB
:10CED00002500E20D36F03500F20D46F2AD29BEC48
:10CEE00070F003E0C1EC70F0FDE130EC72F003E0B3
:10CEF000C8EC70F0FDE17DEC70F003E050EC71F0F7
:10CF0000FDE100500C240901D56F01500D20D66FB2
:10CF100002500E20D76F03500F20D86F0AD2E9C8F5
:10CF2000E0F90901E05129E0EBC801F0006A0801CD
:10CF3000EA5109010024D96F000E0120DA6F680E52
:10CF4000D91905E1010EDA1902E1D96BDA6BF00E9D
:10CF50000801ED1504E00901DB6BDC6B0AD0EDC8BC
:10CF600001F0006AEC5109010024DB6F000E012082
:10CF7000DC6F0901780EE36FDCD10901E36BD9D1D5
:10CF8000E9C890F9EEC891F9EBC801F0006AEA51DE
:10CF900009010024926F000E0120936FCAD14D0E3B
:10CFA0000701CB5D03E1E9C89FF910D0E9C826F07D
:10CFB000276A286A296A490E2B6E060EC9EC71F0A1
:10CFC0001DEC72F053ECB2F026C09FF9EBC801F0F3
:10CFD000006A0801EA51090100248E6F000E012049
:10CFE0008F6FA7D1010EE9C8DBFFEBC803F0026A1F
:10CFF000EA5100010224006E000E0320016E8BEC4A
:10D0000071F0EFC800F0016A026A036A180E1F0B84
:10D0100007E0D8900036013602360336E806F9E11B
:10D02000EEC804F0056A066A076A100E1F0B03E0DB
:10D03000C1EC70F0FDE10EEC72F0080E1F0B03E086
:10D04000C8EC70F0FDE1EFEC71F0ECC80CF00D6A8B
:10D050000E6A0F6A0C5000260D5001220E5002225B
:10D060000F50032292EC71F0060E02C0DBFF070E98
:10D0700003C0DBFFD950020FE96EDACFEAFFFF0EE3
:10D08000EE1802E1FF0EED1801E153D1010EDB5065
:10D0900014080FE1D950020FE96EDACFEAFF190E3A
:10D0A000EE1807E1ED5005E17BEC71F099EC71F0C1
:10D0B00003D0010EDBA014D0D950040FE96EDACFF3
:10D0C000EAFFEECFE6FFEECFE6FFEECFE6FFEFCFD3
:10D0D000E6FF020EDBCFE6FF030EDBCFE6FF02D05A
:10D0E0007BEC71F099EC71F024D1090194510801A5
:10D0F000E95D0EE009019451020803E20F0E945D10
:10D1000007E1040E0801E95D03E0040E76EC70F01F
:10D11000090194510801E95D05E1090195510801F2
:10D12000EA5D09E0020E76EC70F00801E90503E122
:10D130000901020E096FE9C894F9EAC895F90601D8
:10D14000F3A104D00F0E0801EC1504D00801ED394D
:10D150000F0B0F0B0901966FEBC897F9EFC898F901
:10D16000E8D00F0E0901945D02E10801E989080188
:10D17000E9510901995D0FE10801EA5109019A5D40
:10D180000AE10801EB5109019B5D05E10801EC5141
:10D1900009019C5D03E0010E76EC70F0800E090140
:10D1A0009A150AE1800E0801EA1506E0100EEA154C
:10D1B00003E0100E76EC70F0020E09019C1507E1F9
:10D1C000020E0801EC1503E0200E76EC70F0E9C8C1
:10D1D00099F9EAC89AF9EBC89BF9ECC89CF9C0EC3C
:10D1E00071F01EE10901A951AA11AB11AC1118E1AE
:10D1F0000901A551A611A711A81112E00901020EFB
:10D20000096FA5C9A9F9A6C9AAF9A7C9ABF9A8C9FF
:10D21000ACF90901A907000EAA5BAB5BAC5B13D0AC
:10D22000C0EC71F001E185D00901A951AA11AB113F
:10D23000AC1101E17ED00901020E096F0901A96B51
:10D24000AA6BAB6BAC6B010E76EC70F072D009017F
:10D25000090502E1030E096F0801EA51640D33EC80
:10D2600072F0800E0026000E0122080E0F0B05E062
:10D27000D89001320032E806FBE10801EB51640D61
:10D28000F35000240901F56FF4500120F66F51D0DE
:10D29000E9C8C0F9EAC8C1F9EEC8C2F90901780EB7
:10D2A000E26F47D0010EDB6A83EC71F042E224ECBE
:10D2B00071F030EC71F0F8D7010EDB6A83EC71F09D
:10D2C00006E224EC71F0070F30EC71F0F7D7410E55
:10D2D0000801EB5D03E0420EEB5D03E10601320E57
:10D2E00002D00601310ECA6F380E0801EB5D02E173
:10D2F0000601F381330E0801E95D03E10601530ED7
:10D3000002D006014E0ECB6F14D0E9C8BCF9EAC8B2
:10D31000BDF9EBC8BEF90DD00801E8510E0A09E1CC
:10D32000E95109019E5D03E0010E76EC70F0E9C859
:10D330009EF9010E006E080EE15C02E2E16AE55220
:10D34000E16E0050B5EF70F0B9EC70F0E6520F0EE0
:10D350000F0155150801E76F56CFE8F857CFE9F8E8
:10D3600058CFEAF859CFEBF85ACFECF85BCFEDF88D
:10D370005CCFEEF85DCFEFF850CFDFFF0F01509F8D
:10D38000070EDF1404083AE1020E0801E85D01E02F
:10D390008ED00601E551000801E389D0C0EC71F0A0
:10D3A00001E185D00801EA5109019F5D01E17FD0CB
:10D3B0000601F451000801E37AD0E8C800F9E9C891
:10D3C00001F99FC902F9F00E0801EB150901036F7D
:10D3D000ECC804F9EDC805F9EEC806F9EFC807F97D
:10D3E0000F0140B7FDD786EC70F0E5C608F90901DA
:10D3F00008510A085CE20A0E086F59D0070EDF14C4
:10D40000020821E10801EB51000804E2EAC8C7F96B
:10D41000EBC8C3F9EF51000804E2EEC8C8F9EFC841
:10D42000C4F9E951000804E2E8C8C9F9E9C8C5F936
:10D43000ED51000804E2ECC8CAF9EDC8C6F90901CB
:10D44000780EE46F34D00801E851FA0A30E1EBC8F5
:10D4500000F0016A026A036AECC804F0056A066A11
:10D46000076A080E1F0B03E0C1EC70F0FDE10EEC43
:10D4700072F0100E1F0B03E0C8EC70F0FDE10050DD
:10D4800008240901CD6F01500920CE6F02500A20F7
:10D49000CF6F03500B20D06FEFC801F0006A080176
:10D4A000EE5109010024CB6F000E0120CC6F010E5C
:10D4B000E552B5EF70F00901085102E1E5C608F93F
:10D4C00008510A0802E20A0E086F000C090109510E
:10D4D00001082AE20601F45103E10901096B24D095
:10D4E000020E0901095D0EE1010E096F0F0140B73F
:10D4F000FDD738EC72F0D00E476F070E486F63EC23
:10D5000071F012D0030E095D0FE1096B0F0140B7F6
:10D51000FDD738EC72F0476B486B63EC71F084EC2C
:10D520006FF0020E76EC70F00901085101E1000C79
:10D53000020E005D15E10601E551000811E2C0ECA4
:10D5400071F00EE00601F45100080AE2010EE66EE9
:10D55000C1ECB2F0E5520F0140B7FDD786EC70F098
:10D5600009010807000C0F0140B7FDD770EC70F0FF
:10D570000A0E466F010E456F080E406F40B7FED78A
:10D5800012000F0140B7FDD738EC72F02C0E476F38
:10D59000010E486F496B4A6B090E4B6F100E4C6FB2
:10D5A0003CEC72F040B7FED71200E8EC71F00F01CE
:10D5B00040B7FDD7EBEC71F0190E5DEC70F040B7A1
:10D5C000FED7B5EF70F0E8EC71F00F0140B7FDD772
:10D5D000EBEC71F0020E5DEC70F040B7FED7B5EFEA
:10D5E00070F0E8EC71F00F0140B7FDD7EBEC71F093
:10D5F000030E5DEC70F040B7FED7B5EF70F0B9ECFC
:10D6000070F0040EE126D3EC71F0F3EC92F0E552E9
:10D61000E55226C0DEFF27C0DEFF28C0DEFF29C09E
:10D62000DDFFDD52DD52FE0EDB50020803E1C0ECEF
:10D6300071F057E10F0140B7FDD770EC70F00B0EA1
:10D64000466FFE0EDBCF47FF486B496BA8EC70F0CE
:10D6500000504A6FA8EC70F0080EA0EC71F0FDE1EC
:10D6600000500F014B6FA8EC70F0100EA0EC71F0A1
:10D67000FDE100500F014C6FD3EC71F040EC9FF0D6
:10D68000A7EC71F0040ED89000360136E804FBE1F7
:10D69000026A036A180E086ED9CFE9FFDACFEAFFF3
:10D6A000E8501F0BEECF04F0EECF05F0EECF06F002
:10D6B000EECF07F007E0D890073206320532043289
:10D6C000E806F9E10F0E0416056A066A076A67ECB8
:10D6D00070F000C04DFF0F01080E456F406F40B75E
:10D6E000FED7040EE15C02E2E16AE552E16EB5EFBD
:10D6F00070F0E8EC71F00F0140B7FDD7EBEC71F082
:10D700001B0E5DEC70F040B7FED7FE0EDB041BE194
:10D71000EBEC71F01A0E476F486B496B07EC71F038
:10D7200001C000F0016A00504A6FFF0EE76E07EC7F
:10D7300071F0E7500016016A00C04BFF4C6B3CECE7
:10D7400072F040B7FED7B5EF70F0E8EC71F00F0162
:10D7500040B7FDD770EC70F0090E466F476BFE0EB8
:10D76000DBCF48FF030E456F080E406F40B7FED772
:10D77000B5EF70F0B9EC70F0030EE126020EDB6A33
:10D78000FC0EDBCF28F0FD0EDBCF29F0180E281899
:10D7900001E1295001E120D1170E281801E129509B
:10D7A00001E1FDD0160E281801E1295001E1F0D069
:10D7B000150E281801E1295001E1E3D0140E2818B4
:10D7C00001E1295001E1D6D0130E281801E12950BA
:10D7D00001E1CBD0120E281801E1295001E1C0D09F
:10D7E000110E281801E1295001E186D0100E2818E9
:10D7F00001E1295058E00F0E281801E129504CE0B2
:10D800000C0E281801E1295033E00B0E281801E115
:10D81000295015E00A0E281801E1295002E0000EF7
:10D82000FCD00601F45101E1DAD0FA0EDBCFE6FFBD
:10D83000FB0EDBCFE6FFDAEC71F0B7DED8D00601E5
:10D84000F45101E1CCD0040E090199150BE0070E4B
:10D850000901955D07E0010EE66EC3DEE5520501A4
:10D86000FC6BC6D0F30EE66E610EE66E010EC5D0FF
:10D870000601F45101E1B3D0090199A907D0E66A84
:10D88000B0DEE55205011E0EFC6FB2D0190EE66E39
:10D89000620EE66E010EB1D00601F45101E19FD097
:10D8A000C4EC71F025D00601F45101E198D0A6CA6C
:10D8B000DEFFA7CADDFFE0EC70F009E0E0EC70F0FD
:10D8C0002C0805E0DF2A010EF6E3DB2AF4D7E0ECB2
:10D8D00070F02C083FE1ABEC71F001E3DB2AEF6A5A
:10D8E000BEEC70F062DEE552DECFE6FFDDCFE6FF94
:10D8F000DAEC71F068DE7BD00601F45170E0A6CA64
:10D90000DEFFA7CADDFFE0EC70F009E0E0EC70F0AC
:10D910002C0805E0DF2A010EF6E3DB2AF4D7E0EC61
:10D9200070F02C0817E1ABEC71F001E3DB2AEF6A31
:10D93000DECFE6FFDDCFE6FF7EEC92F0A7EC71F0E4
:10D94000F3CFE6FFF4CFE6FFBEEC70F0D2DEE55297
:10D95000E5524DD0AD0EE66E610EE66E010E4DD075
:10D960000601F4513CE0FFDD03D00601F45137E03D
:10D9700008DE3ED00601F45115E0C4EC71F0020E51
:10D980001AD00601F4510EE0C4EC71F0E66A14D02E
:10D990000601F45107E0C4EC71F0030E0CD006014F
:10D9A000F45106E1BF0EE66E610EE66E010E0DD07B
:10D9B000C4EC71F0010EE66E22DEE552E552E5524E
:10D9C000AA0EE66E610EE66E010E59DB010EF36ED5
:10D9D000020EF3CFDBFF12D00601F45106E1BF0EB9
:10D9E000E66E610EE66E010E08D0C8DBAEDEE552D3
:10D9F000AA0EE66E610EE66E010E41DBFE0EDB50F6
:10DA00000BE03FEC2EF0020EE66E62EC72F0E55297
:10DA1000E66A7CEC31F0E552010E006E030EE15C2B
:10DA200002E2E16AE552E16E00509FD3A2DB180EDC
:10DA3000E12624EC72F027AE02D028682968C70ED0
:10DA40000AEC72F0840E2626120EA9DB0C0E26C0FC
:10DA5000DBFF0D0E27C0DBFF24EC72F027AE02D0F7
:10DA600028682968A60E0AEC72F0EA0E2626070E30
:10DA700096DB0E0E26C0DBFF0F0E27C0DBFF0C0E61
:10DA8000DBCF02F00D0EDBCF03F00E0EDB50025C9D
:10DA9000006E0F0EDB500358016E010E0026000EC3
:10DAA0000122020E2D6E2E6A00C028F001C029F05E
:10DAB000CEEC8CF0100E28C0DBFF110E29C0DBFF6E
:10DAC000FE0EDB50030A20E0070A12E0040A03E01E
:10DAD000F36AF46A12D292DB09E1FF0EED1806E157
:10DAE0000E0EDBCF28F00F0E6AEC71F06FDB06D064
:10DAF0006DDB84DB03E1FF0EED180BE015EC72F03B
:10DB0000FA0FF8EC71F00AD079DB08E1FF0EED189E
:10DB100005E10C0EDBCF28F00D0EDCDBF60EDBCFC3
:10DB200000F0F70EDBCF01F0013418E200500008DE
:10DB3000000E015413E2E1EC71F0FC0EDBCF04F0B7
:10DB4000FD0EDBCF05F005500318E8AE02D003341C
:10DB500004D00250045C0350055803E3F368F468F2
:10DB6000CCD1F50EDBCF00F03C0EE76E0018E8AE2E
:10DB700002D0003403D0E750D880005405E23C0EB8
:10DB8000F36EF50EF3CFDBFFFC0EDBCF02F0FD0EE4
:10DB900026DBFC0E00C0DBFFFD0E01C0DBFFFA0E32
:10DBA000DBCF02F0FB0E1BDBFA0E00C0DBFFFB0E2F
:10DBB00001C0DBFF7CDB01340CE20050F408000EF6
:10DBC000015407E2F40EF36EFA0EF3CFDBFFFB0E07
:10DBD000DB6AC8DBD890055004E6FC0E045C080E36
:10DBE000055807E3200E006E010E016E026A036AFB
:10DBF0001BD0E90E066E020E076E086A096A2AEC4F
:10DC000072F027AE02D028682968C70E0AEC72F0BD
:10DC1000E1DA065C006E27500758016E285008585C
:10DC2000026E29500958036E00C0DEFF01C0DDFFFF
:10DC3000040E046E0E0E056E066A076A2AEC72F078
:10DC400027AE02D028682968FA0EE4DBC3DA045C48
:10DC5000006E27500558016E28500658026E295054
:10DC60000758036E58DB020EDBCF00F0030EDBCF4C
:10DC700001F00001800E011404E0020EDB6A030EC5
:10DC8000DB6AF50EDBCF04F0056A04BE0568020E00
:10DC9000DBCF28F0030E27DB26C002F027C003F0FD
:10DCA000E80E2D6E030E2E6E26C028F027C029F038
:10DCB000CEEC8CF0DE502824006EDD502920016E61
:10DCC00031DB50DB066A076A05AE02D006680768DA
:10DCD000040EDBCF00F0050EDBCF01F0026A036A11
:10DCE00001AE02D002680368100E2B6E0E0E2C6E71
:10DCF000CCDABEECB1F022C000F023C001F024C0A9
:10DD000002F025C003F07DDBB6DA060E26C0DBFF8D
:10DD1000070E27C0DBFF080EDB6A090EDB6A0A0E5E
:10DD2000DB6A0B0EDB6A73DAD890015004E6C80E8A
:10DD3000005C000E015832E244DBD890035004E648
:10DD4000C80E025C000E035802E2B1DA03D0C80E1E
:10DD5000006E016A120E00C0DBFF130E01C0DBFF74
:10DD6000120EDBCF06F0130EDBCF07F0FC0EDB50FC
:10DD7000065C046EFD0EDB500758056E060EDBCF09
:10DD800028F0070EB0DA26C000F027C001F0026AC2
:10DD9000036A01AE02D00268036840DA88DA01340F
:10DDA00001E38FD00050C808000E015401E389D070
:10DDB000FC0EDBCF02F0FD0EDBCF03F0033407E2F5
:10DDC0000250C808000E035402E221DA03D0C80E44
:10DDD000006E016A140E00C0DBFF150E01C0DBFFF0
:10DDE000140EDBCF00F0150EDBCF01F0EADA0150A4
:10DDF0000318E8AE02D0033404D00250005C035094
:10DE000001585FE2250E086E010E096E0A6A0B6A60
:10DE1000140EDBCF26F0150E51DA27AE02D028689B
:10DE20002968990E2B6E040EB4DAD4D9085C046EFE
:10DE300027500958056E28500A58066E29500B586D
:10DE4000076E100E006E0E0E016E026A036A00C0AD
:10DE500026F0276E02C028F003C029F00CDA160E57
:10DE600026C0DBFF170E27C0DBFF83DA060EDBCFF1
:10DE700002F0070EDBCF03F001500318E8AE02D02A
:10DE8000033404D00250005C035001580CE2060E2B
:10DE9000DBCF28F0070EDBCF29F0160E28C0DBFF02
:10DEA000170E29C0DBFF65DA026A036A01AE02D0F1
:10DEB00002680368B3D9140EDB2A150E91E3DB2A3E
:10DEC0008FD7080EDBCF00F0090EDBCF01F00A0E72
:10DED000DBCF02F00B0EDBCF03F01E0E0026000E90
:10DEE0000122022203223C0E2B6E2C6ACED9F4ECC6
:10DEF0008CF026C0F3FF27C0F4FF180EE15C02E2AD
:10DF0000E16AE552E16E31D1090199A93ED0ADC96E
:10DF1000E6FF09019051026E036A8EC928F08FC98D
:10DF200029F090C92DF003C02EF055EC8DF026C0DD
:10DF300000F027C001F026C0E6FF27C0E6FFF5C9C4
:10DF400004F0F6C905F0640E2D6E2E6AF5C928F0AE
:10DF5000F6C929F0ABECB2F028C004F029C005F0F6
:10DF600028C0E6FF29C0E6FFE668E668A1C9E6FF2B
:10DF7000A2C9E6FF96C9E6FF59DD066E0A0EE15E0C
:10DF80000650F3CFF7F9F4CFF8F9000CD9CFE6FF3C
:10DF9000020EE1260601540EC86F520EC96FCA6BFD
:10DFA000CB6BCC6B900E6F6E6EAEFED7606A0F01BE
:10DFB000A00E196F1869016B200E006F506BE00EF8
:10DFC0001D6F1C69800E096F680E086F400E0D6F83
:10DFD000800E0C6F116B106F706AD20E716E020E94
:10DFE000726E200E736E0601F451000802E26F6A31
:10DFF00002D0600E6F6E0901006B086B096B0501A2
:10E00000EE850701120ECF6F660ED06F010ED16F35
:10E010000701320ED56FCD0ED66F000ED76F0701F8
:10E02000480ED86FD30ED96F000EDA6F0701B60E07
:10E03000ED6FD40EEE6F000EEF6F0701080EE16F6B
:10E04000DF0EE26F000EE36F0701CC0EF06FD40E0F
:10E05000F16F000EF26F0801740EF06FD70EF16FC2
:10E06000000EF26F020EE15C02E2E16AE552E16E3F
:10E070007CD02D6A2E6ABEECB1F001EF72F0E66E34
:10E0800092D9A30EE66E610EE66E010EE66E000EEC
:10E09000E66E060EE66EC2EC74F0026E070EE15EEE
:10E0A0000250E1D9F3CFE6FFF4CFE6FF8CEC74F039
:10E0B000036E050EE15E03501200476F486B496B1B
:10E0C000FE0EDBCF4AFF4B6B4C6B3CEF72F0045003
:10E0D000002605500122065002220750032212009A
:10E0E000406B400E426F200E416F1200E66EE66AF2
:10E0F000E3EC3FF0E552E552120071D9EFC80CF0A5
:10E100000D6A0E6A0F6A180E1F0B1200406B426BED
:10E11000800E416F00C946FF01C947FF02C948FF91
:10E1200003C949FF04C94AFF05C94BFF06C94CFF93
:10E1300007C94DFFA3D1ECC800F0016A026A036A67
:10E14000EDC804F0056A066A076A080E1F0B120084
:10E15000D9CFE9FFDACFEAFFEECF00F0EECF01F042
:10E16000EECF02F0EFCF03F01200E552E7CFD9FF78
:10E170001200D9CFE6FFE1CFD9FF120005D9DAEFBF
:10E1800071F0D8900436053606360736E8061200D8
:10E19000D890083609360A360B36E80612002722D0
:10E1A000000E282229224B0E2626000E2722282286
:10E1B0002922960E2B6E2C6A2D6A2E6AF4EF8CF0B3
:10E1C000DECFE9FFDDCFEAFFEF5012002ED9FC0FC2
:10E1D000F8EF71F032D9F4EC8CF026501200DBCF5E
:10E1E00003F00C0EDB50025C006E0D0EDB5003588A
:10E1F000016EF40E0026000E01221200D950FA0F13
:10E20000E96EFF0EDA20EA6EFF0EEE181200FC0E29
:10E21000DBCF00F0FD0EDBCF01F01200D950080F6C
:10E22000E96EDACFEAFF0050EE260150EE220250EE
:10E23000EE220350EE221200EEC808F0096A0A6AC4
:10E240000B6A100E1F0B1200010EDB28EA6AE80FA2
:10E25000E96E080EEA22EF50E66E010EDB50120066
:10E26000EA6AAE0FE96E090EEA22E552E750EF6E58
:10E27000010EDB2A120004C02BF005C02CF006C0F2
:10E280002DF007C02EF0F4EF8CF02D6A2E6A00C03E
:10E2900026F001C027F002C028F003C029F01200C8
:10E2A000D8900C360D360E360F36E8061200FA0EF0
:10E2B000DBCF00F0FB0EDBCF01F01200DBCF27F04D
:10E2C000286A296A1200496B4A6B4B6B4C6B400EF3
:10E2D0004D6FD4D0DBCF29F0FA0E28C0DBFFFB0E48
:10E2E00029C0DBFF1200DBCF29F004C02DF005C0F0
:10E2F0002EF028EF8DF0E66AE66AE66AE66A000E1E
:10E30000E66EE66A1200070EF36E010EDBCFF4FF35
:10E31000F350F45C1200020E00C0DBFF030E01C0DC
:10E32000DBFF1200040E00C0DBFF050E01C0DBFFA7
:10E330001200A8EC3FF0006E060EE15E00501200E5
:10E34000D8900332023201320032E8061200E55260
:10E35000E55233EF72F0DFCFE9FFDF2A010EDBCFAA
:10E36000EAFF1200F60EDBCF04F0F70EDBCF05F06C
:10E370001200160EDBCF00F0170EDBCF01F01200FB
:10E38000800E090199151200A6CAE6FFA7CAE6FF8A
:10E3900012002C6E6EDEF40E2626010E2722000ED1
:10E3A000282229221200FC0EDBCFE6FFFD0EDBCF78
:10E3B000E6FF12007EEC92F0E552E552F350E66E75
:10E3C0001200FA0EDBCF02F0FB0EDBCF03F01200DF
:10E3D000D0DEB3EF6AF084DE050E466F12000850FF
:10E3E0000026095001220A5002220B50032212007B
:10E3F000E96EFF0EDA20EA6E0050EE260150ED22A3
:10E40000120022C026F023C027F024C028F025C027
:10E4100029F012002B6E2C6A39EF70F058DEEDC82F
:10E4200008F0096A0A6A0B6A1200100EDBCF00F0CE
:10E43000110EDBCF01F0D9501200E80E2B6E030E47
:10E440002C6E2D6A2E6A1200F80EDBCF26F0F90E24
:10E450005EEF71F0F60EDBCF26F0F70E5EEF71F097
:10E4600036DE1CEF71F0F3CF00F0F4CF01F01200B4
:10E4700037DE060E466F12004D6B00D0080E456F5A
:04E48000406F1200D7
:0CE48400FF00120079EC77F0D1EC78F08A
:10E49000060EDF5C05E29EA2FED79E92DF2AF8D729
:10E4A000E5526EEF77F079EC77F0D1EC78F07A0EF8
:10E4B000DF5C05E29EA2FED79E92DF2AF8D7E552E6
:10E4C0006EEF77F079EC77F0FE0EDB50000804E297
:10E4D000EADFFE0EDB06F8D76EEF77F0D9CFE6FF66
:10E4E0006EEF77F0D9CFE6FF6EEF77F081B005D011
:10E4F0008180050EE66EE6DFE5528190140EE66E31
:10E50000E1DFE5528180120079EC77F00E0EC1EC6C
:10E5100078F0F3EC92F049EC78F02E0EE66EF0EC29
:10E5200078F0D2EC9EF0E552E552E5520C0EF3CFB6
:10E53000DBFF0D0EF4CFDBFFF3CF00F0F4CF01F0E3
:10E54000F350F41001E1C2D0040EDB6A050EDB6A61
:10E55000060EDB6A070EDB6A010EF36E080EF3CFC0
:10E56000DBFF090EDB6A0A0EDB6A0B0EDB6A0C0EA0
:10E57000DB2ADBCFE9FF0D0E01E3DB2ADBCFEAFF6D
:10E58000EF504DE076EC78F0060EDBCF02F0070E90
:10E59000DBCF03F00A0E0EEC79F0BEECB1F005EC27
:10E5A00079F00C0EDBCFE9FF0D0EDBCFEAFFEF5069
:10E5B000D00F046E056A066A076AE8500026055007
:10E5C00001220650022207500322040E00C0DBFF86
:10E5D000050E01C0DBFF060E02C0DBFF070E03C005
:10E5E000DBFF080EDBCF26F0090EDBCF27F00A0E8B
:10E5F000DBCF28F00B0EDBCF29F00A0E7CEC79F094
:10E60000BEECB1F0080E22C0DBFF090E23C0DBFF19
:10E610000A0E24C0DBFF0B0E25C0DBFFA8D722ECBF
:10E6200079F0EECF08F0EECF09F0EECF0AF0EFCFA1
:10E630000BF0E6EC77F0040EDBCF14F0050EDBCF29
:10E6400015F0060EDBCF16F0070EDBCF17F014C067
:10E6500026F015C027F016C028F017C029F044ECAA
:10E660008BF027C010F028C011F029C012F02AC08A
:10E6700013F0080EDBCF1CF0090EDBCF1DF00A0EE5
:10E68000DBCF1EF00B0EDBCF1FF01CC026F01DC031
:10E6900027F01EC028F01FC029F044EC8BF027C0E3
:10E6A00018F028C019F029C01AF02AC01BF0D4ECC9
:10E6B00077F094EC78F0F4EC8BF09DEC78F0D4ECFF
:10E6C00077F03CEC78F05EEC8BF004D0B4EC77F0B3
:10E6D0005DEC78F0DDEC77F027C026F028C027F05D
:10E6E00029C028F02AC029F00E0EE15C02E2E16A9E
:10E6F000E552E16EF3D379EC77F0080EC1EC78F0D7
:10E7000003DF49EC78F022EC79F0EECF00F0EECFA9
:10E7100001F0EECF02F0EFCF03F02C6A2D6AC80EA5
:10E720002E6E420E2F6EA6EC78F0F4EC8BF012EC0D
:10E730008EF0040E26C0DBFF050E27C0DBFF060EA1
:10E7400028C0DBFF070E29C0DBFF42EC79F0060E84
:10E75000DBCF06F0070EDBCF07F05DEC78F0DDECE9
:10E7600077F022EC79F0EECF10F0EECF11F0EECF93
:10E7700012F0EFCF13F0040EDBCF18F0050EDBCF55
:10E7800019F0060EDBCF1AF0070EDBCF1BF0640E7C
:10E790007CEC79F018C026F019C027F01AC028F0D8
:10E7A0001BC029F0BEECB1F022C018F023C019F054
:10E7B00024C01AF025C01BF022C026F023C027F089
:10E7C00024C028F025C029F044EC8BF027C014F0B9
:10E7D00028C015F029C016F02AC017F0E5DB94EC2C
:10E7E00078F05DEC8BF09DEC78F02C6A2D6A700E61
:10E7F0002E6E420E2F6EF4EC8BF027C008F028C06E
:10E8000009F029C00AF02AC00BF0CEDBA6EC78F0A4
:10E810005EEC8BF060EC78F0A7DBD8EC78F03CECA9
:10E8200078F047EC8CF0C9DB2C6A2D6A2E6A450E15
:10E830002F6E47EC8CF012EC8EF0080EE15C02E2D9
:10E84000E16AE552E16E4AD354DB040EE126DE684C
:10E85000DD68FB0EDBCF00F0FC0EDBCF01F00134F6
:10E8600038E200500008000E015433E2E8EC78F082
:10E8700001E3DB2AEF50DF1AFB0EDB06FC0E01E2A0
:10E88000DB06020EDB6A030EDB6A020EDBCF00F052
:10E89000030EDBCF01F0D890015004E6080E005CB7
:10E8A000000E0158D6E2DF50010B07E0C4EC78F00F
:10E8B000010E001AA00E011A02D0C4EC78F000C0BC
:10E8C000DEFF01C0DDFF020EDB2A030EDEE3DB2AE2
:10E8D000DCD762EC79F000C0F3FF01C0F4FF040E56
:10E8E000E15C02E2E16AE552E16EF8D202DBDFECC4
:10E8F00078F0EE50ED100FE039EC79F00CE039ECE7
:10E9000079F00D0803E1EEDA0A0EEF6E90EC78F084
:10E91000EEE3DB2AECD7E2D2ECDAD950FA0F77EC4F
:10E9200079F0EFCFF6FFEE2AEFCFF7FF000EEE22E1
:10E93000EFCFF8FFEE220800F55049EC79F004E043
:10E94000EFDBEBE3DB2AE9D7B7DAC8D2D2DAFB0E8A
:10E95000DBCFE9FFDB2AFC0EDBCFEAFF01E3DB2A9A
:10E96000EF5049EC79F004E0DBDBF1E3DB2AEFD791
:10E97000A3DAB4D218EC79F001E089DA4FEC79F03F
:10E9800095DBACD218EC79F001E081DA93DB9EECF8
:10E9900093F067EC79F039EC79F004E0C1DBFBE34C
:10E9A000DB2AF9D789DA9AD218EC79F001E06FDA2C
:10E9B000BEDA38EC94F0E0DB39EC79F004E0B0DB5F
:10E9C000FBE3DB2AF9D778DA89D218EC79F001E099
:10E9D0005EDAADDA2BEC95F0CFDB39EC79F004E0C0
:10E9E0009FDBFBE3DB2AF9D767DA78D282DAE652DB
:10E9F00084DB040EEE26000EED22FB0EDBCFE9FFDA
:10EA0000FC0EDBCFEAFFEF6A040EDF6EDF5023E07F
:10EA1000C0DBE76EFD0EDBCF03F0FE0EE750031602
:10EA2000046A056AE6DAFB0EDB06DBCFE9FFFC0EC3
:10EA300001E2DB06DBCFEAFFE552E750EF6EBFDB1A
:10EA4000040E0F0B06E0EC52D890ED32EF32E806E0
:10EA5000FAE1DF06DBD7E55241D2EADB01E017DA63
:10EA600029DBC4DF67EC79F039EC79F004E058DB9E
:10EA7000FBE3DB2AF9D720DA31D23BDAE652D95070
:10EA8000F90F77EC79F0080EEE26000EED22F90E64
:10EA9000DBCFE9FFFA0EDBCFEAFFEF6A080EDF6E8D
:10EAA000DF502AE076DB036E046A056A066A25DB1E
:10EAB000EE500316EE500416EE500516EE500616F4
:10EAC00098DAF90EDB06DBCFE9FFFA0E01E2DB068E
:10EAD000DBCFEAFFE552E750EF6E0FDB040EE76E87
:10EAE000D890030EEB32020EEB32010EEB32EF3216
:10EAF000E706F6E1DF06D4D7E552F0D199DB01E075
:10EB0000C6D915DABADF38DBB4DB04E009DBFCE395
:10EB1000DB2AFAD7D1D9E2D1ECD90C0EE126BFD944
:10EB200001E0B5D950DB6DDB92DB2BEC95F024DBFB
:10EB30004ADB40EC9FF0E552E5520B0EF3CFDBFFD2
:10EB4000DB50006E016AF40EDBCF02F0F50EDBCF76
:10EB500003F001500318E8AE02D0033404D0025091
:10EB6000005C0350015809E233DB01E3DB2AF30EBA
:10EB7000DBCFEFFF0B0EDB2AE3D725DB97DA5BDB7E
:10EB80009BD90C0EE15C02E2E16AE552E16EA6D18E
:10EB9000B0D9050EE126010EDE6EDE6ADE6ADD6AA0
:10EBA000DD52DD52F40EDB50E76E040EE7CFDBFFE3
:10EBB000DB50000809E246DB0A0E19DBBEECB1F0BF
:10EBC000CEDA040EDB06F4D7B6D9F4EC8CF022DAF8
:10EBD00083DBEADE086E090ECBDAFADA01E3DB2A20
:10EBE0002E0EEF6E300EE66EF40EDBCFE6FFF50E66
:10EBF000DBCFE6FFA0D92EC0F5FFF4EC8CF0F5AE2C
:10EC000008D0000E226C231E2322241E2422251E3F
:10EC10002522FBDA22C0E6FF23C0E6FF24C0E6FF80
:10EC200025C0E6FF6EDA78DF086E0C0EA1DA44D953
:10EC3000050EE15C02E2E16AE552E16E4FD136DB9E
:10EC400001E025D963DA66D90050011002100310E3
:10EC50000AE1FCD9E8AE02D0053404D00450065CC9
:10EC6000055007584CE3040EDBCF02F0050EDBCF56
:10EC700003F0F40EDB50025C006EF50EDB5003581F
:10EC8000016E030E2D6E2E6A00C028F001C029F01F
:10EC9000CEEC8CF024C000F025C001F024502510EB
:10ECA0000FE1D4D9E8AE02D0053404D00450065C9C
:10ECB0000550075805E28CDA01E3DB2A2C0EEF6ED3
:10ECC00029D90A0EFFD801E3DB2ADFD90A0E16D9AB
:10ECD000040EDB2ADBCF00F0050E01E3DB2ADBCFDD
:10ECE00001F0F40EDB500018AEE1F50EDB50011818
:10ECF000AAE16EDA01E3DB2A2E0EEF6EA4D79BD9D0
:10ED0000AFD90AE23BD901E3DB2AE5D901E2DB0610
:10ED1000060EDBCFEFFFF4D7AFDA02E2E16AE5528D
:10ED2000E16EDCD0E6D8040EE126B9D801E0AFD818
:10ED300068DAD890030EEB50000A08E6000EEE5C8D
:10ED4000000EEE58000EEE58000EEE5816E240DAB5
:10ED500001E3DB2A2D0EEF6EDDD8001E011E021E20
:10ED6000031EF60E00C0DBFFF70E01C0DBFFF80E3E
:10ED700002C0DBFFF90E03C0DBFFF60EDBCF08F0AD
:10ED8000F70EDBCF09F0F80EDBCF0AF0F90EDBCF80
:10ED90000BF01CD92C6A2D6A2E6A450E2F6EF4ECEE
:10EDA0008BF00BD905DAF4EC8BF08AD9060EE66EFF
:10EDB000E66ADAD82C6A240E2D6E740E2E6E490E79
:10EDC0002F6E5AD947EC8CF012EC8EF023D999D9DA
:10EDD000DFDE086E0B0EE15E0850040EE15C02E21D
:10EDE000E16AE552E16E7AD061DA01E050D88ED95D
:10EDF0007DD9D890015004E6030E005C000E015846
:10EE000033E274D901340AE200500008000E0154C4
:10EE100005E2DED901E3DB2A3A0EEF6ED950040F8A
:10EE2000E96EDACFEAFF020EEE1808E1ED5006E1D6
:10EE3000E8D9180EDCD953ECB2F091D96BD80A0E90
:10EE400041D801E3DB2A21D90A0E58D863D8060E2F
:10EE500039D801E3DB2A19D9060E50D8040EDB2A73
:10EE6000050EC6E3DB2AC4D7E6D8FAD80AE286D86C
:10EE700001E3DB2A30D901E2DB06060EDBCFEFFF30
:10EE8000F4D7FAD902E2E16AE552E16E27D024DA3A
:10EE900043DD006E050EE15E00501BEF79F0FA0EC7
:10EEA000DBCF00F0FB0EDBCF01F0FC0EDBCF02F07E
:10EEB0000050011002101200FED900C0F3FF01C083
:10EEC000F4FF1200ABD953ECB2F09FD9300E0026FC
:10EED000000E012202220322E8EF78F0E552E7CF8C
:10EEE000D9FF1200FD0EDBCFE9FFFE0EDBCFEAFFFC
:10EEF0001200D9CFE6FFE1CFD9FF120078D953EC49
:10EF0000B2F029C0EDFF28C0EDFF27C0EDFF26C0FD
:10EF1000EFFF1200F60EDBCF00F0F70EDBCF01F0B3
:10EF2000F80EDBCF02F0F90EDBCF03F0120058D958
:10EF300068D927EF79F0F60EDBCF04F0F70EDBCFC0
:10EF400005F0F80EDBCF06F0F90EDBCF07F088D91D
:10EF5000DFCF2BF0010EDBCF2CF0020EDBCF2DF03C
:10EF6000030EDBCF2EF012006DD9EECF04F0EECF02
:10EF700005F0EECF06F0EFCF07F01200DECFE9FF8D
:10EF8000DDCFEAFF060EEFCFDBFF020EDBCFE9FF9E
:10EF9000030EDBCFEAFFEF50E66EDFCFE9FFDF2A9B
:10EFA000010EDBCFEAFF120027C02CF028C02DF0A5
:10EFB00029C02EF02AC02FF0120027C000F028C070
:10EFC00001F029C002F02AC003F0120008C026F0A8
:10EFD00009C027F00AC028F00BC029F044EC8BF0E0
:10EFE00027C004F028C005F029C006F02AC007F0A9
:10EFF000120000500324F36E01500420F46E0250FE
:10F000000520F86EF4CFF7FFF3CFF6FF0800F550B8
:10F01000E66E120026C000F027C001F028C002F002
:10F0200029C003F026C0E6FF27C0E6FF28C0E6FFA0
:10F0300029C0E6FF12003FD90006000E015A020E59
:10F0400000C0DBFF030E01C0DBFF12001BD9F40E72
:10F05000DBCF06F0F50EDBCF07F0075005181200E6
:10F0600031D9020EDBCF02F0030EDBCF03F00250EA
:10F07000005C03500158120004C027F005C028F0BE
:10F0800006C029F007C02AF0120000C0EFFF01EF10
:10F0900079F0E552E55226C0DEFF27C0DEFF28C02A
:10F0A000DEFF29C0DDFFDD52DD52120099D84EDCB3
:10F0B00067EF79F095D84FEF79F0D2D844EF8BF025
:10F0C00027C0DEFF28C0DEFF29C0DEFF2AC0DDFF2B
:10F0D000DD52DD521200E552E750EF6E020EDBCF3B
:10F0E000E9FFDB06030EDBCFEAFF1200040EDBCFE5
:10F0F00000F0050EDBCF01F01200D950FB0F77EFC7
:10F1000079F0E66AE66AE66AF0EF78F0FD0EDBCFAA
:10F11000DEFFDBCFDDFF040EDB6A050EDB6A1200CB
:10F12000FD0EDB2AFE0E120010C027F011C028F0E1
:10F1300012C029F013C02AF0120027C00CF028C01A
:10F140000DF029C00EF02AC00FF0120000C027F009
:10F1500001C028F002C029F003C02AF0120025C027
:10F16000EDFF24C0EDFF23C0EDFF22C0EFFF120032
:10F17000E15E08501BEF79F0006E060EE15E005074
:10F180001200E126F0EF78F09DD8D89001320032DD
:10F1900012008B0E006EFA0E016E000E026E0F0E44
:10F1A0001200E652DF6A7C0ECA6ECC6ACB6812008F
:10F1B0002C6A2D6A610E2E6E450E2F6E1200D950EC
:10F1C000FD0F77EF79F0D9CFE6FFDACFE6FF120037
:10F1D000FD0EDBCFE9FFDB2AFE0EDBCFEAFF1200DC
:10F1E000FD0EDBCFE6FFFE0EDBCFE6FF120084D87C
:10F1F000EECF26F0EECF27F0EECF28F0EFCF29F0BC
:10F200001200D950F60F77EF79F022C000F023C03A
:10F2100001F024C002F025C003F012006DD800C038
:10F2200026F001C027F002C028F003C029F0120028
:10F2300060DE4FEF77F0FD0EF3CFDBFFFE0EF4CF75
:10F24000DBFF1200D9CFE9FFDACFEAFF1200EECFE1
:10F25000E6FFEECFE6FFEECFE6FFEFCFE6FF1200D0
:10F2600004C026F005C027F006C028F007C029F02A
:10F27000120038DEEF50120035DEEF6A1DDE070E99
:10F28000E15C1200040EDBCF04F0050EDBCF05F0CD
:10F290001200E66E27DEE552E750EF6E1200F80E20
:10F2A000DBCFE6FFF90EDBCFE6FF120022DE070E12
:10F2B000E1264FEF77F0FD0EDBCF00F0FE0EDBCF47
:10F2C00001F01200DECF00F0DDCF01F01200E552B8
:10F2D000E552E552E5521200FA0EDBCFE6FFFB0ED7
:10F2E000DBCFE6FFFC0EDBCFE6FFF0EF78F0E96E58
:10F2F000FF0EDA20EA6E12002B6E2C6A2D6A2E6A3F
:02F300001200F9
:0EF3020053544154002B435553443A002B43BF
:10F3100046554E3A005244590053454E442046410A
:10F32000494C00434F4E4E454354204641494C0002
:10F33000434C4F53454400444154412041434345CD
:10F3400050540053454E44204F4B002B4353513AE9
:10F350000053544154453A2054435020434C4F539A
:10F3600045440053544154453A2054435020434FA0
:10F370004E4E454354494E470053544154453A205C
:10F38000434F4E4E454354204F4B00535441544538
:10F390003A2000434F4E4E454354204F4B003634E5
:10F3A0002C002C00322C002B434C4950002B504495
:10F3B000503A204445414354002B435245473A209C
:10F3C0003000222C2236383637220D0041542B4390
:10F3D000495053544152543D22544350222C220050
:10F3E00041542B43494653520D0041542B4349503D
:10F3F000484541443D310D0041542B434949435256
:10F400000D00222C220041542B435354543D220022
:10F41000220D0041542B434744434F4E543D312C61
:10F42000224950222C22002B43524547002B434FA8
:10F4300050533A002B434D45204552524F520053F2
:10F440004554555000223B2B434F50533F0D004134
:10F45000542B434F50533D312C312C220041542B1F
:10F46000434C504F52543D22544350222C223638A4
:10F470003637220D0041542B434950434C4F5345DE
:10F480000D0041542B434950534855540D00002D55
:10F49000002200495000534D53004D502D30205054
:10F4A0004500562900562C207265663D004D502DB2
:10F4B0003020504131325620424154544552592057
:10F4C0004F4B2028004D502D30205041414C45528B
:10F4D0005421212120313256204241545445525961
:10F4E00020435249544943414C2028002520534F82
:10F4F0004329004D502D30205041414C455254215C
:10F50000212120435249544943414C20534F432029
:10F510004C4556454C20415050524F41434845447C
:10F520002028004D502D302050415472756E6B20B4
:10F53000686173206265656E206F70656E6564201A
:10F540002876616C6574206D6F6465292E004D50BE
:10F550002D3020504156656869636C6520616C618F
:10F56000726D20697320736F756E64696E67210018
:10F570000D204341433A20000D204F444F3A2000D4
:10F580000D204573742E2052616E67653A20000D80
:10F5900020496465616C2052616E67653A200025E0
:10F5A000000D20534F433A20004E6F742063686172
:10F5B0007267696E6700206D696E73000D20526579
:10F5C0006D61696E3A20004100562F000D20004306
:10F5D00068617267696E672053746F70706564004C
:10F5E0004368617267696E672C2048656174696E53
:10F5F0006700507265706172696E6700436861727E
:10F6000067696E6720446F6E650043686172676961
:10F610006E672C20546F7070696E67206F6666008D
:10F620004368617267696E6700506572666F726DDC
:10F63000616E6365202D200052616E6765202D206C
:10F640000053746F72616765202D20005374616EE2
:10F6500064617264202D2000206B6D00206D6900B4
:10F660002C312C496E76616C6964205553534420CB
:10F67000726573756C74002C302C00202D204D5356
:10F68000473A2000534D532046524F4D3A20004DEB
:10F69000502D30205041000D00222C31350D0041FD
:10F6A000542B435553443D312C22004D502D3020D6
:10F6B00063332C302C004D502D302063312C302CF6
:10F6C000004D502D302061004D502D3020004D5008
:10F6D0002D53203020004D502D3020482A2D4F56DC
:10F6E0004D2D446562756743726173682C302C320E
:10F6F0003539323030302C004D502D3020455400FB
:10F700004D502D3020670043312D362C4334302DA1
:10F7100034312C433439004D502D302056004D509B
:10F720002D302044002F56002F002E004D502D303C
:10F73000204600302C302C004D502D302057004DED
:10F74000502D30204C002C706572666F726D616EAA
:10F750006365002C72616E6765002C73746F726153
:10F760006765002C7374616E64617264002C73743D
:10F770006F70706564002C68656174696E67002C39
:10F7800070726570617265002C646F6E65002C7418
:10F790006F706F6666002C6368617267696E6700E0
:10F7A0002C004D502D3020530020004D502D432073
:10F7B0003020004D502D3020454D001A000D0A001C
:10F7C00041542B43495053454E440D002320004DD6
:10F7D000502D302063002000436F6D6D616E6473A7
:10F7E0003A002F56002F002E004F564D53204669E9
:10F7F000726D776172652076657273696F6E3A20FB
:10F8000000340050455200330052414E0031005345
:10F81000544F003000535441000D0A2000466561EA
:10F8200074757265733A002053544B554E46002050
:10F8300053544B46554C002052490020544F002051
:10F8400050440020504F520020424F52000A202EB8
:10F850002E6C6173743A000A204372617368657399
:10F860003A00207265663D000A20313256204C690C
:10F870006E653A000A204E45542053746174653A0F
:10F880003078000A2047524E204C65643A000A2026
:10F89000524544204C65643A00444941473A000DC2
:10F8A0000A20506172616E6F69643A000D0A204946
:10F8B000503A005365727665723A0043757272650C
:10F8C0006E743A2000286E6F6E65290D0A0047534A
:10F8D0004D4C4F434B3A200029000D0A2047534D11
:10F8E0002F475052533A204E6F7420636F6E6E65EF
:10F8F0006374656420283078000D0A2047534D3A20
:10F90000204F4B0D0A205365727665723A204E6F78
:10F910007420636F6E6E6563746564000D0A204722
:10F920005052533A204F4B0D0A2053657276657240
:10F930003A20436F6E6E6563746564204F4B000D13
:10F940000A2047534D3A000D0A2050617373776FB8
:10F9500072643A000D0A20557365723A000D0A2050
:10F9600041504E3A00475052533A000D0A20566516
:10F970006869636C65547970653A200056656869FA
:10F98000636C653A000D0A204E6F746966696361A5
:10F9900074696F6E733A000D0A20556E6974733A7C
:10F9A000000D0A2056656869636C65547970653A84
:10F9B000000D0A2056656869636C6549443A004D3C
:10F9C0006F64756C653A003A000A00506172616DAF
:10F9D000733A002C004D6F64756C65207061737311
:10F9E000776F72643A200052656769737465726557
:10F9F00064206E756D6265723A2000562900562C9F
:10FA0000207265663D004D502D30205041313256F8
:10FA10002042415454455259204F4B2028004D500C
:10FA20002D30205041414C4552542121212031326A
:10FA30005620424154544552592043524954494357
:10FA4000414C2028002520534F432900414C45526A
:10FA50005421212120435249544943414C20534FC2
:10FA600043204C4556454C20415050524F4143484D
:10FA700045442028001A000D0A00220D0A004154B6
:10FA80002B434D47533D2200232000303132333485
:10FA90003536373839414243444546000D0A232064
:10FAA000526573756C74203D20000D0A2320646537
:10FAB00067416D6269656E743A20000D0A232077F4
:10FAC000417661696C3A20000D0A23206361633A34
:10FAD00020000D0A2320696D456E643A20000D0A4E
:10FAE0002320696D53746172743A20002320636887
:10FAF000676D6F643A20000D0A23204D696E75749E
:10FB00006573546F4368617267654341433A0D0AF8
:10FB1000002000232053746F707065642043414EB1
:10FB20002073696D0D0A0023205374617274696E2D
:10FB3000672043414E2073696D0D0A0041542B43E9
:10FB400053510D0041542B4350494E3F0D00415439
:10FB50002B434F50533F0D000A0023202053696D63
:10FB60002054783A200020657374206D696C6573A9
:10FB7000290D0A0020696465616C2C20002520286D
:10FB800000232020534F433A20202020202000290A
:10FB90000D0A0020280023202056494E3A2020201C
:10FBA000202020000D0A0A002320205369676E617F
:10FBB0006C3A2020200020560D0A002320203132EC
:10FBC00056204C696E653A20002320205357495433
:10FBD00043483A202020002F56002F002E002320DB
:10FBE0004669726D776172653A20000D0A232044E0
:10FBF0004941470D0A0A0023204C656176696E670A
:10FC000020446961676E6F7374696373204D6F641C
:10FC1000650D0A002320274D2720434F4D4D414EAF
:10FC200044533A0D0A202000232027532720434F16
:10FC30004D4D414E44533A0D0A2020002320434F9E
:10FC40004D4D414E44533A2048454C50203F2044AE
:10FC5000494147205245534554206F722053202E6E
:10FC60002E2E0D0A000D0A004F564D5344494147B0
:10FC7000000D0A23204E4F5449465920414C415211
:10FC80004D20414C4552540D0A000D0A23204E4F81
:10FC900054494659205452554E4B20414C455254DC
:10FCA0000D0A000D0A23204E4F544946592043485F
:10FCB0004152474520414C4552540D0A001B5B32CE
:10FCC0004A1B5B30313B3031480D23204F564D539A
:10FCD00020444941474E4F5354494353204D4F44CC
:10FCE000450D0A0A002000200D0A5477697A792010
:10FCF000436F6D6D616E64733A0056200043292096
:10FD000000432E2E0043202800503A0042617474B4
:10FD1000657279206D6F6E69746F7220726573659C
:10FD2000742E0052542D5057522D42617474436505
:10FD30006C6C2C0052542D5057522D4261747450EB
:10FD400061636B2C004D502D302048004D00432046
:10FD50000054656D70733A20003A003A2B0043005E
:10FD60002E2E2E004F4B20006D56200053443A009B
:10FD70003F002100566F6C74733A20000A204675CC
:10FD80006C6C206368617267653A20000A205469D0
:10FD90006D653A2000206F7220004F464600436890
:10FDA0006172676520416C6572743A2000554E534C
:10FDB0004554004D617820696465616C2072616E04
:10FDC00067653A20000D204F444F3A200025290056
:10FDD000252E2E00252028000D20534F433A2000C9
:10FDE000206B6D00206D6900202D20000D205261D8
:10FDF0006E67653A20000D2046756C6C2063686163
:10FE00007267653A20004E6F74206368617267699B
:10FE10006E6700206D696E2E000D2046756C6C3A81
:10FE200020000D204348473A20004368617267690B
:10FE30006E672053746F7070656400436861726709
:10FE4000696E6720446F6E65004368617267696E12
:10FE5000672C20546F7070696E67206F6666004370
:10FE600068617267696E67002073733D00206C746F
:10FE7000613D002074613D002074773D00206C7668
:10FE8000613D002076613D000A232076773D002009
:10FE90004449523D0020414C543D00204C4F4E3DC2
:10FEA00000204C41543D000A23204649583D002083
:10FEB00053513D002064723D002064693D00204F95
:10FEC000444F3D00205354533D002C302C00630020
:10FED0004D502D3020004D502D30205041002C3001
:10FEE000004D502D302063004D502D30204852548D
:10FEF0002D5057522D557361676553746174732C7F
:10FF0000302C3836343030000D20446F776E2000AE
:10FF10006D20000D20557020000D20446563656C38
:10FF200020000D20416363656C20002520000D201A
:10FF3000436F6E7374200025002057682F6B6D206F
:10FF4000523D00456666696369656E6379200020ED
:10FF500057680D20446F776E20006D202D002057CC
:10FF6000680D20557020002057680D20446563659A
:10FF70006C20002057680D20416363656C200025CC
:10FF8000202D00206B6D0D20436F6E7374200020B8
:10FF90005768200020576800202B00506F7765724B
:10FFA000202D00495000534D53000A00232073694F
:10FFB0006D2064617461206C696E6520002C002CDA
:10FFC00038363430302C004D502D30204852542DCE
:10FFD0004750532D4C6F672C002C002C302C0063A5
:10FFE000004D502D302000545A004E4C0054430018
:10FFF0004F32005254005641005452002C002C3015
:020000040001F9
:0A0000002C0063004D502D3020004D
:06000A000A0EE66E010E75
:10001000E66E26EC85F00A0EE66EE66A26EC85F0C2
:10002000E5ECACF00501CE6BCF6B0501CD6B0501A6
:10003000BD0EFD6FFC0EFE6F000E8FEC85F0F4C65A
:1000400040FB0B01416942691200FDEC84F0030E94
:10005000E1260B01800E421501E0ABD06A0E006E66
:10006000560E016E010E026E720E066E560E076E71
:10007000010E086E41CB09F042CB0AF0090E0A02CC
:10008000F3CF0AF00902F3CF09F0F4500A260B6A05
:100090000ABE0B6806500924F36E07500A20F46E5E
:1000A00008500B20A3EC85F00800F5CF03F0046A9C
:1000B000056AD890033604360536CBEC84F0090087
:1000C000F5CFDEFF0A00F5CFDDFF0F01406B4BECF3
:1000D00085F0070E0016000E0116050ED8900036AA
:1000E0000136E804FBE100C042FF4BEC85F0030E53
:1000F000D89001320032E804FBE100C041FF010E5C
:10010000F36E020EF3CFDBFFA0EC84F004BE0568B3
:1001100097EC85F0F5CF46FFA0EC84F004BE0568AF
:1001200097EC85F0F5CF47FFA0EC84F004BE05689E
:1001300097EC85F0F5CF48FFA0EC84F004BE05688D
:1001400097EC85F0F5CF49FFA0EC84F004BE05687C
:1001500097EC85F0F5CF4AFFF3DB04BE056897EC1A
:1001600085F0F5CF4BFFECDB04BE056897EC85F01E
:10017000F5CF4CFFE5DB04BE056897EC85F0F5CFC5
:100180004DFF0F01080E456F4087010E0B01412501
:10019000416F000E4221426F110E2D6E2E6A41CB2F
:1001A00028F042CB29F0CEEC8CF024C041FB25C0D6
:1001B00042FB040E0501FA15006E040E50EC85F0AA
:1001C0000AE00501A30EFD6FFC0EFE6F000E55EC5C
:1001D00085F0FA95FB95100EFA15006E100E50EC96
:1001E00085F00AE005018A0EFD6FFC0EFE6F000E21
:1001F00055EC85F0FA99FB99200EFA15006E200E49
:1002000050EC85F00AE00501710EFD6FFC0EFE6FEB
:10021000000E55EC85F0FA9BFB9B030EE15C02E2BD
:10022000E16AE552E16EEED3E8DB020EE126E66A12
:1002300051ECA8F0E552F3CFDEFFF4CFDDFFEDDBAC
:1002400010E0140EE66EE66ADECFE6FFDDCFE6FFD5
:1002500058EC85F09EEC9FF0006E060EE15E0050BB
:100260000AD0680EE66EFC0EE66E58EC85F006ECE1
:100270009FF05DEC85F09DDBC9DB40EC9FF0E55223
:10028000E552F350E66EC2DB58EC85F076EC62F096
:10029000006E050EE15E0050020EE15C02E2E16AD2
:1002A000E552E16EAFD3A9DB84DBB0DBB6EC34F012
:1002B000E552E5520A01A451A51105E00A01645175
:1002C00002E186EC36F09ED398DB73DBC4DB3C0E98
:1002D000FD6FFC0EFE6F000E8FEC85F00501280E01
:1002E000FD6FFC0EFE6F000E8FEC85F088EC85F044
:1002F00088EC85F099DFE1DB0501140EFD6FFC0E43
:10030000FE6F000E8FEC85F0E66A26EC32F0E552C7
:1003100079D373DBE66A010EE66E98DBE66AE66A7D
:1003200095DBE5ECACF045DB96DBF70EFD6FFB0EE5
:10033000FE6F000EF4DB0A0EF5DB42EC72F062D3C6
:100340005CDB050EE126010EF36E020EF3CFDBFF40
:10035000F36EDB6E0501EB0EFD6FFB0EFE6F000E04
:10036000DEDB0E0EF66E000EF76E000E69DBDE0EA3
:10037000E66EFB0EE66E000EDDEC85F00F0EF66EFF
:10038000000EF76E000EC4EC85F0100EF66E000E37
:10039000F76E000EC4EC85F00E0EE66E51ECA8F080
:1003A000E552F3CF00F0F4CF01F0F3CFE6FFF4CF46
:1003B000E6FF3BDBBAEC74F0026E070EE15E025022
:1003C00091DB0701CC51CD11CE1107E0CCC7E6FF80
:1003D000CDC7E6FFCEC7E6FFDFDB020EDBCFE6FFD1
:1003E000E66AD70EE66EFB0EE66E000EE66E6FDB7B
:1003F00087DBFCECB1F0E66EE66AC90EE66EFB0E3A
:10040000E66E000EDEDA7CDB01ECB2F026C000F016
:1004100027C001F028C002F029C003F02C6A2D6A21
:10042000200E2E6E410E2F6E26C027F001C028F040
:1004300002C029F003C02AF047EC8CF0E3EC8DF009
:1004400028C0DEFF29C0DDFF010EE66EE66A23DB71
:10045000026A036A8ADB02C0E6FF03C0E6FFBB0E46
:10046000E66EFB0EE66E000EACDAC8EC75F0046EBC
:100470000B0EE15E045036DBB60EE66EFB0EE66E4A
:10048000000E7CDA0901E951E66EE66AA80EE66E16
:10049000FB0EE66E000E91DBA40EE66EFB0EE66E22
:1004A000000E6CDAAE0EE66E090EE66E960EE66E85
:1004B000FB0EE66E000E85DAC0DAC80EE66E060E9A
:1004C000E66E930EE66EFB0EE66E000EE66EFFDA4B
:1004D000B4DA8F0EE66EFB0EE66E000E4FDA0901FF
:1004E000A051E66EE66A810EE66EFB0EE66E000E29
:1004F00064DBA1C9E6FFA2C9E6FF7D0EE66EFB0E36
:10050000E66E000E74DBA3C9E6FFA4C9E6FF740E15
:10051000E66EFB0EE66E000E6ADB660EE66EFB0E06
:10052000E66E000E2BDA0B01800E42150FE141CB77
:10053000E6FF42CBE6FF5A0EE66EFB0EE66E000EBD
:100540003CDB110EE66EE66A70DADADA0501580E67
:10055000FD6FFB0EFE6F000E63DA4E0EFD6FFB0E9D
:10056000FE6F000E5DDA440EFD6FFB0EFE6F000E97
:1005700057DA3C0EFD6FFB0EFE6F000ED0DA050E53
:10058000E15C02E2E16AE552E16E3CD236DA3EDA43
:10059000F1DAF3CFE9F936D230DAF4C640FB0601DE
:1005A000010EF46FA7EC9BF00B01416B426B050150
:1005B000270EFD6FFB0EFE6F000E08D31EDA40CB38
:1005C000F4F6A7EC9BF00B01416942690501130E9B
:1005D000FD6FFB0EFE6F000EF9D20FDA0E0EE12654
:1005E000B8DA14DAE2DAF350DF6ECCD9DE52F3CFA8
:1005F000DEFFF4CFDDFFDD52C5D974DAC3D9050EB5
:10060000F3CFDBFF060EF4CFDBFFBCD9070EF3CF31
:10061000DBFF080EF4CFDBFFB5D9090EF3CFDBFF0C
:10062000DBCFE6FF1CDA22DA52DA27DADFCFE6FF89
:1006300016EC6DF0006E0A0EE15E00500A0EF3CF6C
:10064000DBFF0B0EF4CFDBFF0501F70EFD6FFA0E9B
:10065000FE6F000E64DADFCFE6FFE66AEC0EE66EB0
:10066000FA0EE66E000EADD9B5DA07DADE0EE66EEA
:10067000FA0EE66E000E99D92ADAD20EE66EFA0E5E
:10068000E66E000E92D9F2D9C80EE66EFA0EE66E4C
:10069000000E8BD9E4D9BB0EE66EFA0EE66E000EA4
:1006A00084D9090EDBCF00F0016A00BE01685DDA73
:1006B000AA0EE66EFA0EE66E000EE66E1ADAC2ECCE
:1006C00074F0026E070EE15E02508ADA0A0EDBCF8A
:1006D000E6FF0B0EDBCFE6FF9C0EE66EFA0EE66E33
:1006E000000E63D9650EE66EFC0EE66E000EE66E39
:1006F00000DA8CEC74F0006E050EF0D91BDA0E0EE9
:10070000E15C02E2E16AE552E16E7CD176D9040E49
:10071000E1266CD9EF5001E10CD168D9EF502308E4
:1007200001E107D1FD0EDBCFDEFFDBCFDDFF75D9A9
:1007300018E073D9200815E070D960080DE21FDABF
:10074000EFCF00F07B0E005C07E267D9E00FE66EAA
:1007500016DAE552E750EF6EDF2A010EE8E3DB2AF6
:10076000E6D75BD9200804E1DF2A010E01E3DB2A8A
:10077000020EDB6A030EDB6A0B0E006E570E016E73
:10078000010E026E020EDBCF03F0030EDBCF04F08E
:10079000056A04BE056896D903C027F004C028F096
:1007A00005C029F073EC8DF024C003F025C004F0DF
:1007B00026C005F000502424F36E01502520F46E6D
:1007C00002502620C0D90800F55001E1A0D00B0E40
:1007D000056E570E066E010E076E020EDBCF08F097
:1007E000030EDBCF09F00A6A09BE0A686BD908C09C
:1007F00027F009C028F00AC029F073EC8DF024C05E
:1008000008F025C009F026C00AF005502424026E25
:1008100006502520036E07502620046E02C0E6FF16
:1008200003C0E6FFE66E4EEC9FF0E552E552E5525E
:1008300027C000F028C001F027C0E6FF28C0E6FF6F
:100840000B0E0E6E570E0F6E010E106E020EDBCFEA
:1008500011F0030EDBCF12F0136A12BE136832D907
:1008600011C027F012C028F013C029F073EC8DF0EE
:1008700024C011F025C012F026C013F00E5024241D
:100880000B6E0F5025200C6E105026200D6E0BC0E5
:10089000E6FF0CC0E6FFE66E3BD92EEC9EF0146E30
:1008A000070EE15E145000092BE1020EDBCFE9FFD9
:1008B000030EDBCFEAFFEA02F3CFEAFFE902F3CF50
:1008C000E9FFF450EA26430EE9260B0EEA22EECFAA
:1008D00000F0EECF01F0EFCF02F0DECFE6FFDDCF8C
:1008E000E6FFFD0EDBCFE6FFFE0EDBCFE6FF06D018
:1008F00002C0FBFF01C0FAFF0050F96EF9DF18D00B
:10090000020EDB2A030E01E237D7DB2A35D76ED879
:10091000EF50530805E124D903E159D885DC08D00C
:1009200065D8EF504D0805E11BD903E150D8BBDC79
:10093000C4D8040EE15C02E2E16AE552E16E62D0E5
:10094000720E006E560E016E010E026E020EDBCFAD
:10095000F3FFDB2AF350066E076A090E286E296A38
:1009600041CB2DF042CB2EF028EC8DF02650062402
:10097000036E27500720046E056A1200E66E0CD93C
:100980009AEF85F0E6D8000EE66EE66AD5EF85F0C0
:10099000C2EC74F015D100500324F36E0150042012
:1009A000F46E02500520A3EF85F0E66EA2D8EAEFC0
:1009B00085F00501650EFD6FFC0EFE6F000E8FEFDA
:1009C00085F0E66E000EE66E060EE66E1200020E72
:1009D000E76EFD0EDBCF00F0FE0EDBCF01F0E7503F
:1009E0000026000E0122C1D888EF85F0FD0EDBCF76
:1009F000E9FFFE0EDBCFEAFF1200D9CFE6FFE1CF21
:100A0000D9FF1200E552E7CFD9FF1200FB0EDBCF72
:100A1000E6FFFC0EDBCFE6FF1200B1D8EF5012006C
:100A20007ED8050E7FD805011200DA0EE66EFB0EA9
:100A3000E66E000EE66E67EF85F0BAEC74F0C0D09B
:100A4000F86E0800F550E66EE66A1200BEECACF0F7
:100A5000E552E5521200010E65D805011200070E9D
:100A6000DBCFE6FF080EDBCFE6FF1200050EDBCF83
:100A7000E6FF060EDBCFE6FF1200010EDBCFE6FF3E
:100A8000020EDBCFE6FF1200E750E926000EEA2255
:100A9000EF5020081200DECF00F0DDCF01F0120091
:100AA000FB15016E00500110120039D8050112002B
:100AB000D60EE66E050EE66E1200E552E552E552E0
:100AC000E55212001B0E2C6E2D6A2E6A1200030EC8
:100AD000DBCFE6FF040EDBCFE6FF1200E15E005045
:100AE000F0EF85F0030EF3CFDBFF040EF4CFDBFF56
:100AF00012000C0EDBCFE6FF0D0EDBCFE6FF12007F
:100B000047DF650EE66EFC0EE66E000EBEEF84F06B
:100B1000FD0EDBCFE6FFFE0EDBCFE6FF1200FF6F20
:100B2000FEEF3EF0E66E62EC72F0E552120033DF4B
:100B300008001200000EE66E060EE66E4DEC3FF069
:100B4000E552E5521200F86EF4CFF7FFF3CFF6FF4F
:100B50001200110EE66EFB0EE66E000EE66E12003F
:100B6000010EE76E43DF44EF85F000C0E6FF01C0F1
:100B7000E6FF12007EEC92F0E552E5521200DECF65
:100B8000E9FFDDCFEAFF12005BDFDC0EE66EFB0E55
:100B9000E66E000EF7EF85F09ADF8CEC74F0006ED5
:100BA000050EE15E005072EF85F018ECAEF0006EBD
:100BB000050E94DF9EDFBAEF85F003DFC8EF84F007
:100BC000006E070EE15E005072EF85F0A8DF020EA6
:100BD000A9DF18D7C2EC74F0006E070E6EEF85F037
:100BE0000C0EF3CFDBFF0D0EF4CFDBFF1200E66E31
:060BF0006EDFC8EF84F087
:0A0BF600DEEC8AF0030EE126020E89
:100C0000DB6A000E0901E76EE119E8AE02D0E135BA
:100C100003D0E750D880E15501E2E107000E090159
:100C2000E76EE219E8AE02D0E23503D0E750D88093
:100C3000E25501E2E20709010A51000807E20A074A
:100C400003E109019B9102D009019B810901A52BB8
:100C5000000EA623A723A8230901905157E00901FC
:100C60008E518F1153E0090199B715D00C0E9913CD
:100C70000901966B0901976B0901010E946F090137
:100C8000030E956F0901100E916F0901926B936B22
:100C90000901986B5FD00901052B3C0E055D63E3EC
:100CA000056B0901922B000E932309019051026EEE
:100CB000036A90C928F003C029F08EC92DF08FC9AE
:100CC0002EF055EC8DF026C000F027C001F0000199
:100CD0002650090106270001275009010723000EAD
:100CE00008230923600E065DEA0E0759000E085915
:100CF000000E095938E30901982B600E0901065FBF
:100D0000EA0E075B000E085B095B2DD009019051CC
:100D10002AE109018E518F1126E1090199A723D0FB
:100D2000F30E99170901966B0901976B5F0E090184
:100D3000A05D0AE20901150E946F09010E0E956F70
:100D4000040ECDEC8AF006D00901040E946F09015F
:100D5000030E956F0901056B066B076B086B096B3A
:100D6000020ECDEC8AF009010F5119E0010EE66E7A
:100D700062EC72F0E55212EC2EF0100EE66E090EE7
:100D8000E66E000EE66E060EE66E06EC9FF0E5528D
:100D9000E552E552E5523FEC2EF009010F6B04518C
:100DA00008E10901905105E109018E518F1101E11E
:100DB00092D00601F45101E18ED0DE6ADD6A9ADB41
:100DC00006BE076819EC8BF00050011001E181D0DC
:100DD000280E046E650E056E010E066EDECF07F05E
:100DE000DDCF08F0096A08BE0968050E2C6E2D6A71
:100DF0002E6A07C027F008C028F009C029F073EC5C
:100E00008DF024C007F025C008F026C009F004507A
:100E10002424F36E05502520F46E06500BEC8BF065
:100E2000020EE0DB0800F550026E036AC8C728F026
:100E3000C9C729F02D6E03C02EF0ABECB2F024C070
:100E400000F025C001F0245025103DE1020EDB50DA
:100E500002E053EC72F00F0140B7FDD7406B4ADB64
:100E600006BE0768E6DB070E0016000E0116050E2B
:100E7000D89000360136E804FBE100C042FF3ADBBF
:100E800006BE0768D6DB030ED89001320032E804B4
:100E9000FBE100C041FF0F01030E466F220E476FBA
:100EA00029DB06BE0768B2DB01C000F0016A00C0A2
:100EB00048FF20DB06BE0768A9DB005052DBF36E5B
:100EC000020EF3CFDBFFDF2A010E01E278D7DB2A27
:100ED00076D70901046B000E006E030EE15C02E29E
:100EE000E16AE55238D36ADB080EE1266250026EF1
:100EF000036A050ED89003320232E804FBE1615028
:100F0000046E056A030ED89004360536E804FBE14A
:100F100002500424006E03500520016E060E00C02E
:100F2000DBFF070E01C0DBFF0F0E65140801E76F42
:100F300066CFE8F867CFE9F868CFEAF869CFEBF851
:100F40006ACFECF86BCFEDF86CCFEEF86DCFEFF821
:100F5000609E09013C0E0A6FEAC803F0026A0801AC
:100F6000EB510224006E000E032000C0DEFFDD6E98
:100F7000020EECC8DBFFDECF00F0DDCF01F009018F
:100F80000D51001854E10E51011851E1060EDBCF4E
:100F900002F0070EDBCF03F00B51021848E10C51B1
:100FA000031845E10F5143E1E10EE66EFF0EE66ED8
:100FB000000EE66E100EE66E090EE66E8CEC74F016
:100FC000006E050E1ADB2E0EE66EE66ADF0EE66E8A
:100FD000FF0EE66E000E81DA060EDBCFE6FF070E8F
:100FE000DBCFE6FFDB0EE66EFF0EE66E000E75DA77
:100FF000DECFE6FFDDCFE6FFFADA6FDA030EDB6A5B
:10100000080EF36E030EDBCFF4FFF350F45C08E23E
:10101000030E98DAE66AEBDA60DA030EDB2AF0D721
:101020000901010E0F6F0B6B0C6B0D6B0E6B620EDB
:101030000801E95D02E0010EDED0D950060FE96E2D
:10104000DACFEAFFEC0EEE1801E091D0070EED18B2
:1010500001E08DD0000EDFCF28F0010EDBCF29F0AC
:10106000340E281802E1830E291859E0430E28187F
:1010700002E11C0E29184FE04F0E281802E1430E22
:10108000291845E01E0E281802E1800E29183BE0C1
:101090001F0E281802E1800E291827E0680E281874
:1010A00002E1430E291818E0690E281801E0A2D0C9
:1010B000430E291801E09ED0020EDB50006E016A3B
:1010C000050E2D6E2E6A00C028F001C029F0ABEC91
:1010D000B2F028C090F98ED0020EDB5009018E6F5D
:1010E0008F6BD8908E378F3785D009013C0EE16F1A
:1010F000020EDB50E8307F0B006E280E005E000E03
:1011000000C0ADF977D009013C0EE26F73D04CDA24
:1011100000C0C2F96FD048DA00C0C0F96BD0090135
:101120003C0EE26F020EDB50270DF3CF00F0F4CF40
:1011300001F0630E50DACEEC8CF028C000F029C02C
:1011400001F028C0A0F909012850250DF3CFA1F91D
:10115000F4CFA2F9640E3FDAABECB2F028C0A1F9EB
:1011600029C0A2F928C0A3F929C0A4F943D0D950B5
:10117000060FE96EDACFEAFFE80EEE183BE1070E44
:10118000ED1838E1D9CFE9FFDACFEAFF0D0EEE18FE
:1011900031E1EE502FE14B0E0701CB5D04E1020E71
:1011A000DBCF9FF927D0020EDBCF26F0276A286A13
:1011B000296AE80E2B6E030E2C6E2D6A2E6ABEEC89
:1011C000B1F022C026F023C027F024C028F025C0AB
:1011D00029F0F40E2626010E2722000E28222922AD
:1011E000490E2B6E060E2C6E2D6A2E6A53ECB2F051
:1011F00026C09FF9010E006E080EE15C02E2E16A72
:10120000E552A9D1DBD9020EE1260F0E0F015515CB
:101210000801E76F56CFE8F857CFE9F858CFEAF85A
:1012200059CFEBF85ACFECF85BCFEDF85CCFEEF886
:101230005DCFEFF850CFDFFF0F01509F0901010E86
:10124000046F3C0E0A6F070EDF14020850E0070E11
:10125000DF1403080EE1010EDB6AB5D907E2010EC7
:1012600071D9010EDB50090F87D9F7D70901BF6B80
:101270003ED0070EDF1404080DE10901310EAE6FF8
:10128000010EDB6AA0D933E2010E5CD9010EDB2826
:1012900073D9F8D7070EDF14050829E10801E851D2
:1012A00017E10901998D999F0901A951AA11AB1163
:1012B000AC111DE1A5C9A9F9A6C9AAF9A7C9ABF93D
:1012C000A8C9ACF9A907000EAA5BAB5BAC5B0DD05B
:1012D0000901999D998F0901A951AA11AB11AC116E
:1012E00006E0A96BAA6BAB6BAC6B010E56D9010E75
:1012F000006E020EE15C02E2E16AE5522CD15ED999
:10130000FC0EDBCF28F0FD0EDBCF29F02E0E2818C7
:101310004CE129504AE16BD9E66E84D9F7D80CE04C
:1013200036D9F3CF0BF9F4CF0CF961D9E66E000E84
:10133000E66EE66AEBD802E1000E38D028D9F3CF8A
:101340000DF9F4CF0EF909010F6B53EC72F00F0198
:1013500040B7FDD7406B070E09010B15006E016AFF
:10136000050ED89000360136E804FBE100C042FFCC
:101370000BC900F00CC901F0030ED8900132003205
:10138000E804FBE100C041FF080E09010B27000E35
:101390000C230F01030E466F220E476F016A0EC920
:1013A00048FF09010D51DDD801D0000EE552E7CF0D
:1013B000D9FF1200D9CFE6FF020EE1260601560E34
:1013C000C86F410EC96FCA6BCB6BCC6B0901DC0EC9
:1013D000006FDA0E016FD40E026F340E036F046BD0
:1013E000056B066B076B086B096B0A6B0B6B0C6B61
:1013F0000D6B0E6B0F6B0901E5690901A56BA66BFF
:10140000A76BA86B900E6F6E6EAEFED7606A0F0171
:10141000196B1869016BFD0E006F506BE00E1D6FAC
:101420001C69C00E096F400E086F200E0D6F9C0ED8
:101430000C6F800E116FA20E106FA00E156F260E8E
:10144000146F010E706ED20E716E020E726E200E4F
:10145000736E0601F451000802E26F6A02D0600E5A
:101460006F6E0701E60ED56F0E0ED66F010ED76FA9
:101470000701040ED86F120ED96F010EDA6F070143
:10148000F60EDB6F0B0EDC6F010EDD6F0801FE0E3A
:10149000F06F120EF16F010EF26F0501EE81EE8317
:1014A000010E006E020EE15C02E2E16AE55253D0E9
:1014B000050E2C6E2D6A2E6A05C027F006C028F096
:1014C00007C029F073EC8DF002502424F36E035012
:1014D0002520F46E04500BEF8BF0E66E040EDBCF8C
:1014E000E6FF050EDBCFE6FFC2EC74F0006E070EE0
:1014F000FDEF8AF0280E026E650E036E010E046E7B
:10150000DECF05F0DDCF06F0076A120018ECAEF072
:10151000006E050EE15E0050FA0EF3CFDBFFFB0E0E
:10152000F4CFDBFFD950FA0FE96EFF0EDA20EA6E36
:10153000EE50ED1012000900F5CF00F00800F5CFD5
:1015400001F01200DB50EA6AE80FE96E080EEA22A9
:10155000EF50E66E1200E16E0050E552E7CFD9FF82
:1015600012000F01496F4A6B4B6B4C6B4D6B080EB1
:10157000456F406F010E1200EA6AAE0FE96E090E68
:10158000EA22E552E750EF6E010EDB2A12004AD83C
:101590007EEC92F0E552E5521200E66EE66AE3EC6C
:1015A0003FF0E552E552120009013C0EE26F020ED7
:1015B000DB50006E280E005E000E1200D9CFE6FF51
:1015C000E1CFD9FF1200080EF36E010EDBCFF4FF5E
:1015D000F350F45C12002D6E2E6AF3CF28F0F4CF96
:1015E00029F01200F626000EF722F8221200D90E7A
:1015F000E66EFF0EE66E000E1200E15E0050040E75
:10160000F3CFDBFF050EF4CFDBFF120051DF030E3B
:10161000E9DF9BEF8AF02620F86EF4CFF7FFF3CFD7
:10162000F6FF1200FA0EDBCFE6FFFB0EDBCFE6FF84
:0816300012003EDF9BEF8AF07F
:08163800219E05D0219E29AE80
:1016400002D0296C218E29C023F0226A336A326AC3
:10165000860E246E256AC3EF8EF0219E08D0219E4F
:1016600029AE05D0286C291EE86A2922218E29C0BE
:1016700023F028C022F0336A326A8E0E246E256A67
:10168000C3EF8EF0219E0CD0219E29AE09D0266C8E
:10169000271E281E291EE86A272228222922218E99
:1016A00029C023F028C022F027C033F026C032F032
:1016B0009E0E246E256AC3EF8EF02F7E216AFFEC0A
:1016C0008EF017EC8FF021B6A7EF8EF021A20AD092
:1016D00021AA03D021BEA7EF8EF021A4B3EF8EF094
:1016E000B0EF8EF021AA05D021ACB3EF8EF0B0EFB1
:1016F0008EF021A00AD021A808D021BE04D021A4B8
:1017000002D0BCEF8EF0C0EF8EF0326A256A2F5007
:101710002A5C316E10E327C033F028C022F029C0C4
:1017200023F02AC030F02CC027F02DC028F02EC0A6
:1017300029F0213A09D02CC033F02DC022F02EC060
:1017400023F02FC030F0316C219E21BC218E30C09F
:1017500024F021B0EFEF8EF01A0E3160EFEF8EF033
:10176000246A2A6A21A408D0276C281E291E2A1E52
:10177000E86A282229222A2221AC08D0336C221EB2
:10178000231E241EE86A222223222422266A3152A2
:1017900007E02A342932283227322632312EF9D76F
:1017A0002750332628502222295023222A5024222F
:1017B00026C032F0219E24AE0BD0326C331E221E86
:1017C000231E241EE86A3322222223222422218E71
:1017D00024A006D0D8802332223233323232302A4B
:1017E00030C024F0C3EF8EF0216AFFEC8EF017ECCE
:1017F0008FF021B6A7EF8EF021A205D021BAA7EF76
:101800008EF0AEEF8EF021BABAEF8EF021A005D0A7
:1018100021B8A7EF8EF0BAEF8EF021B8AEEF8EF0C0
:10182000256A7F0E2A24246EE86A25222F50245E22
:10183000E86A255A1A0E306E2A6A326A336A226AB8
:10184000236A2C50275E2D50285A2E50295A000EFC
:101850002A5A09E72C5027262D5028222E502922BB
:10186000000E2A2201D0328AD8902736283629360F
:101870002A36D8903236333622362336302EE1D708
:10188000295028102710D8A4328AC3EF8EF0216A7D
:10189000FFEC8EF017EC8FF021B6A7EF8EF021A2AF
:1018A00005D021B8A7EF8EF0AEEF8EF021AA05D0BB
:1018B00021B0A7EF8EF0AEEF8EF021B002D021A8BC
:1018C00002D0BAEF8EF0256A2F502A24246EE86ADF
:1018D00025227E0E245EE86A255A326A336A226A1D
:1018E000236A2E502902F4CF23F0F3CF22F02D509B
:1018F0002902F3503326F4502222000E23222E50C8
:101900002802F3503326F4502222000E23222C50BA
:101910002902F3503226F4503322000E22222322D1
:101920002D502802F3503226F4503322000E22228A
:1019300023222E502702F3503226F4503322000E79
:10194000222223222C502802F4503226000E332269
:10195000222223222D502702F4503226000E332259
:1019600022222322C3EF8EF0206A2EAEBAEF8CF033
:101970002E6C201E29AEBFEF8CF0296C201EEFECE0
:10198000B2F029BEC9EF8CF020AE000C296C256C9A
:10199000000C20BEC6EF8CF02188FF0C206A2EAE12
:1019A000D7EF8CF02D6C2E1EE86A2E22201E29AE59
:1019B000DFEF8CF0286C291EE86A2922201EABEC90
:1019C000B2F029BEEFEF8CF020AE000C286C291E7F
:1019D000E86A2922246C251EE86A2522000C20BE14
:1019E000E6EF8CF02188FF0C206AE86A2EAE01EF4A
:1019F0008DF02B6C2C1E2D1E2E1E2C222D222E2205
:101A0000201E29AE0CEF8DF0266C271E281E291EE5
:101A1000272228222922201E53ECB2F029BE23EFD0
:101A20008DF020AE000C266C271E281E291EE86AA9
:101A3000272228222922226C231E241E251E23222F
:101A400024222522000C20BE13EF8DF02188FF0CEC
:101A500029C033F028C032F028502D02F4CF27F0EF
:101A6000F3CF26F029502E02F4CF29F0F3CF28F03F
:101A70002D02F3502726F4502822E86A29223250FA
:101A80002E02F3502726F4502822E86A29222EAE8F
:101A90004EEF8DF03250285E3350295A33AE000C91
:101AA0002D50285E2E50295A000C28C032F02850A4
:101AB0002D02F4CF27F0F3CF26F029502E02F4CFD9
:101AC00029F0F3CF28F02D02F3502726F4502822D6
:101AD000E86A292232502E02F3502726F450282299
:101AE000E86A2922000C29C033F028C032F027C050
:101AF00031F027502C02F4CF25F0F3CF24F02850FA
:101B00002D02F4CF27F0F3CF26F02C02F350252638
:101B1000F4502622E86A272231502D02F350252660
:101B2000F4502622E86A272229502C02F350262658
:101B3000F450272229502D02286AE86A2822F350FF
:101B40002726F450282231502E02F3502626F45036
:101B50002722296AE86A2822292232502E02F350CD
:101B60002726F4502822E86A292233502E02F35007
:101B70002826F4502922000C216AFFEC8EF021B6B1
:101B8000C6EF8DF021A20AD021B403D07F0E296EBA
:101B900019D0800E296E16D0296A14D021B0FCD736
:101BA000870E2A60F1D77E0E2A64F6D7860E2A5C4D
